:020000040800F2
:1000000078C80220D1010008394000083B360008BA
:1000100089360008950E00086553000800000000AE
:10002000000000000000000000000000874D0008F4
:10003000F10F0008000000005B4000080D4E0008B2
:10004000EB010008EB010008EB010008EB010008E0
:10005000EB010008EB010008EB010008EB010008D0
:10006000EB010008EB010008EB010008EB010008C0
:10007000EB010008EB010008EB010008EB010008B0
:10008000EB010008EB010008EB010008EB010008A0
:10009000EB010008EB010008EB010008EB01000890
:1000A000EB010008EB010008EB010008EB01000880
:1000B000EB010008654E00089D4E0008EB010008AA
:1000C000EB010008EB010008EB010008EB01000860
:1000D000EB010008F9520008EB010008EB010008F1
:1000E000EB010008EB010008EB010008EB01000840
:1000F000EB010008EB010008EB010008EB01000830
:10010000EB010008EB010008EB010008EB0100081F
:10011000EB010008EB010008EB010008EB0100080F
:10012000EB010008EB010008EB010008EB010008FF
:10013000EB010008EB010008EB010008EB010008EF
:10014000EB010008EB010008EB010008EB010008DF
:10015000EB010008EB010008EB010008EB010008CF
:10016000EB010008EB010008EB010008EB010008BF
:10017000EB010008EB010008EB01000800000000A3
:10018000EB010008EB010008EB010008EB0100089F
:10019000EB010008EB010008EB010008EB0100088F
:1001A000EB010008EB010008EB010008DFF80CD0C0
:1001B00000F02EFC00480047D9A4000878C80220AF
:1001C00030BF72B6704762B6704780F308887047D8
:1001D0000648804706480047FEE7FEE7FEE7FEE7E1
:1001E000FEE7FEE7FEE7FEE7FEE7FEE7114E00084A
:1001F000AD0100082DE9F05F0546002092469B46C0
:1002000088460646814640241BE02846414647462C
:10021000224600F02BF953465A46C01A914110D39A
:1002200011461846224600F012F92D1A67EB010814
:100230004F4622460120002100F009F917EB000982
:100240004E41201EA4F10104DFDC484631462A4617
:100250004346BDE8F09F40EA01039B0703D009E055
:1002600008C9121F08C0042AFAD203E011F8013BA2
:1002700000F8013B521EF9D27047D2B201E000F8FB
:10028000012B491EFBD270470022F6E710B513463A
:100290000A4604461946FFF7F0FF204610BD421EED
:1002A00012F8013F002BFBD111F8013B02F8013B92
:1002B000002BF9D17047421C10F8011B0029FBD11B
:1002C000801A704710B5002200E0521C835C8C5CE1
:1002D000A34201D1002BF8D1D8B2E1B2401A10BD2F
:1002E0002DE9FE4F81EA030404F0004421F00041AF
:1002F00000944FF0000B23F0004350EA01045ED05D
:1003000052EA03045BD0C3F30A54C1F30A552C44E8
:10031000A4F2F3340194A0FB0254C1F3130141F49D
:100320008011C3F3130343F4801301FB024400FB69
:10033000034E840A970A44EA815447EA8357A4FB90
:10034000076802958D0A05FB07854FEA932C04FB8D
:100350000C542705029D4FEA065847EA1637B5EBBD
:1003600008056EEB070C870E920E47EA811742EAEA
:100370008312A7FB0201B6EB0B0164EB00042B0D0B
:1003800043EA0C335E1844EB1C50DA465146E7FB57
:100390000201C5F313044FEA0B3343EA14534FEA47
:1003A0000432019C43EA0603A4F10C040294009C6D
:1003B000CDE900B400F0FEF803B0BDE8F08F0020F6
:1003C0000146F9E700F0004230F000400AD0C10DCC
:1003D00001F56071C0F3160042EA0151C2084007FE
:1003E0001143704700200146704701F0004330B4CC
:1003F00021F0004150EA010206D00A0DA2F5607218
:10040000C1F31301002A02DC30BC00207047440F06
:1004100044EAC104C100E01830BC00EBC25000F057
:1004200083B830B50B46014600202022012409E0A4
:1004300021FA02F59D4205D303FA02F5491B04FA9D
:1004400002F52844151EA2F10102F1DC30BD202A7C
:1004500004DB203A00FA02F1002070479140C2F11B
:10046000200320FA03F3194390407047202A04DB4D
:10047000203A21FA02F00021704721FA02F3D0401D
:10048000C2F1200291400843194670470FB400237F
:1004900000B589B00CA900910B996FF00042CB60B8
:1004A0001E4B06931E4B07930423CDE901321D4AD0
:1004B000089202466B46002000F054FB09B05DF83C
:1004C00014FB70B586B006464FF0FF300091CDE9C1
:1004D0000101002015460C4604903246694604A8E6
:1004E000FFF7D4FF02460498211825B108B1084649
:1004F00000E020462860049800280DD0002A02DD84
:100500000098884208D0081B0094CDE901043246C7
:10051000694604A8FFF7BAFF06B070BD9D0D00083C
:10052000BB0D0008590A00080029A8BF7047401CED
:10053000490008BF20F00100704710B4B0FA80FCF9
:1005400000FA0CF050EA010404BF10BC704749B136
:10055000CCF1200421FA04F411FA0CF118BF0121A6
:1005600021430843A3EB0C01CB1D4FEA00614FEA86
:10057000102042BF002010BC704700EBC350104455
:100580000029A4BF10BC7047401C490008BF20F0E0
:10059000010010BC704710B5141E73F1000408DA96
:1005A000401C41F1000192185B411A4301D120F037
:1005B000010010BD2DE9F04D92469B4611B1B1FAF4
:1005C00081F202E0B0FA80F220329046FFF73FFF5E
:1005D00004460F4640EA0A0041EA0B0153465A46D8
:1005E000084313D0114653EA010019D0C8F1400264
:1005F0005046FFF73BFF05460E46504659464246D9
:10060000FFF725FF084305D0012004E020463946C6
:10061000BDE8F08D0020054346EAE0762C433743E1
:100620000A986305E40AA0EB08000022FD0A44EAE8
:1006300047540A3002D500200146E9E701051019A8
:100640006941DDE9084500196941BDE8F04DA2E7BF
:100650002DE9FE4F804681EA0300C00F0C46009052
:1006600021F0004123F00045B8EB0200A94105D27A
:100670004046214690461C460B46024623F0004069
:10068000104347D0270DC7F30A00C3F30A51029065
:10069000401A019040286BDAC3F3130040F4801B2A
:1006A0000098924620B10023D2EB030A63EB0B0BB8
:1006B00001985946C0F140025046FFF7C8FE064671
:1006C0000D4650465946019A00F0B4F910EB080067
:1006D0006141002487EA115284EAE7731A4340D04B
:1006E000009A62B3019A012A4FEA075215DC001BF7
:1006F00061EB02014FF0004202EA0752CDE90042ED
:10070000001C41F5801132462B46FFF753FF03B022
:10071000BDE8F08F40462146F9E7001B61EB02017E
:10072000001C41F5801300185B412018A2F500174A
:1007300047EB030140EAD570B6196D4111E06D0831
:100740004FEA360645EAC0754FEA0752001B61EBD7
:100750000201001C41F5801149084FEA30000019E0
:10076000514132462B4603B0BDE8F04FFFF713BFAF
:100770000098012240000023D0EB020263EBE073FB
:10078000009821464FEAE074B8EB000061EB0401E9
:10079000E9E783F000435BE781F0004158E72DE98A
:1007A000F04D81EA030404F0004B21F000451446AB
:1007B0004FF0000A23F0004150EA050220D054EA2D
:1007C00001021DD0C5F30A570246C5F31303C1F356
:1007D0001300C1F30A5640F4801543F48013A7EBCD
:1007E0000608101BD64608F2FD3873EB050002D34D
:1007F00008F1010801E092185B41B8F1000F03DA3B
:1008000000200146BDE8F08D00204FF4801106461F
:1008100084460EE0171B73EB050705D3121B63EB31
:10082000050306434CEA010C49084FEA30009218D0
:100830005B4150EA0107EDD152EA030012D082EA8F
:10084000040083EA0501084305D0101BAB4106D222
:100850000122002306E000224FF0004302E06FF087
:10086000010253101AEB06004CEB085110EB0A0082
:1008700041EB0B01BDE8F04DFFF78DBE2DE9F04DCA
:1008800000231A461B1A8A4103DB00200146BDE8FB
:10089000F08DC1F30A52C1F3130141F480154FF0FA
:1008A000000BD10702D100186D41521E00270446EB
:1008B00040F2FF11384601EB620A3E46804602468E
:1008C00000204FF48011FFF7D1FDC2197141BB1810
:1008D00046EB0100B4EB030C75EB000C04D3E41AF7
:1008E00065EB000517460E46241908F101006D411D
:1008F00080463428E3DDF91946EB0600091BA841C0
:1009000003D24FF0FF32134601E0002213461BEBE7
:10091000070046EB0A51BDE8F04DFFF73CBE0EB5AF
:10092000C10F80EAE0700844CA07002140F2334357
:100930008DE80E000A460B46FFF73CFE03B000BDF3
:1009400070B5C1F30A5201F000450024C1F3130150
:1009500040F2FF3341F480119A4201DA002070BD69
:1009600040F233439A42A2F2334203DC5242FFF791
:100970007DFD00E090402C43F1D0404270BDC1F3BA
:100980000A52C1F3130140F2FF3341F480119A423D
:1009900002DA00200146704740F233439A42A2F245
:1009A000334202DC5242FFF761BDFFF750BD000049
:1009B00030B5041E71F1000404DB4FF000444042E6
:1009C00064EB0101141E73F1000405DB1C464FF0BB
:1009D0000043524263EB04038B4208BF824230BDA6
:1009E00030B5041E71F1000404DB4FF000444042B6
:1009F00064EB0101141E73F1000405DB1C464FF08B
:100A00000043524263EB0403994208BF904230BD59
:100A1000064C074D06E0E06840F0010394E807004B
:100A200098471034AC42F6D3FFF7C4FB5084030858
:100A300070840308202A06DBCB17203A41FA02F023
:100A400043EAE07306E041FA02F3D040C2F120022B
:100A50009140084319467047C0B24FF4F05100F07E
:100A6000BDB900002DE9FF4F087881B09946FF28F5
:100A700005D0491C2D2804D00024002308E00023C1
:100A80000BE00124F9E703EB830300EB4303491C6C
:100A90000878FF28F7D104B15B4200200090147859
:100AA00001462D2C01D02B2C04D1521C2D2C12D000
:100AB0000024009400251678FF2E0ED00A24A0FBF7
:100AC00004C801FB0481002700FB0711521C16EB30
:100AD0000C006941EFE70124EBE7994450EA010279
:100AE0000ED00024AA4D2646DFF8A88200F08AF92D
:100AF00082468B46B9F1000009DAC9F100071BE014
:100B000001980021C0E9001105B0BDE8F08F07464B
:100B100012E0F80707D022462B4630464146FFF741
:100B2000DFFB0646884622462B4610461946FFF74D
:100B3000D7FB04460D467F10002FEAD1B9F1000F14
:100B4000324643465046594602DAFFF728FE01E096
:100B5000FFF7C6FB009A0AB181F00041019AC2E991
:100B60000001D1E72DE9FF4F1F468DB0D7E90146BF
:100B70004FF0FF382E2045464FF000090B90B96921
:100B80006D1C0E988847396A824688470028F6D13E
:100B9000BAF1FF3F0AD024F4D064002E11DDBAF17F
:100BA0002B0F08D0BAF12D0F0BD102E0404611B047
:100BB000ABE744F48064B9696D1C0E98884782469F
:100BC000761E6946600501D52D2000E02B208DF8AA
:100BD000000001F1010B0DF1200809E0B9696D1C5D
:100BE0000E98884782460F9844F40074761E05607C
:100BF000002E02DDBAF1300FF0D00B998A453ED1BC
:100C000044F0800406E00F99681CA9F1010944F43E
:100C100000740860B9696D1C761E0E98884782467C
:100C20003028F0D02BE00B998A4505D1200603D45B
:100C300044F08004761E18E0504605F001F908B330
:100C40000DF11301761E44F400748B4508D2AAF10D
:100C500030000BF8010B200607D5A9F1010003E0D5
:100C6000200602D409F101008146A00502D50F99A2
:100C7000681C0860B9696D1C0E9888478246002E72
:100C8000D1DC53E0002E51DDBAF1650F02D0BAF18C
:100C9000450F4BD1A00549D5B9696D1C24F44074AA
:100CA000761E0E9888478246002E0CDD2B2804D035
:100CB000BAF12D0F07D144F48074B9696D1C0E98F8
:100CC00088478246761EE00501D52D2100E02B21C4
:100CD00008F8011BCDF82C8021E00DF12901761ECA
:100CE00044F4007488450CD2AAF1300010F0FF00E3
:100CF00088F8000002D10B99884509D908F101084C
:100D000006E0E00501D5244801E042F20F7081467B
:100D1000B9696D1C0E98884782460F980560002EB1
:100D200004DD504605F08CF80028D6D1F9690E98FC
:100D30008847FF208BF8000088F80000002006900C
:100D400007904B466A4608A906A8FFF78BFEA00548
:100D500002D46FF001002AE714F0240F0AD0E00754
:100D600014D1DDE906123868031D3B600068C0E954
:100D700000120BE0DDE90601FFF737FB0146E00753
:100D800004D13868021D3A600068016028460EE709
:100D9000000024400000F03FF1D8FFFF426842B15C
:100DA000016811F8013B23B1521EC0E90012184638
:100DB00070470121C160881E704742685AB1C368FC
:100DC000016843B983688B4205D0491E521CC0E9B3
:100DD0000012002070474FF0FF3070477F2801D984
:100DE000002208E0064A02EB5002C007127800D148
:100DF000120902F00F0201209040084070470000E5
:100E0000108003080EB540F2334202920022CDE971
:100E100000221346FFF7CEFB03B000BD70B58C185F
:100E200010F8015B15F0070301D110F8013B2A11FE
:100E300006D110F8012B03E010F8016B01F8016BEB
:100E40005B1EF9D12B0705D40023521E0DD401F8E7
:100E5000013BFAE710F8013BCB1A921C03E013F8B0
:100E6000015B01F8015B521EF9D5A142D8D30020E5
:100E700070BD10B500230AE000EB8304D4ED000A36
:100E800002EB83045B1C70EE800AC4ED000A8B4207
:100E9000F2DB10BDFEE70000F0B500269FED101A52
:100EA0001AE0002515E006FB0257B0EE410A0024C7
:100EB00008E050F824C0641C0CEB870CDCED000A41
:100EC00030EE800A8C42F4DB03EB87046D1C84ED6A
:100ED000000A9542E7DB761C9642E2DBF0BD00009B
:100EE0000000000010B5DFED0A0A00230AE000EB65
:100EF000830494ED001A02EB83045B1CD4ED001A0A
:100F000041EE210A8B42F2DB30EE800A10BD000078
:100F1000000000002DE9F04F8046934603EBD370AC
:100F200042108946514209EB410E1546A9EB020ACF
:100F30002CE0144627E09FED170A002117E000205F
:100F40006E18B61A10E02718BF1A06FB097C01FBC1
:100F5000030708EB8C0C0BEB8707DCED000A97ED21
:100F6000001A401C00EE810A9842ECDB491C9942B1
:100F7000E5DBA11AAE1A06FB0E100999641C01EB01
:100F8000800080ED000AA245D5DC6D1CAA45D0DCAE
:100F9000BDE8F08F000000000649087820B100206D
:100FA000087018B104A102E00120F9E703A104A030
:100FB00004F072BB900200204F4E00004F464600E6
:100FC00044454255472049533A202573000000000C
:100FD0000FB4064810B50078002803D003A9029882
:100FE00004F07EFB10BC5DF814FB000090020020B2
:100FF0007047102A0FD0C26AD1E9002342EA0322C7
:101000000B89097B4FEA034343EA016142EA01028B
:1010100003D1C26002E0C268EEE7C2624FF0000096
:101020007047102A0FD0826AD1E9002342EA0322D6
:101030000B89097B4FEA034343EA016142EA01025B
:1010400003D1826002E08268EEE782624FF0000026
:101050007047000030B50A68102A1AD0026A104B97
:1010600002EA0302D1E9013443EA0403D1E903456A
:1010700044EA050443EA04034C69896943EA4423CA
:1010800043EA413141EA020141F0080103D1016024
:1010900002E00268E3E701624FF0000030BD0000AB
:1010A0008101F0FF30B5D1E901231A43D1E90334BE
:1010B00023431A434B690D681A438B691A43D1E9DC
:1010C0000734012D496A05686FF30E0505D01A43F0
:1010D00022430A432A43026008E0234329430B4387
:1010E000416803606FF30E010A434260002030BD87
:1010F000426942EA4101416100207047F8B5144657
:101100000546D1E9000210438A686FF01F03C968E1
:1011100003EB421242EA412108430090286100F0AB
:1011200053FD064609E0601C07D024B100F04CFDD9
:10113000801BA04201D90320F8BDA8698006F2D423
:101140000020F8BDF0B56FF00F05D1E9003405EBD4
:1011500004145B1E2E0123438C682F0306EB04242A
:101160004FEA054C23430D8A8E8ACC68097E4FF0E6
:101170007F4E07EB05450CEB06560EEB0161012A8D
:101180000CD082683F1107EB043423432B433343D5
:1011900002F070420B43134383600FE0C2682B439D
:1011A0000B4302F070428168134301F07042210347
:1011B000A1F5805131431143C36081600020F0BD2F
:1011C00038B50446094D4FF0AA300090A8790423A1
:1011D00060436A46002102F01FFFA87904236043A0
:1011E0006A460021401C02F017FF38BD2817002076
:1011F0002DE9FC47254F89460646002500240DF1C0
:10120000040810E0CDF80080798870438B084A46C6
:10121000002102F099FD7888BDF80410B1EB900F21
:1012200004D1641CA4B2B879A042EBD8B879A0422A
:1012300002D10020BDE8FC87304602F0A7FB20B1B8
:10124000294613A004F028FA16E0B9F1FF3F13D0A5
:1012500000200AE07A8806FB00109308002211465D
:1012600002F0B0FEBDF80400401CADF80400B879EF
:10127000BDF804108842EDD86D1CADB2032DBDD36E
:10128000314609A004F008FA0120D3E7281700200E
:101290006572726F7220657261736520626C6F6334
:1012A0006B3A25640D0A000062616420626C6F6312
:1012B0006B20636865636B65643A25640D0A000002
:1012C00038B50446104D00208DF80000A8790123A0
:1012D00060436A46002102F06BFD9DF80000FF2884
:1012E00001D0022038BDA879012360436A4600215D
:1012F000401C02F05DFD9DF80000FF2801D0012098
:1013000038BD002038BD0000281700202DE9F84F17
:1013100091462F4A8A461D469179B0FBF1F3B0FB06
:10132000F1F801FB130B404600F0B8F828490746D6
:101330004889B84202D20120BDE8F88F002428E095
:101340005C4516D3ADB14A88A2EB0A01A94201D28D
:101350008EB200E0AEB207FB004108FB00404B46F6
:101360005246009602F092F94FF0000AB144AD1BCC
:1013700005E007FB004108FB004002F05BFA30B1DA
:101380003846FFF71DFF012000F024F8CBE7641C6E
:10139000A4B20F498879A042D2D80D46A879A042BC
:1013A00014D1384600F028FA404602F0EFFA002047
:1013B0006A89696908E031F81040444502D121F892
:1013C000107003E0401C80B28242F4D80020B3E7E2
:1013D00028170020F8B506460021294D4FF6FF706A
:1013E00003E06A6922F81100491C6A898A42F8D828
:1013F0000020A88104461CE0A879042360436A46C3
:10140000002102F0D5FC9DF80000FF280CD1B6B1F8
:10141000A879012360436A460021401C02F0C8FC01
:101420009DF80000FF280AD0214616A004F034F9E8
:10143000641C6989A142DFD800206A6916E09DF822
:1014400002009DF8031000EB01206989814202D956
:10145000696921F81040A889401CA881E8E732F8A2
:1014600010308B4201D3E88102E0401C8142F6D863
:10147000E889642801D20220F8BD0020F8BD0000F0
:101480002817002062616420626C6F636B20696EB4
:101490006465783A25640D0A0000000070B5104EAE
:1014A000104C71892268491E914200D2216000F0DF
:1014B00001052946206800F017F8411C0AD17089FF
:1014C0002168401E884207D92946206000F00CF8A8
:1014D000411C01D0206070BD4FF0FF3070BD000096
:1014E0002817002028000020F8B50D460021401CD8
:1014F0000091040012D00C4F012626EA0400A842F5
:101500000AD1B879611E484304236A46002102F0DB
:101510004FFC0098401C04D0641EEED14FF0FF3009
:10152000F8BD601EF8BD000028170020F8B5254E54
:1015300000273C46B78113E02046FFF7C1FE70B993
:10154000204602F023FA38B121461FA004F0A4F887
:101550002046FFF735FE02E0B089401CB081641CD4
:101560007089A042E8D8B1891BA004F095F8B08931
:10157000642801D20120F8BDC0EB4010642100EBCB
:101580004000B0FBF1F50024009710E02046FFF783
:1015900097FE58B9B079022360436A46194602F0B3
:1015A0003BFD0098401C0090A84203D0641C708949
:1015B000A042EBD80120FFF70DFF0028DBD002206E
:1015C000F8BD00002817002042616420626C6F6340
:1015D0006B3A25640D0A0000676F6F645F626C6F81
:1015E000636B6E756D3A25640D0A000010B502F04C
:1015F000F9F900BB184C616911B100200AF0A0FC98
:101600006089410000200AF0A7FC606161894900FF
:10161000FEF73AFE606970B10120FFF7DBFE60B1B2
:101620000EA004F039F8FFF781FF90B111A004F08B
:1016300033F8022010BD012010BD618912A004F012
:101640002BF8A18916A004F027F8E18919A004F06D
:1016500023F8002010BD000028170020666F726D6F
:101660006174206E616E6420666C6173682E2E2E2C
:101670000D0A0000666F726D6174206661696C65A9
:1016800064210D0A00000000746F74616C20626CAC
:101690006F636B206E756D3A25640D0A00000000C3
:1016A000676F6F6420626C6F636B206E756D3A2597
:1016B000640D0A0076616C696420626C6F636B2054
:1016C0006E756D3A25640D0A000000000549CA894F
:1016D000824202D24FF6FF707047496931F810001C
:1016E00070470000281700202DE9FF5F9B46154634
:1016F0008246002679E03F4C6088B0FBF5F1A07986
:10170000414301988319B3FBF1F0FFF7DFFF6189D3
:10171000814203D8012004B0BDE8F09F354C6188B8
:10172000A479B1FBF5F26243B3FBF2F702FB173287
:101730006A43B2FBF1F300FB0437B2FBF1F001FBAB
:101740001028A1EB0800B0FBF5F084B2ABEB06006B
:10175000A04200D284B204FB05F91FFA89F31FFAF4
:1017600088F15246384602F0D1F9032809D11FFA10
:1017700089F31FFA88F15246384602F0C7F9032868
:1017800004D004282ED068B30220C4E74B461FFAC9
:1017900088F152463846FFF7B9FDDFF858804FF020
:1017A000FF3198F80600B7FBF0F0FFF721FD80B994
:1017B00098F806000021B7FBF0F0FFF719FD81460D
:1017C00098F80600B7FBF0F002F0E0F8B9F1000F6E
:1017D00008D098F80600B7FBF0F0FFF7F1FC012005
:1017E000FFF7F8FD05FB04AA26445E4583D30020DD
:1017F00091E700002817002008B5CC218DF80010D3
:10180000044901236A4689794843194602F004FCD9
:1018100008BD0000281700202DE9FF4F85B01546B0
:1018200000274FF0FF3B7BE0404C6088A179B0FB84
:10183000F5F048430699CB19B3FBF0F0FFF746FFEC
:1018400061898046414503D8012009B0BDE8F08F89
:10185000364A50889279B0FBF5F15143B3FBF1F46D
:1018600001FB143101FB05FABAFBF0F308FB02316E
:10187000BAFBF0F200FB12A9A0EB090080B2B0FBAA
:10188000F5F002910899ADF80400C91B8CB20391E0
:10189000844200D3044601A804FB05F600901FFA19
:1018A00089F1C6F38F034FF0FF32029802F04CFA31
:1018B00008B10220C9E7BDF80400B0EB960F0FD1C4
:1018C000B3B21FFA89F1059A029802F0CFFA38B93B
:1018D0004146C34520D00846FFF78EFFC346D8B126
:1018E0001248817940884143A1EB0A00B0FBF5F032
:1018F000039980B28CB2ADF80400844200D3044650
:1019000004FB05F61FFA89F13346059A0298FFF7A2
:10191000FDFC08B1032098E7059827443044059062
:101920000898874280D300208FE700002817002006
:10193000F0B500261AE0002506FB02FC13E00024A7
:101940000EE005FB024750F826E0641C0EEB870E04
:101950000CFB02779EED000A03EB870787ED000A78
:101960009442EEDB6D1C9542E9DB761C8E42E2DB95
:10197000F0BD0000F0B500238D1C9FED120A05FBA1
:1019800005F404E002EB83065B1C86ED000A9C4232
:10199000F8DC002412E00023661C0CE004FB013795
:1019A00000EB870797ED000A06FB053702EB870778
:1019B0005B1C87ED010A8B42F0DB641C8C42EADB86
:1019C000F0BD00000000000031B500F0FDF8044655
:1019D00000F0FAF80099001B8842F9D338BD0000E6
:1019E0002DE9F84FDFF8A091002209F1040A0AF16D
:1019F000040B4FF00F080BF1040E01260B68964004
:101A00003340B34271D14C68022C01D0122C11D159
:101A1000D40800EB84073D6A5407E40E08FA04FC7E
:101A200025EA0C05D1F810C00CFA04FC4CEA050CB0
:101A3000C7F820C007685400032591F804C0A540EA
:101A40000CF0030CAF430CFA04FC4CEA070CC0F892
:101A500000C04F68012F05D0022F03D0112F01D0F5
:101A6000122F11D18768D1F80CC0AF430CFA04FCD7
:101A70004CEA070CC0F808C04768B7430E79C6F3B4
:101A8000001696403E434660C668AE438D68A5404A
:101A90003543C5604C68E4006FD53C4C256845F47F
:101AA00080452560246822F0030504F480440094F6
:101AB000374C2E19D6F808789407250F08FA05F444
:101AC000A743344CA04201D100242EE0324CA04266
:101AD00001D1012429E0314CA04201D1022424E0AB
:101AE0002F4CA04202D103241FE046E02D4CA0421F
:101AF00001D1042419E02C4CA04201D1052414E0AA
:101B00002A4CA04201D106240FE0294CA04201D169
:101B100007240AE0274CA04201D1082405E0264C06
:101B2000A04201D1092400E00A24AC403C43C6F89D
:101B30000848D9F800404D464E689C43F60300D54E
:101B40001C432C60DAF8004055464E689C43B603AF
:101B500000D51C432C60DBF800405D464E689C437A
:101B6000F60200D51C432C60DEF8004075464E6836
:101B70009C43B60200D51C432C60521C102AFFF473
:101B80003CAFBDE8F88F0000003C01404438024003
:101B90000030014000000240000402400008024002
:101BA000000C0240001002400014024000180240E5
:101BB000001C024000200240002402400AB1816162
:101BC00070470904FBE70000014800687047000007
:101BD0001400002002480168491C016070470000A1
:101BE000140000200B4810B5016841F40071016039
:101BF000016841F480610160016841F48071016015
:101C0000052000F0D3F80F2000F006F800F015F8DA
:101C1000002010BD003C024010B5044600F020FA40
:101C20004FF47A71B0FBF1F001F087FA00222146FF
:101C3000501E00F09BF8002010BD08B50020009059
:101C400008BD70B515460E46040003D094F8210077
:101C500010B107E0012070BD002084F8200020466C
:101C600000F020F8211D2068FFF7F4F9D4E9000204
:101C70003146FFF7D6F9D4E900022946FFF7B9F952
:101C800060681028206808D0016A41F004010162F0
:101C9000012084F82100002070BD016841F004019A
:101CA0000160F5E770B5274886B00024016841F06F
:101CB00001010160006800F001000590214808382A
:101CC000016841F008010160016801F00801059117
:101CD000016841F010010160016801F010010591F7
:101CE000016841F0400101600068032500F04000F8
:101CF00005904020CDE900040120CDE90205124EF7
:101D000069463046FFF76CFE7015009001A902206D
:101D100081E831000C20049069460C48FFF760FE12
:101D20004DF633000090694602943046FFF758FEA6
:101D30004FF4F060009069460548FFF751FE06B089
:101D400070BD000038380240000C0240001802400C
:101D50000010024000F01F02012191404009800064
:101D600000F1E020C0F8001170470000F0B40E4B05
:101D70001B68C3F30223C3F10704042C00D9042415
:101D80001D1D072D01D2002300E0DB1E012606FAEF
:101D900004F56D1E0D409D409E40761E164045EA9E
:101DA0000601F0BC02F049B90CED00E0064A00F073
:101DB000070110684FF6FF03184040EA012003496D
:101DC00008431060704700000CED00E00000FA05C9
:101DD0002DE9F8431D48016841F080510160006819
:101DE000012700F080500090380490FAA0F0DFF84E
:101DF0006080B0FA80F048F82070FFF7E5FE0446F6
:101E00004FF47A75134E04E0FFF7DEFE001BA84284
:101E100013D87068C003F7D54FF4003090FAA0F0E3
:101E2000B0FA80F048F82070FFF7CEFE044607E0D5
:101E3000FFF7CAFE001BA84202D90320BDE8F883C1
:101E400070688003F4D50020F8E7000040380240B5
:101E500000000E42007000402DE9F05FDFF8F8A1AD
:101E600004460F46DAF80000DFF8F08100F00F02B8
:101E7000C8B27A49814641F2883608F10808BA4268
:101E800061D202468AF80020DAF8000000F00F0064
:101E9000B8427DD12078800707D5D8F80020A36804
:101EA00022F0F0021A43C8F800202078C0072DD095
:101EB000606801281AD002281BD0032819D00968AD
:101EC0008907002964DAD8F80010474621F0030199
:101ED0000143C8F80010FFF777FE05466068012847
:101EE0000FD0022818D003281CD027E009688903E6
:101EF000E7E709688901E4E7FFF766FE401BB042A7
:101F000058D83868C0F381000128F5D188E0FFF780
:101F10005BFE401BB0424DD83868C0F381000228F8
:101F2000F5D17DE03868FFF74FFE401BB042F9D98C
:101F300040E0FFF749FE401BB0423BD8386810F044
:101F40000C0FF6D16CE02078800707D5D8F8002078
:101F5000A36822F0F0021A43C8F800202078C007D6
:101F60004CD06068012828D0022829D0032827D027
:101F700009688907002949DAD8F8002022F003020D
:101F80000243C8F80020FFF71FFE0546606800E026
:101F90003CE001281DD0022829D0032838D0B346C0
:101FA0004646306810F00C0F28D0FFF70DFE411B9D
:101FB0005945F6D90320BDE8F09F09688903D9E7A0
:101FC00009688901D6E7FFF7FFFD411B594502D992
:101FD000F0E7B34646463068C0F381000128F2D1ED
:101FE0000CE0FFF7F1FD411B594502D9E2E7B3468A
:101FF00046463068C0F381000228F2D18AF800908A
:10200000DAF8000000F00F00B84209D00120D2E752
:1020100044462068FFF7D8FD401BB042F9D9C9E714
:102020002078400707D5D8F80010E26821F4E05185
:102030001143C8F800102078000708D5D8F8001020
:10204000226921F4604141EAC201C8F800100F2062
:10205000FFF7E2FD0020AEE7003C024000380240FE
:1020600010B500F043F808490968F02292FAA2F28C
:1020700001F0F001B2FA82F2D140044A515CC8404A
:102080000349086010BD00000838024082D30008F0
:102090000000002010B5FFF7E3FF074909684FF47F
:1020A000E05292FAA2F201F4E051B2FA82F2D14087
:1020B000024A515CC84010BD0838024082D3000873
:1020C00010B5FFF7CDFF074909684FF4604292FA57
:1020D000A2F201F46041B2FA82F2D140024A515CAC
:1020E000C84010BD0838024082D3000830B51948F6
:1020F000006810F00C01184812D0184C04290ED0BA
:1021000008290DD1134A121F1168136801F03F010D
:102110005D0247F6C07304D5B4FBF1F003E020463E
:1021200030BDB0FBF1F01168194093FAA3F3B3FA94
:1021300083F3D940484311684FF4403292FAA2F237
:1021400001F44031B2FA82F2D140491C4900B0FB9F
:10215000F1F030BD083802400024F40040787D01E1
:102160002DE9F84F04460078DFF8FCA2BF4DC00708
:102170004FF0000648D0DAF800105046C1F3810154
:10218000012908D00068C0F3810002280AD1281D67
:102190000068400206D52868800335D560680028AD
:1021A00073D031E0DFF8C49209F1020989F80060C8
:1021B000FFF70AFD074641F2883804E0FFF704FD07
:1021C000C11B41457AD828688003F7D4207989F863
:1021D0000000606860B1FFF7F7FC074604E0FFF716
:1021E000F3FCC11B4145EDD828688003F7D50BE00F
:1021F000FFF7EAFC074604E0FFF7E6FCC11B414598
:10220000E0D828688003F7D42078DFF8649280074C
:1022100044D5DAF80010504611F00C0F4FF0F808D2
:1022200009D00068C0F3810002280BD18E48001F3E
:102230000068400206D42868800714D5E0680128A9
:1022400023D110E0E068D0B10120C9F80000FFF709
:10225000BBFC074604E0FFF7B7FCC01B6428B1D8FD
:1022600028688007F7D5286898FAA8F22169B2FA99
:1022700082F220F0F8009140084328600EE0C9F88F
:102280000060FFF7A1FC074605E0EAE0FFF79CFCD1
:10229000C01B642812D828688007F7D4207800076C
:1022A00025D5DFF8C4817348616908F16C0881B1F4
:1022B00001210160FFF788FC074605E07EE0FFF79B
:1022C00083FCC01B642879D8D8F800008007F6D5B5
:1022D0000DE00660FFF778FC074604E0FFF774FCAA
:1022E000C01B64286AD8D8F800008007F6D420788C
:1022F000400753D55C483830016841F08051016097
:102300000068DFF8748100F080500090D8F8001069
:1023100041F48071C8F80010FFF756FC074604E04E
:10232000FFF752FCC01B642848D8D8F80000C0054D
:10233000F6D5DFF834B10BF1680B8BF80060FFF7CE
:1023400043FC074641F2883804E0FFF73DFCC11B1F
:1023500041457ED8DBF800008007F6D4207A8BF860
:102360000000A06868B1FFF72FFC074604E0FFF704
:102370002BFCC11B41456CD8DBF800008007F6D56B
:102380000CE0FFF721FC074604E0FFF71DFCC11B32
:1023900041455ED8DBF800008007F6D4A069E8B3B9
:1023A000DAF80010C1F3810102295AD0022806D0C0
:1023B000C9F86060FFF708FC04464DE049E04F466D
:1023C000C9F86060FFF700FC064604E0FFF7FCFB7D
:1023D000801B64283DD828688001F7D4D4E9070120
:1023E000084347F6C07191FAA1F1626AB1FA81F12E
:1023F0008A40A16A4FF0FF3303EB51014FF44033A1
:1024000093FAA3F3B3FA83F399400A4310434FF0CE
:10241000706292FAA2F2B2FA82F200E01FE0E16A80
:10242000914008431049091F086001203866FFF7F2
:10243000CBFB044604E0FFF7C7FB001B642808D869
:1024400028688001F7D50AE0FFF7BEFB001B64286F
:1024500002D90320BDE8F88F28688001F4D4002059
:10246000F8E70120F6E70000083802400038024093
:1024700000004742800E47420070004070B50D4694
:10248000040003D094F82C0010B107E0012070BDC7
:10249000002084F82D00204600F012F8022084F875
:1024A0002C00211D2068FEF7FDFDD4E9000229461D
:1024B000FEF748FE012084F82C00002070BD0000CB
:1024C000304800B5016887B041F001010160006843
:1024D00000F0010005902B480838016841F0040124
:1024E0000160016801F004010591016841F00801F3
:1024F0000160016801F008010591016841F01001D7
:102500000160016801F010010591016841F02001AE
:102510000160016801F020010591016841F040016E
:1025200001600068694600F0400005900D200090B1
:102530000220019001200290032003900C200490BF
:102540001148FFF74DFA4CF20370009069460F48AE
:10255000FFF746FA4FF68370009069460C48FFF784
:102560003FFA4FF63F00009069460A48FFF738FAF5
:1025700048F23710009069460748FFF731FA07B074
:1025800000BD00003838024000080240000C024044
:1025900000100240001402400018024010B504462A
:1025A00090F82C00022809D0022084F82C00206822
:1025B000FEF79EFD012084F82C00002010BD70B5B0
:1025C000044690F82C000D4602280CD0022084F816
:1025D0002C002068FEF792FD2868022804D0012014
:1025E00084F82C00002070BD0520F9E72DE9F047A4
:1025F00090F8202081F85620828CA1F85420826A1D
:102600000023120E94090C70C2F383044C7002F084
:1026100003028A70826A120CCA70028D120A0A7151
:1026200090F828204A71C26A4FF6FF7A120E0AEA21
:102630000212CA80C26ACC88C2F3074244EA12146A
:10264000CC8002F00F020A72828DC2F30722D409F5
:102650004C72C2F380148C72C2F34014CC72C2F379
:1026600000140C7300264E73046A4FF00109002C0D
:102670007DD0012CFCD0022C7AD02923C2F3801407
:102680004C769206520E01F81A2F10F8302F0C7863
:1026900044EAD21401F8014B02F07F0201F8012B49
:1026A00050F8042F120ED4090C70C2F341144C7070
:1026B000C2F382048C709207120FCA7004C8CC78DF
:1026C000C2F3074244EA9214CC70C2F340140C7176
:1026D0004E7102F001028A7130F8042CC2F3072215
:1026E000D409CC71C2F380140C72C2F340144C7242
:1026F000C2F300148C72C2F38104CC7202F00302A4
:102700000A7310F8042C52084A734C4681F80E9054
:1027100050F8082B120E0A7450F8082C120C0AEA12
:1027200002224A8230F8082C4D8AC2F30722154350
:102730004D8210F8082C120641F8142F50F8042C82
:102740000D68120E45EA02420A6050F8042C0D682A
:10275000C2F3074245EA02220A6030F8042C0D68F1
:10276000C2F30722154320C110F8042C01E034E025
:1027700076E001F8012B0268120E01F8032B0268C3
:10278000120C12060A6002880D68C2F3072245EA9D
:1027900002420A6002780D6845EA02220A60426835
:1027A0000D6845EA126520C142680D78C2F3074200
:1027B00045EA121501F8025B1207120D0A808288A1
:1027C0000D88C2F30722154321F8025B0079400807
:1027D00008704C701846BDE8F0879207120D0A6128
:1027E00090F82C200C6944EA82020A61026B0C69A1
:1027F000120E44EA92140C61C2F3C2040C7502F08A
:1028000007024A75026BC2F3074254098C75C2F382
:102810008204CC759207520F0A76028E0C7EC2F3A8
:10282000072244EAD2140C760C690F7EBF1C09FA09
:1028300007F5641CA4FB05784FEAE57C06FB0585DB
:1028400004FB0C5591F808C009FA0CF4A7FB04C866
:102850000C6505FB048407FB0644C1E912C40DE7BF
:1028600090F82C209206920A0A61026B0C69120EF3
:1028700044EA02220A61026B0C69C2F30742144364
:102880000C61028E0C69C2F30722641C46F100053C
:10289000ED0445EA5435E404C1E912454FF40074EF
:1028A0000C65EBE670B586B000250E4604468DF843
:1028B0000C50057700F046F876200095CDE90150E0
:1028C0002B462A462946206801F06EFC204602F07D
:1028D00005F88DF80C009DF80C0038B9204601F081
:1028E000F1FE8DF80C009DF80C0018B19DF80C005D
:1028F00006B070BD31462046FFF778FE8DF80C001B
:102900009DF80C00A0B9B6F8540069460004009088
:10291000072001904020CDE90205000104902068C5
:1029200001F05BFC0721204601F03EFD8DF80C0014
:1029300004F1100007C88DE8070094E80F0001F0CB
:1029400033FCD3E71D4800B5016887B041F400614E
:102950000160006800F400600590184814380168B0
:1029600041F480010160016801F480010591016872
:1029700041F004010160016801F004010591016862
:1029800041F0080101600068694600F00800059008
:102990004FF4F85000900220019001200290032093
:1029A00003900C2004900648FFF71AF804200090CA
:1029B00069460448FFF714F807B000BD44380240E8
:1029C00000080240000C02402DE9F04F8BB0044695
:1029D0000D46DDE91478216800201646C862216A98
:1029E000022903D10F02560A46EAC3561021CDE947
:1029F00000714021834608010291CDE903B0694688
:102A0000206801F0EAFB1021204601F0CDFC0028EF
:102A10006DD14FF0FF3A08FB07F0CDE905A007A9FB
:102A200090204FF0020981E8010A01200A9005A9CF
:102A3000206801F097FBB8F1010F01D9122000E0E6
:102A40001120CDE900606946206801F0C6FBB8F1AD
:102A5000010F1AD91221204601F0A6FC070046D129
:102A600040F22A3B2068416B11EA0B0F28D1406BE2
:102A70000004F7D50026206801F0ACFB45F82600DD
:102A8000761C082EF7D32035ECE71121204601F003
:102A90008BFC07002BD140F22A6B2068416B11EAB6
:102AA0000B0F0DD1406B0004F7D50026206801F014
:102AB00091FB45F82600761C082EF7D32035ECE76D
:102AC000406BC0050CD5B8F1010F09D9206A18B1C7
:102AD000012801D0022803D1204600F033F8074630
:102AE0002168486B000705D50820886304200BB0D7
:102AF000BDE8F08F486B800703D54846C1F8389091
:102B0000F5E7486B800603D5202088630620EEE7B2
:102B1000486B800504D54FF4007088630720E6E712
:102B2000564603E001F056FB01C5761E2068416B56
:102B3000890201D5002EF5D1216840F2FF5088634B
:102B40003846D4E710B586B0044600200C21CDE904
:102B500000014021CDE90210080104906946206877
:102B600001F03BFB0C21204601F01EFC06B010BD1D
:102B7000FEB50446006A00250E46032805D030B194
:102B8000012804D0022802D01FE02720FEBDB6F5A0
:102B9000805F05D0B6F5006F04D03EB1262514E065
:102BA000272512E0204601F0D4FF02E0204601F084
:102BB00097FF050009D1211DD4E905070EC9CDE90C
:102BC00000600297206801F0EFFA2846FEBD2DE96B
:102BD000F04F8DB0064600250C468DF82C50DDE9EF
:102BE0001698316817462846CD62316A4FF4007B4B
:102BF000022903D1570AD94647EAC3571021CDE924
:102C000000914021824608010291CDE903A0694666
:102C1000306801F0E2FA1021304601F0C5FB0028CF
:102C20006ED1B8F1010F01D9192000E01820CDE9CB
:102C300000706946306801F0D0FAB8F1010F01D98F
:102C4000192100E01821304601F0AEFB00287FD1A9
:102C5000411E09FB08F99020CDE906900591CDF8B9
:102C600020A00120CDE909A005A9306801F07AFA79
:102C7000B8F1010F24D84FE0406B400420D5A9EBF8
:102C80000500202811D281074FEA900000D0401C97
:102C90008246002706E02146306801F0AEFA241D86
:102CA0002D1D7F1C57450BD2F5E7002704EB87014C
:102CB000306801F0A2FA7F1C082FF7D320342035AA
:102CC0003068416B40F21A321142D5D02AE0406B95
:102CD000400421D5A9EB0500202812D281074FEA34
:102CE000900000D0401C8246002706E02146306854
:102CF00001F083FA241D2D1D7F1C57450CD2F5E7EA
:102D000026E0002704EB8701306801F076FA7F1C8B
:102D1000082FF7D3203420353068416B40F21A6217
:102D20001142D4D0406BC0050BD5B8F1010F08D9C2
:102D3000306A18B1012801D0022802D13046FFF7CD
:102D400001FF3168486B000705D50820886304201F
:102D50000DB0BDE8F08F486B800702D50220886374
:102D6000F6E7486BC00603D5102088630520EFE71F
:102D7000486B800503D5C1F838B00720E8E740F27A
:102D8000FF5088630BA9304601F00AFD0028DFD10F
:102D90009DF82C100729F5D00629F3D0D8E770B597
:102DA000040004D094F85100002510B106E0012081
:102DB00070BD84F85050204600F034F8022084F8AA
:102DC00051002068016821F040010160D4E901014F
:102DD0000843D4E903121143084361690843218B76
:102DE00001F400710843E1690843216A0843A16ABC
:102DF000084321680860A069042101EA1040616A63
:102E00000843216848602168E06A08612068C16958
:102E100021F40061C1616565012084F85100002042
:102E200070BD0000124800B5016887B041F0200174
:102E30000160006800F0200005900D481430016822
:102E400041F4801101600068012100F480100590B8
:102E50004FF4607000900220CDE90101039005203D
:102E6000049069460348FEF7BBFD07B000BD0000B3
:102E700030380240001402402DE9F843044690F82F
:102E80005100DDF82080012801D022287ED169B1CF
:102E900062B15BB194F85000012877D0012784F823
:102EA000507094F85100012803D005E00120BDE8DE
:102EB000F883322084F8510000266665A263A38758
:102EC000E3872163A386E386A664E664A06A4FF4E1
:102ED0000055A84209D12068016821F40051016021
:102EE0002068016841F400510160206801684906CA
:102EF00003D4016841F040010160E0684FF4827141
:102F0000B0F5006F606807D0002867D088426ED1A6
:102F1000E08E012862D06AE020B188420CD1E08EB8
:102F2000012809D1206B21680088C860206B801CB3
:102F30002063E08E401EE086E08E80B9A06AA84241
:102F400044D12068016841F4805101603EE020686E
:102F5000C068A16B0880A06B801CA0639EE0434604
:102F600000220221204601F0BFFE002874D1206B10
:102F700021680088C860206B801C2063E08E401EA2
:102F80000004000CE08609D1A06A00E0C7E0A84276
:102F900004D12068016841F4805101604346002259
:102FA0000121204601F0A0FE00286FD12068C068F2
:102FB000A16B0880A06B801CA063E08F401EE0879F
:102FC000E08E0028CBD1606800286AD143460022F9
:102FD0000121204601F088FEF0BBB8E7206B411CC0
:102FE000216321680078C860E08E401EE086E08E94
:102FF00098B9A06AA84204D12068016841F48051C0
:103000000160434600220121204601F06DFE18BBFD
:103010002068C068A16B087040E04346002202218E
:10302000204601F061FEB8B9206B411C2163216884
:103030000078C860E08E401E0004000CE08607D1D6
:10304000A06AA84204D12068016841F4805101605F
:1030500000224346012100E018E0204601F044FE32
:10306000A0B92068C168A06B421CA2630170E08F08
:10307000401EE087E08E0028CFD1606888B94346C3
:1030800000220121204601F02FFE08B103200EE7A7
:103090002068C168A06B421CA2630170E08F401ED3
:1030A000E087A06AA84210D14346002201212046B1
:1030B00001F01AFE18B1606D40F002000FE02068C8
:1030C000C068ADF80000BDF8000043460122802131
:1030D000204601F009FE20B1606D40F020006065DF
:1030E000D4E784F8517020688168A26AC1F30011A6
:1030F000AA4210D179B1616D41F0020161650168A8
:1031000021F4005101602068016841F40051016020
:1031100084F85060CAE684F850600020C7E60220B8
:10312000C5E64FF0E0210428086903D020F0040030
:103130000861704740F00400FAE710B5401EB0F196
:10314000807F01D3012010BD4FF0E02460610F218A
:10315000601700F072FF0020A061072020610020AE
:1031600010BD7047704710B5040003D094F83900C3
:1031700010B107E0012010BD002084F8380020467F
:1031800000F00CF8022084F83900211D206801F0BD
:103190009FFE012084F83900002010BD08B50068AA
:1031A0000B49884212D10B48016841F002010160CD
:1031B0000068032200F00200009001211D20FEF7AC
:1031C000D5FDBDE808401D20FEF7C4BD08BD0000C8
:1031D00000040040403802400168CA6842F0010221
:1031E000CA600068016841F0010101600020704779
:1031F000704770B50446006801694FF00005C94387
:10320000890715D4C168C943890711D4E91E016132
:1032100001202076206880698007204602D0FFF7D1
:10322000E7FF04E000F098F8204600F096F82576D5
:1032300020680169C943490717D4C168C9434907D0
:1032400013D46FF0040101610220207620688069A8
:1032500010F4407F204602D0FFF7CAFF04E000F0E0
:103260007BF8204600F079F8257620680169C9438B
:10327000090716D4C168C943090712D46FF00801C1
:103280000161042020762068C0698007204602D0B2
:10329000FFF7AEFF04E000F05FF8204600F05DF8B5
:1032A000257620680169C943C90617D4C168C94396
:1032B000C90613D46FF01001016108202076206840
:1032C000C06910F4407F204602D0FFF791FF04E070
:1032D00000F042F8204600F040F8257620680169A9
:1032E000C943C90708D1C168C943C90704D1891EA8
:1032F0000161204600F032F820680169C9430906DF
:1033000009D4C168C943090605D46FF08001016181
:103310002046FFF726FF20680169C943490609D402
:10332000C168C943490605D46FF0400101612046D8
:1033300000F026F820680169C94389060BD4C168EA
:10334000C943890607D46FF0200101612046BDE81A
:103350007040FFF707BF70BD70477047064988424D
:1033600006D10649D1F8800218B10020C1F88002C8
:1033700070470120FAE700003CC202200080404272
:103380007047704738B5016804460868CA68C0F3DA
:10339000000002F4807238B132B1086848680090C9
:1033A000E06B40F00100E06308684A69C0F3400048
:1033B00002F0010238B132B1086848680090E06B51
:1033C00040F00400E06308684A69C0F3800002F03E
:1033D000010238B132B1086848680090E06B40F0F3
:1033E0000200E06308684A69C0F3C00002F001020D
:1033F00038B132B1086848680090E06B40F00800CE
:10340000E0630868C968C0F3401001F0200118B1FA
:1034100011B1204601F0E6FD20680168C068C1F3E3
:10342000C01100F0800019B110B1204601F0E8FE93
:1034300021680868CA68C0F3801002F040020125C4
:1034400068B162B1CA68204622F04002CA6094F8AE
:10345000391032290CD080F8395000F0EDF8E06BCB
:10346000002804D084F839502046FFF78AFF38BD81
:10347000222180F83910F0E770B5040004D094F8E8
:103480003900002510B106E0012070BD84F83850E5
:10349000204600F021F8022084F839002068C16835
:1034A00021F40051C160204601F0F0FD206801695F
:1034B00021F4904101612068416921F02A014161B4
:1034C0002068C16841F40051C160E563012084F8BF
:1034D0003900002070BD000030B504460068204966
:1034E00087B0884239D11F48016841F0010101606D
:1034F000006800F0010005901A481430016841F09E
:10350000100101600068012100F0100005904FF4E7
:10351000007000900220CDE9010103900720124DB8
:10352000049069462846FEF75BFA28150090694624
:103530002846FEF755FA2068C16821F04001C160B5
:103540002068C16841F02001C1602520FEF702FC1F
:10355000032211462520FEF709FC07B030BD00000C
:103560000010014030380240000002402DE9F047D1
:10357000044690F8390099460D46012801D01228DA
:1035800057D125B31AB394F83800012851D0012639
:1035900084F838600027E76394F83900122819D0BE
:1035A000222084F83900A285E2854FF48058E08D0E
:1035B0004B46401EE085A0684FF0000240454FF0AA
:1035C0002001204616D101F04EFEB0B904E00120E2
:1035D000BDE8F0873220E4E72069002820684068D1
:1035E00003D0C1B225F8011B12E0C0F3080125F891
:1035F000021B0DE001F037FE08B10320E8E7206967
:1036000000282068406801D000F07F0005F8010B19
:10361000E08D0028CBD194F83900322805D084F809
:10362000396084F838700020D2E7122084F839001D
:10363000F7E70220CCE770477047FEE7104810B567
:10364000016886B041F0020101600068012100F0CC
:10365000020005900320CDE90210CDE90001094CDC
:1036600069462046FEF7BCF9012211462046FEF7C6
:10367000A5FA012202212046FEF7A0FA06B010BDED
:103680003038024000040240FEE700002DE9F84F08
:103690001C4600230A9E17460D46ADF800306249CD
:1036A0008979B0FBF1F2B5FBF1F1D207B2EBC17F42
:1036B0007DD1DFF87891984689F80080DFF870B105
:1036C0008BF800808BF800808BF80000020A8BF8E2
:1036D0000020000C8BF80000352089F80000002045
:1036E00000F0AAFB20B9012000F0A6FB010002D0E7
:1036F0000220BDE8F88F852289F800208BF8007041
:103700003A0A8BF800208BF800502A0A8BF8002028
:103710002A0C8BF800201E2000F0CEF8F0054FF0A8
:1037200000450ED0404605E014F8010B2870BDF8A6
:103730000000401CADF80000BDF80000B042F3D31B
:1037400064E0760A7A0A4FF02043C2464FF4007CC8
:10375000354F27E0D3F8800040F04000C3F88000E8
:10376000504605E014F8010B2870BDF80000401C1D
:10377000ADF80000BDF800006045F3D3D3F8840035
:103780004006FBD5D3F8940001EB020807EB88084C
:10379000C8F81C00D3F8800020F04000C3F8800077
:1037A000491CC9B2B142D5D37988102000E037E076
:1037B00000EB82000844ADF800001E2000F07CF809
:1037C000852189F80010BDF800008BF80000BDF8D5
:1037D0000000000A8BF800001E2000F06DF807EBD7
:1037E0008201ADF800A01C310CE0002011F8012B83
:1037F0002A70401CC0B20428F8D3BDF80000401C59
:10380000ADF80000BDF80000B042EED3102089F8FA
:103810000000C82003F040FF00F0FCFA402801D06F
:10382000012066E7002064E72817002000000180DF
:10383000000002802DE9F0410C461C498979B0FB5B
:10384000F1F2B4FBF1F1D207B2EBC17F29D1184FED
:1038500000263E70174D2E702E702870010A2970B8
:10386000000C287035203870304600F0E5FA18B9A1
:10387000012000F0E1FA10B10220BDE8F0818520BE
:1038800038702E702E702C70200A2870200C287032
:1038900010203870C82003F0FFFE00F0BBFA40286B
:1038A00001D00120E9E70020E7E700002817002009
:1038B000000001800000028001B5009801E0401E78
:1038C00000900028FBD108BD2DE9F0410546904647
:1038D0000E46012000F042F804463146002000F078
:1038E0003DF807464146012000F038F806464146BB
:1038F000002000F033F884EA070272404240A2F54B
:103900007060FF3805D00AA001F0C6FE0120BDE8B6
:10391000F081744021460DA001F0BEFEE10804F0E4
:103920000703685C01229A40504068540020EEE78B
:103930003262697420656363206572726F72206FF2
:1039400072206D6F72650D0A000000006572726F63
:1039500072706F733A25640D0A00000070B5054659
:1039600000200C460246012602F00101A94208D1BE
:1039700024FA02F1C90704D0510806FA01F31844E9
:1039800080B2521CD2B2182AEED370BD104910B5C5
:103990000969104A914201D1C00103E00E4A9142E7
:1039A00000D180010D4A602111700D490870030A91
:1039B0000B70000C0870D0201070042003F05EFE25
:1039C00000F028FA402801D0012010BD002010BDD1
:1039D0002817002089260048569590DC00000180B9
:1039E0000000028010B5274888B0254901604FF4D7
:1039F00080714160002181604FF4C022C160C0E944
:103A0000041281610121C16102200322CDE9040277
:103A1000CDE90601CDE90002CDE902016A4604A91B
:103A20001848FEF70EF900F0E7F9642003F026FECF
:103A300000F048F8134C38342061042000F028F8D6
:103A4000114B4FF4805220695110984207D14FF426
:103A5000875020806280E020A080802008E00B4B0F
:103A600098420BD14FF40460208061804020A080F8
:103A7000A07121816281002008B010BD0120FBE708
:103A8000600000A0F016002089260048569590DCC2
:103A90000A4A00B5EF211170094A01211170C907C6
:103AA0000870002008700870087000F0B3F9402812
:103AB00001D0012000BD002000BD000000000180F9
:103AC000000002800CB50F49902008700E490020BC
:103AD0000870880301788DF8001001788DF80110C6
:103AE00001788DF8021001788DF8031000788DF8B8
:103AF0000400DDF801009DF8041000BA20F0FF007A
:103B000008430CBD00000180000002802DE9F84F41
:103B10004FF000081C46154682468946ADF80080E5
:103B2000744A474682F8008073480170090A0170A0
:103B300080F800A04FEA1A2101704FEA1A41017083
:103B400030201070002000F077F918B9012000F043
:103B500073F910B10220BDE8F88FE2054FF0004183
:103B60000ED0404605E0087805F8010BBDF80000CE
:103B7000401CADF80000BDF80000A042F3D3B2E055
:103B8000660A4FEA5924AB464FF02042DFF86CE159
:103B90004FF4007C2AE0D2F8801041F04001C2F8D6
:103BA00080100021ADF800104FF0004307E01978B5
:103BB00005F8011BBDF80010491CADF80010BDF858
:103BC00000106145F3D3D2F884104906FBD5D2F832
:103BD000943000EB04080EEB8801CB61D2F8801022
:103BE00021F04001C2F88010401CC0B2B042D2D3D4
:103BF000BEF80200102101EB840108447546ADF8BF
:103C000000002320FFF758FE3A4805210170BDF857
:103C1000002039490A70BDF80020120A0A70E0211C
:103C200001701920FFF748FE002205EB8400ADF873
:103C300000204FF000433C3007E0197800F8011BEA
:103C4000BDF80010491CADF80010BDF80010B1EB34
:103C5000860FF2D3ADF8002041E0BDF80000BDF8BA
:103C60000010204405EB8000C06B214405EB81016E
:103C7000C96988422ED0BDF80000204405EB8000C1
:103C8000C26BBDF80000204405EB8000C1691CA098
:103C900001F002FD224631461FA001F0FDFC4A461C
:103CA000514623A001F0F8FCBDF80000204405EBCC
:103CB0008000C269BDF80000BDF80030204405EB6B
:103CC0008000C16B0BEB4320FFF7FEFD08B104271A
:103CD00000E00327BDF80000401CADF80000BDF86F
:103CE0000000B042B9D300F095F8402800D0012779
:103CF000384630E7000001800000028028170020CD
:103D00006572722068642C72643A307825782C30A1
:103D10007825780D0A0000006563636E756D2C656B
:103D2000636373746172743A25642C25640D0A0010
:103D3000506167654E756D2C436F6C4E756D3A25FD
:103D4000642C25640D0A0000F0B51D46164B0024B6
:103D5000059F16461C70154A1170090A11701070E3
:103D6000010A1170000C107030201870204600F00D
:103D700063F818B9012000F05FF808B10220F0BD27
:103D80004FF0004004E00168B14203D1641CA4B2CA
:103D9000AC42F8D33C8000F03DF8402801D001202F
:103DA000F0BD0020F0BD0000000001800000028096
:103DB00030B4064D2C79641AE4B2A34200D92346EC
:103DC0006C88214430BC89B2FFF7A0BE28170020C0
:103DD00008B500208DF800000649702008701920F1
:103DE000FFF76AFD4FF0004000788DF800009DF865
:103DF000000008BD00000180054900B5FF200870E3
:103E000000F008F8402801D0012000BD002000BDCE
:103E10000000018008B500206FF060420090FFF7BD
:103E2000D7FF400606D40098401C00909042F6D37D
:103E3000022008BD402008BD01B581B000200090DF
:103E400009486FF07E41009A521C0092D0F8182267
:103E50009DF804309A4201D100200CBD009A8A429C
:103E6000F1D301200CBD0000008041422DE9F84F44
:103E70004FF000081D46ADF80080DFF83CA1802619
:103E800044468AF80060DFF834B18BF800100E0A5F
:103E90008BF800608BF80000060A8BF80060000CBD
:103EA0008BF800001E20FFF707FDE8054FF00046E5
:103EB0000FD0ADF8008007E012F8010B3070BDF8AC
:103EC0000000401CADF80000BDF80000A842F3D38C
:103ED00062E06D0A490A4FF02043394FC1464FF462
:103EE000007C27E0D3F8800040F04000C3F8800059
:103EF000484605E012F8010B3070BDF80000401C88
:103F0000ADF80000BDF800006045F3D3D3F884009D
:103F10004006FBD5D3F8940004EB010807EB8808B2
:103F2000C8F81C00D3F8800020F04000C3F88000DF
:103F3000641CE4B2AC42D5D37A88102000EB810037
:103F40001044ADF800001E20FFF7B6FC85228AF869
:103F50000020BDF800208BF80020BDF80020120AD8
:103F60008BF800201E20FFF7A7FC07EB8101ADF8BE
:103F700000901C310CE0002011F8012B3270401C25
:103F8000C0B20428F8D3BDF80000401CADF8000012
:103F9000BDF80000A842EED310208AF80000C82027
:103FA00003F07AFBFFF736FF402802D00120BDE87E
:103FB000F88F0020FBE70000000001800000028075
:103FC0002817002070B5124E1D4600248023337040
:103FD000104B1970090A19701870010A1970000C39
:103FE00018701E20FFF768FCF00302E00260641CFA
:103FF000A4B2AC42FAD310203070C82003F04CFBBE
:10400000FFF708FF402801D0012070BD002070BDDF
:10401000000001800000028030B4064D2C79641A43
:10402000E4B2A34200D923466C88214430BC89B253
:10403000FFF71CBF2817002070470907090E00284A
:1040400006DA00F00F0000F1E02080F8141D704740
:1040500000F1E02080F80014704770472DE9F04F20
:104060008246881AB0FBF3F7002589467F1CDDF8ED
:1040700024B028E0002123E09FED150A002416E07B
:1040800005FB034600200FE001FB030C06FB09CCF7
:104090000AEB8C0CDCED000AF4EEC00AF1EE10FA2B
:1040A00001DDB0EE600A401C9042EDDB641C9442DE
:1040B000E6DB05FB07100BEB8000491C80ED000AD6
:1040C000B942D9DB6D1CBD42D4DBBDE8F08F0000E6
:1040D000000000002DE9F04115460E460746002479
:1040E00014E057F82400FCF76DF941EC100B09A01F
:1040F00053EC102B01F0D0FA601C90FBF5F105FB9E
:10410000110010B904A001F0C7FA641CB442E8DB46
:10411000BDE8F081256620000900000010B50023ED
:10412000DFED0A0A0FE000EB830494ED000AB5EE20
:10413000C00AF1EE10FA01DCB0EE600A02EB830473
:104140005B1C84ED000A8B42EDDB10BD000000001B
:10415000B5EEC00AF1EE10FA01DC9FED010A7047DE
:10416000000000000A6842624A688262D1E90223C4
:104170001A43D1E904310B43C16A1A4321F0F70114
:104180001143C162002070470069C0B270470068E7
:1041900000F003007047000008B502490844009091
:1041A000006808BD142C014070B50DF1100C1143CE
:1041B0009CE870002343194329434268314347F682
:1041C000FF639A430A434260002070BD03210160EF
:1041D00000207047D0F8800070470A688260D1E9FB
:1041E00001231A43D1E903310B43C1681A436FF32A
:1041F0000B011143C160002070470968C0F88010AE
:104200000020704700B5164887B014490022C0E965
:1042100000120121816008211023C0E9031340230B
:1042200043614FF4C073C0E906320A0202624A02D7
:1042300042628A0282620220CDE9000106210291D7
:10424000CDE903100590069069460548FEF716F97A
:10425000034800F007F807B000BD0000400100A0CF
:10426000A803002010B5002301221146184600F0D3
:1042700021F84FF4FA7003F00FFA00230122022113
:10428000184600F017F8002308220321184600F012
:1042900011F84FF40C7301220421002000F00AF8F9
:1042A000BDE8104040F2AB210148FEF777B90000AD
:1042B000A80300201FB5002410B1012802D002E09D
:1042C000102400E00824CDE90014CDE902234FF4C6
:1042D000805269460348FEF772F9002800D0012099
:1042E00004B010BDA803002070B586B000200125E1
:1042F00007F008FE0A24B0FBF4F1B0FBF4F204FB73
:10430000110316A1684601F0D7F9694616A001F01D
:10431000C3F90226284607F0F5FDB0FBF4F1B0FB27
:10432000F4F204FB11030DA1684601F0C5F96946DA
:1043300013A001F0B1F9304607F0E4FDB0FBF4F151
:10434000B0FBF4F204FB110304A1684601F0B4F9D8
:10435000694610A001F0A0F906B070BD25642E25B5
:1043600030316425250000000D0A5352414DCAB971
:10437000D3C3C1BFCEAAA3BA25730D0A00000000A3
:10438000534452414DCAB9D3C3C1BFCEAAA3BA2523
:10439000730D0A0043434DCAB9D3C3C1BFCEAAA30C
:1043A000BA25730D0A00000070B5044600680E4679
:1043B0000025416B11F0450FFBD0416B490703D538
:1043C00003210422826304E0416BC90703D0012169
:1043D0008163084670BDFFF7D7FEB0422BD121683C
:1043E00040F2FF5088630020FFF7D6FE28490842BC
:1043F0004BD0002801DA1C2070BD410001D50920F6
:1044000070BD810001D50A2070BDC10001D50B200F
:1044100070BD010101D50C2070BD410101D50D20F9
:1044200070BDC10101D50E2070BD010201D50F2064
:1044300070BD410201D5102070BD810201D511204F
:1044400070BDC10201D5122070BD010301D513203A
:1044500070BD410301D5142070BD810301D5152025
:1044600070BDC10301D5162070BD010401D5172010
:1044700070BD410401D5182070BD810401D51920FB
:1044800070BD000701D51A2070BD284670BD000020
:1044900008E0FFFD0146002009684A6B12F0450F55
:1044A000FBD04A6B520702D50320042207E04A6B77
:1044B000D20702D001208863704740F2FF528A631E
:1044C00070472DE9F0410446006815460E46002766
:1044D000416B11F0450FFBD0416B490703D5032118
:1044E0000422826304E0416BC90704D00121816387
:1044F0000846BDE8F081FFF747FEB04212D12168BF
:1045000040F2FF5088630020FFF746FE10F4604F32
:1045100003D0810404D51320EBE7000C288007E0CA
:10452000410401D51020E4E7000401D50F20E0E7A5
:104530003846DEE70246292012684FF48031536B7B
:1045400013F0450307D0012305E0536B13F0450337
:1045500000D00123491E0BB90029F6D1536BC3F3D8
:10456000800301B113B10320042104E0516B49061B
:1045700002D500204021916370472DE9F04F8DB0A6
:1045800000250F460B9508261021CDE9006140213A
:104590000C950446CDE9021508010490A846694629
:1045A0002068FFF71AFE10212046FFF7FDFE0028C5
:1045B00044D1A08C69460004009037200190206807
:1045C000FFF70BFE37212046FFF7EEFE002835D11E
:1045D000401ECDE9050630204FF00209CDE907095C
:1045E0000120CDE90980B246464605A92068FFF7BB
:1045F000B9FD3320CDE9006069462068FFF7EDFD85
:1046000033212046FFF7D0FE060017D10DF12C080C
:1046100040F22A6B2068416B11EA0B0F08D1416B05
:104620008902F7D5FFF7D6FD48F825006D1CF1E7A4
:10463000416B090705D5C0F838A004200DB0BDE8CE
:10464000F08F416B890703D5C0F838904846F5E7ED
:10465000416B890603D5202181630620EEE7416B7B
:10466000890504D54FF4007181630720E6E740F225
:10467000FF5181630B9800BA78600C9800BA3860DB
:104680003046DBE70E4810B50C490160002141605F
:104690008160C16001614161816100F16001FEF7EB
:1046A00001F908B1012010BD4FF400610448FEF784
:1046B0005FFA0028F7D0022010BD0000002C014056
:1046C000E003002070B586B004460120ADF8140068
:1046D00000252068FFF75BFD58B3206A04285DD0F1
:1046E00000200221C0268DE8430003904802049078
:1046F00069462068FFF771FD2046FFF7CBFE0500F5
:1047000018D1FFF749FDA0630420FFF745FDE063E2
:104710000820FFF741FD20640C20FFF73DFD606499
:10472000206A48B1012807D0062805D0022803D006
:1047300011E0252006B070BD0320019040200290BA
:1047400069462068FFF749FD05AA03212046FFF7C7
:10475000B8FE0500EED1206A04281FD0BDF8140071
:104760006062000400900920CDE9010669462068D6
:10477000FFF733FD2046FFF78DFE0500DAD1FFF786
:104780000BFDA0620420FFF707FDE0620820FFF7A1
:1047900003FD20630C20FFF7FFFC60632846C9E798
:1047A00070B586B0044600260D460096A18C09041B
:1047B00001910D2102914021CDE9031608010590D8
:1047C00001A92068FFF709FD2068416B11F0450F32
:1047D000FBD0416B490703D503210422826304E027
:1047E000416BC90704D001218163084606B070BD42
:1047F000FFF7CAFC0D2838D1216840F2FF508863CA
:104800000020FFF7C9FC0090C0F343202870324914
:10481000009808425DD00098002801DA1C20E5E7E6
:10482000400001D50920E1E70098800001D50A2069
:10483000DCE70098C00001D50B20D7E70098000105
:1048400001D50C20D2E70098400101D50D20CDE71D
:104850000098C00101D50E20C8E70098000201D5DC
:104860000F20C3E70098400201D51020BEE7009852
:10487000800201D51120B9E70098C00201D51220AD
:10488000B4E70098000301D51320AFE70098400378
:1048900001D51420AAE70098800301D51520A5E7CB
:1048A0000098C00301D51620A0E70098000401D5A8
:1048B00017209BE70098400401D5182096E7009840
:1048C000800401D5192091E70098000701D51A202E
:1048D0008CE730468AE7000008E0FFFD2DE9F04F45
:1048E00087B04FF0000904468DF81490DFF870A1EE
:1048F0004F464D464E46C846CAF8A0900068FFF79E
:1049000065FC0120FDF760F84FF0010BCAF8A0B07C
:10491000CDE90099CDF808904FF48060CDE903907F
:1049200069462068FFF759FC226800234FF4803065
:10493000516BC1F3C01104E0516B401EC1F3C011B3
:104940000CD00029F8D048B140F2FF5090638DF8A8
:1049500014309DF8140000287DD101E00323F6E710
:104960004FF4D570009008204FF04009CDE90109BF
:1049700069462068FFF731FC2046FFF7DBFD8DF824
:1049800014009DF8140018B94FF08048C4F820B006
:104990004FF0000A3720CDE900A069462068FFF7F4
:1049A0001CFC37212046FFF7FFFC8DF814009DF812
:1049B00014004FF6FF7180B34DE03720CDE900A021
:1049C000CDF808904FF48067CDE903A756466946B5
:1049D0002068FFF702FC37212046FFF7E5FC8DF841
:1049E00014009DF8140088BB1E4948EA010000909D
:1049F0002920CDE90109CDE9036769462068FFF761
:104A0000ECFB20680021426B12F0450FFBD0426B9B
:104A1000520703D50321042202E00EE040F2FF52C8
:104A200082638DF814109DF8140078B90020FFF708
:104A3000B3FBC60F07466D1C00E08B460EB95D4503
:104A4000BBD35D4503D31B208DF8140003E0780031
:104A500001D5022020629DF8140007B0BDE8F08F58
:104A600000802542000010802DE9FC5F924605463B
:104A70004FF00008CE0D4F02FBF7A3FBA9074FF440
:104A800000701CD000244FF0010B814614E060023E
:104A9000C2191249CDE9009B46EBE073A1F1B800C1
:104AA000FDF792FF80464A460C492846FBF7D3FBA8
:104AB000641CE4B205F500755445E8D309E0CDE97E
:104AC000000A06483A4633462946B838FDF77CFFC7
:104AD0008046FBF778FB4046BDE8FC9F9804002029
:104AE00030B587B000250446059528460695FFF7A2
:104AF00053FB800102D50E2007B030BD05A920462A
:104B0000FFF73BFD0028F7D10698C0031FD5A08C06
:104B1000694600040090372001904020CDE902054D
:104B2000000104902068FFF758FB37212046FFF76B
:104B30003BFC0028E0D10620CDE900506946206802
:104B4000FFF74BFB06212046FFF72EFCD4E725207C
:104B5000D2E730B587B0002504460595284606956E
:104B6000FFF71AFB800102D50E2007B030BD05A962
:104B70002046FFF702FD0028F7D10698400320D514
:104B8000A08C694600040090372001904020CDE9B8
:104B90000205000104902068FFF71FFB3721204623
:104BA000FFF702FC0028E0D10220009006200190CF
:104BB00069462068FFF711FB06212046FFF7F4FB4A
:104BC000D3E72520D1E700002DE9FC5F914605469B
:104BD0004FF00008CE0D4F02FBF7F3FAA8074FF491
:104BE00000711DD000248A464FF0010B15E0D0461D
:104BF000524629461248FBF72EFB6002C2191049A3
:104C0000CDE9008B46EBE073A1F1B800FDF7DFFFC3
:104C1000641C8046E4B205F500754C45E7D309E015
:104C2000CDE9001906483A4633462946B838FDF71B
:104C3000CEFF8046FBF7C7FA4046BDE8FC9F000068
:104C40009804002010B5124C1048022120604FF447
:104C5000827060600020A060C4E9030101216161ED
:104C60004902A1613821C4E907106062A0620720EF
:104C7000E0622046FEF793F82068016841F04001A9
:104C80000160BDE81040FF2000F004B80050014072
:104C90009806002001B582B04FF47A70009001238D
:104CA00001AA02A90248FEF7E7F89DF804000EBD2C
:104CB000980600200B4A10B511680B6823F04003DA
:104CC0000B6011680B684FF6C77423400B601168C6
:104CD0000B6803430B601068016841F040010160FC
:104CE00010BD0000980600202DE9F0471D469046B3
:104CF0000F460446FCF768FF06465FEA08004FF0DF
:104D000000084FF4005A4FF0010926D034E0681C27
:104D100023D025B1FCF758FF801BA8421DD920687D
:104D2000416821F0E00141602068016821F0400104
:104D30000160A06A504509D12068016821F4005142
:104D400001602068016841F40051016084F85190CD
:104D500084F850800320BDE8F0872068806837EA37
:104D60000000D4D10DE0681C06D0002DD7D0FCF790
:104D70002BFF801BA842D2D82068806837EA000049
:104D8000F1D00020E7E7704770B51E4C92B00025C7
:104D9000266846F080562660246804F080541194FA
:104DA000194C266846F44046266024680DF1240C10
:104DB00004F44044119401240094019402240694C4
:104DC0008CE80D006605CDE907616846FDF7C8F976
:104DD00000B1FEE7FCF7FCFF00B1FEE70CA90F20D5
:104DE00081E831004FF4A0500F904FF480501090A4
:104DF00005210CA8FDF730F8002800D0FEE712B01E
:104E000070BD00004038024000700040FCF7E2BE78
:104E10001048016841F4700101600F48016841F0D9
:104E2000010101600C4A00210832116002680B4B3D
:104E30001A400260031D0A4A1A60026822F48022A6
:104E4000026005480C30016002495806803908604C
:104E50007047000088ED00E000380240FFFFF6FEDA
:104E6000103000240148FEF7C4B900003CC2022003
:104E7000094A10B5074BC2E900310021C2E902100E
:104E800010461161FEF76FF9BDE810400248FEF7C9
:104E9000A3B90000000400403CC2022010B50A4C37
:104EA0002068C068C043C00709D10848006980472E
:104EB00021680020486221686420C862E06021689F
:104EC0006FF00100086110BDA0BF02208401002026
:104ED000F0B50268234D244E244FDFF894C0254BD3
:104EE0004FF0804EA84209D0704507D0B04205D09F
:104EF000B84203D0604501D0984203D122F070043B
:104F00004A682243A8421BD0704519D0B04217D03E
:104F1000B84215D0604513D0984211D0164CA0422B
:104F20000ED0164CA0420BD0154CA04208D0154C08
:104F3000A04205D0144CA04202D0144CA04203D190
:104F400022F44074CA68224302608A68C2620A6816
:104F50008262A84201D0984201D10969016301210E
:104F60004161F0BD00000140000400400008004025
:104F7000000C00400004014000400140004401409A
:104F80000048014000180040001C00400020004084
:104F9000F8B5064610480D460024016841F00401AA
:104FA00001600068032200F00400009011461E20FA
:104FB000FCF7DCFE1E20FCF7CDFE094A0748106016
:104FC000C2E90154C2E903641046FEF7CCF8BDE81B
:104FD000F8400348FEF700B940380240000800409E
:104FE000A0BF022010B590F83910222903D0322931
:104FF00001D0022010BD8168B1F5805F11D0016938
:10500000002901681FD0496801F07F03816A4A1CAA
:1050100082620B70C18D491E0904090CC18518D02C
:105020002FE00269816A002A0268526805D0D2B274
:105030000A80816A491C8162ECE7C2F308020A8097
:10504000816A891CF7E74A68816A4B1C83620A708F
:10505000E0E70168CA6822F02002CA6090F83910BF
:10506000322910D00168CA6822F48072CA600168CF
:105070004A6922F001024A61012180F83910FEF7E5
:10508000DAFA002010BD1221F7E700002DE9F04107
:10509000044600680169E26821F440510A43026154
:1050A0002068C16849F20C6291432369A268E569EE
:1050B0001A4363692B431A430A43C260206841695B
:1050C00021F44072A16911434161E06964263225EF
:1050D000B0F5004F484A494920681DD0884201D0A8
:1050E000904269D1FCF7ECFF00EBC00101EB00102E
:1050F0006168B0468900B0FBF1F1B1FBF8F6FCF74E
:10510000DFFF00EBC00101EB001061688900B0FB1C
:10511000F1F7FCF7D5FF68E0884201D0904219D141
:10512000FCF7CEFF00EBC00101EB00106168B04658
:105130004900B0FBF1F1B1FBF8F6FCF7C1FF00EB61
:10514000C00101EB001061684900B0FBF1F7FCF70A
:10515000B7FF18E0FCF79EFF00EBC00101EB001069
:105160006168B0464900B0FBF1F1B1FBF8F6FCF71D
:1051700091FF00EBC00101EB001061684900B0FB3A
:10518000F1F7FCF787FF00EBC00101EB001061684D
:105190004900B0FBF1F1B1FBF8F06FF018014843A2
:1051A00007EB800005EB0011B1FBF8F0216866F316
:1051B0001F108860BDE8F081FCF76CFF00EBC001B8
:1051C00001EB00106168B0468900B0FBF1F1B1FB62
:1051D000F8F6FCF75FFF00EBC00101EB001061681F
:1051E0008900B0FBF1F7FCF755FF00EBC00101EBC4
:1051F000001061688900CCE70014014000100140F4
:1052000090F83910122903D0322901D002207047BA
:105210008168B1F5805F016A0BD04A1C02620268A6
:1052200009785160C18C491E0904090CC1840ED053
:1052300017E009880268C1F308015160016900297B
:10524000016A02D0491C0162ECE7891CFBE7016896
:10525000CA6822F08002CA600068C16841F040015B
:10526000C160002070472DE9F0471D4690460F466B
:105270000446FCF7A9FC06465FEA08004FF0000967
:105280004FF0010808D030E0681C05D095B1FCF75C
:105290009BFC801BA8420DD82068006837EA0000FC
:1052A000F2D127E0681C20D025B1FCF78DFC801BD3
:1052B000A8421AD92068C16821F08001C160206825
:1052C000C16821F02001C1602068C16821F48071AB
:1052D000C1602068416921F00101416184F8398091
:1052E00084F838900320BDE8F0872068006837EA2A
:1052F0000000D7D00020F6E738B5184800680068ED
:10530000C043800622D44FF47A73012269461348C1
:10531000FEF72CF9124A1088010417D441049DF8B5
:1053200000104FF0000304D50A290ED140F40040CC
:1053300012E00D290ED0C0F30D04084D401CC83DED
:1053400080B229551080C72800D913800348FEF782
:1053500019F838BD40F480401080F7E7680300205A
:105360001C000020FEE7000070B5040300F02EF9D9
:1053700000F0D6F8104D0020C5F898022020FFF765
:1053800089FC0E480088A0F56F41183902D1200E23
:10539000FFF780FCC4F30740FFF77CFCC4F3072051
:1053A000FFF778FCE0B2FFF775FC0120C5F8980222
:1053B000BDE8704000F0B4B80080424224000020F4
:1053C00070B51A4886B00025016841F020010160DF
:1053D0000068012400F0200005904020CDE9000481
:1053E0000220CDE9024069461148FCF7F9FA114E56
:1053F000C6F89842FFF726FC0020FFF75BFC00F0A0
:1054000051F80D490880A0F56F4118390BD10320E0
:1054100000F06AF8C00706D1C6F89852B720FFF727
:1054200039FCC6F8984206B070BD00003038024022
:105430000014024000804242240000202DE9F04187
:10544000164F0646002015460C46C7F89802032062
:10545000FFF720FC12480088A0F56F41183902D1EF
:10546000200EFFF717FCC4F30740FFF713FCC4F34B
:105470000720FFF70FFCE0B2FFF70CFC002405E06B
:10548000FF20FFF707FC3055641CA4B2AC42F7D3F1
:105490000120C7F89802BDE8F08100000080424278
:1054A0002400002070B50F4D0024C5F898429020CC
:1054B00005F52675FFF7EEFB0020FFF7EBFB00205C
:1054C000FFF7E8FB0020FFF7E5FBFF20FFF7E2FB1B
:1054D00044EA0024FF20FFF7DDFB2043012129607F
:1054E00070BD00000080424210B5012803D00228A0
:1054F00003D0032803D0052002E0352000E015206A
:10550000064C0021C4F8981204F52674FFF7C2FB7C
:10551000FF20FFF7BFFB0121216010BD0080424248
:1055200010B50120FFF7E0FFC007FAD110BD000061
:105530002DE9F05FC1F30B06DFF88C800F0BC6F589
:1055400080548A4681461546A24200D81446390343
:105550008B464FF480524046FFF770FF002006E074
:10556000321818F80210FF2903D1401C80B2A04263
:10557000F6D3A04221D23846FFF7F6FE002006E01F
:1055800019F800208319401C08F8032080B2A042BB
:10559000F6D359464FF48052404600F027F8A54212
:1055A0000FD0281BA144A244002685B24FF480549A
:1055B0007F1CA542CBD82C46C9E722465146484617
:1055C000EBE7BDE8F09F0000F006002010B5064CA8
:1055D0000020C4F89802062004F52674FFF75AFB51
:1055E0000120206010BD0000008042422DE9F04102
:1055F0000746C8B2C0F580740E461546A24200D8D0
:1056000014464FF4807822463146384600F00EF8B2
:10561000A54208D0281B2744264485B24446A5420B
:10562000F1D82C46EFE7BDE8F08100002DE9F0410C
:1056300015460C460646FFF7C9FF154F0020C7F870
:1056400098020220FFF726FB12480088A0F56F4160
:10565000183902D1200EFFF71DFBC4F30740FFF7F6
:1056600019FBC4F30720FFF715FBE0B2FFF712FBAD
:10567000002404E0305DFFF70DFB641CA4B2AC42D3
:10568000F8D30120C7F89802BDE8F041FFF748BF02
:1056900000804242240000200FB4054B10B503A93E
:1056A000044A029800F0D4FB10BC5DF814FB000023
:1056B000AD9E0008200000200FB4084B10B504A9CF
:1056C00002AA039800F0C4FB044602A9002000F0DF
:1056D00056FF204610BC5DF814FB00007F650008F3
:1056E000014B024A00F0B4BBAD9E00082000002030
:1056F00003B401984100009850EAC12018BF04206B
:105700004A0D18BF40F0010040F2FF72B2EB515F4A
:1057100008BF40F00200012808BF052002B0704712
:1057200030B583B0044600F0A7FA9FED090B05469B
:105730008DED000B002221466846FAF7C2FE28468E
:1057400000F0B0FA9DED000B03B030BD000000008A
:10575000000000000000000070B52DED020B2DEDE3
:105760000A8B82B00D98C40F20F00045AE488542E8
:1057700048D3AE48854219D30C99C5F313000843AA
:1057800009D09DED0C0B02B0BDEC0A8B02B0BDE858
:10579000704000F046BA002C14BF9FEDA50B9DEDA4
:1057A0000C0B02B0BDEC0A8B02B070BD9FEDA20BDA
:1057B00053EC102B9DED0C0B51EC100BFBF710F97B
:1057C0000AD2022000F06EFA02B0BDEC0A8B02B0E1
:1057D000BDE8704000F030BA9FED990B53EC102BF0
:1057E0009DED0C0B51EC100BFBF7E2F80AD20220F6
:1057F00000F058FA02B0BDEC0A8B02B0BDE8704070
:1058000000F02ABA90489FED92BBA8425CD2924821
:10581000854219D29148784400EBC40090ED000B0A
:1058200053EC102B9DED0C0B51EC100BFAF7B1FF64
:1058300041EC1A0B8A48784400EBC40090ED009BC1
:10584000C4F10100041B36E09FED870B53EC102BD5
:105850009DED0C0B51EC100BFAF742FD41EC100BD7
:105860008348784400EBC40090ED001B51EC100B12
:1058700053EC112BFAF7ECFEFBF762F80446FBF74A
:105880004EF841EC180B9FED7C0B53EC102BFAF704
:1058900027FD9DED0C1B53EC112BFAF77DFF41EC1E
:1058A0001A0B9FED770B51EC180B53EC102BFAF7FA
:1058B00017FD41EC190B51EC1A0B53EC192BFAF7AD
:1058C00068FFCDE90C011BE06F48854217D29FEDC0
:1058D000700B53EC102B9DED0C0B51EC100BFAF7E9
:1058E000B7FE53EC1B2BFBF77BF808D29DED0C0B9E
:1058F00053EC1B2B51EC100BFAF7AAFE6EE00024C0
:105900009DED0C0B53EC102B51EC100BFAF7E8FC4F
:1059100041EC180B60480521B0EE480AF0EE680A29
:10592000784400F002F953EC182B51EC100BFAF705
:10593000D7FC9DED0C1B53EC112BFAF72DFF41EC1E
:10594000180B9FED570B5CB353EC182B51EC100B5D
:10595000FAF71FFF9DED0C0B41EC1C0B53EC182BC1
:1059600051EC100BFAF7BCFC53EC1C2BFAF717FFA9
:1059700053EC192BFAF710FF53EC1A2BFAF709FF27
:1059800053EC1B2BFAF708FFCDE900016FF47F7091
:10599000844226DB01EB045001909DED000B00E7F3
:1059A00053EC102B51EC180BFAF7F3FE9DED0C0B9A
:1059B00041EC190B53EC182B51EC100BFAF790FC3F
:1059C00053EC192BFAF7EBFE9DED0C1B53EC112B4E
:1059D000FAF7DFFE53EC1B2BFAF7DEFE41EC100B5F
:1059E000DFE608464FF07A5101EB04519FED2E0B94
:1059F000084453EC102B01909DED000B51EC100B63
:105A0000FAF76EFC0D4645EC100B044651EC100BFA
:105A1000FFF76EFE042808BF00F01EF945EC104B9E
:105A2000BFE6000000000000422E86400000F07F2C
:105A30000000000000000000EF39FAFE422E864010
:105A400051302DD5104987C0422ED63F00000000AE
:105A5000000000000000F03FB2A2F03FAE270300BC
:105A60009E27030000000000FE822B654715F73FCC
:105A700052270300000000000000E0FE422EE63F37
:105A8000763C7935EF39EA3D0000303E00000000F9
:105A90009C7500883CE4377EC426030000000000AB
:105AA0000000000000000040000000000000700145
:105AB00000B52DED048BB0EE409AF0EE609A83B005
:105AC00051EC190BFAF7DAFE41EC180B18EE100A3C
:105AD00018EE901A8DED008B002818BF01200843A6
:105AE00020F00040C0F17F6000F1E040C00F14D012
:105AF00019EE101A19EE900A8DED009B002918BFBF
:105B00000121084320F00040C0F17F6000F1E04037
:105B1000C00F04BF012000F0C5F8B0EE480A03B082
:105B2000F0EE680ABDEC048B00BD70B504462DEDA7
:105B3000028B4D1E00EBC500B0EE408AF0EE608A8D
:105B400090ED000B35F0060017D053EC182B51ECFC
:105B5000100BFAF7C5FB41EC100B6D1E04EBC500F2
:105B600090ED001B51EC100B53EC112BFAF770FD6C
:105B700041EC100B35F00600E7D1022D36D0042D94
:105B80001CD0062D1CBFBDEC028B70BD53EC182B36
:105B900051EC100BFAF7A4FB94ED0A1B53EC112BFC
:105BA000FAF756FD53EC182BFAF79AFB94ED081B05
:105BB00053EC112BFAF74CFD41EC100B53EC182B66
:105BC00051EC100BFAF78CFB94ED061B53EC112BE8
:105BD000FAF73EFD53EC182BFAF782FB94ED040B19
:105BE00053EC102BFAF734FD41EC100B53EC182B4F
:105BF00051EC100BFAF774FB94ED021B53EC112BD4
:105C0000FAF726FD53EC182BFAF76AFB94ED001B0C
:105C100053EC112BFAF71CFDBDEC028B41EC100B81
:105C200070BD10B553EC102B51EC100BFAF710FDB2
:105C300041EC100B10BD00009FED050B10B553ECAF
:105C4000102B51EC100BFAF74BFB41EC100B10BD75
:105C500000000000000000709FED050B10B553EC34
:105C6000102B51EC100BFAF73BFB41EC100B10BD65
:105C700000000000000000100148006870470000AC
:105C80009C02002002E008C8121F08C1002AFAD1B5
:105C900070477047002001E001C1121F002AFBD1AC
:105CA0007047000001490860704700009C02002016
:105CB0000149012008707047910200202DE9FF5F23
:105CC00082B00021DDE90430020DDDF840B003436D
:105CD00018D044F61050A2F2FF3242431514119826
:105CE00001281FD0A5EB0B00401C5FEA000A4FF013
:105CF00000064E4FDFF83891B046504615D5CAF130
:105D0000000413E0119801244AA3012801D16FEA8D
:105D10000B010298119AC0E90031C0E9024206B0B5
:105D2000BDE8F09FCBF10000DFE704460021404AC8
:105D3000491842EB0450CDE9001012E0E00707D00B
:105D400032463B4640464946FAF7CAFA80468946FB
:105D500032463B4610461946FAF7C2FA06460F4647
:105D60006410002CEAD1DDE90401DDE90023BAF179
:105D7000000F06DAFAF7B4FA42464B46FAF7B0FAE1
:105D800005E0FAF70CFD42464B46FAF708FD0446DB
:105D90000E460022284BFAF723FE03D84FF0FF30BF
:105DA000014607E00022254B20463146FAF750FC19
:105DB000FAF7E5FD102409E0002C0ADB0A22002393
:105DC000FAF718FA039B30321A55641E50EA0102A2
:105DD000F2D1641C039AC4F111031444119A012AEC
:105DE00003D0012208430DD10AE0084304D000206B
:105DF0004FF0110B119072E7A3EB0B056D1E0DE038
:105E00005B4504DD4FF0000205F1010504E003DA13
:105E10004FF00002A5F10105002AECD0029811997B
:105E2000C0E90231C0E9004579E7000000001440F4
:105E30000000F03F300000000000F0430000E03FB1
:105E400030380A2801D20120704700207047000036
:105E50002DE9FF4F95B09B468946064600250FE287
:105E6000252877D100242746F84A0121059400E02F
:105E7000044316F8013F203B01FA03F01042F7D12A
:105E800030782A2811D06FF02F033078A0F130023B
:105E9000092A16D8059A44F0020402EB820203EBA9
:105EA00042021044761C0590EFE759F8042B059246
:105EB000002A03DA504244F40054059044F00204EE
:105EC000761C30782E2816D116F8010F44F0040401
:105ED0002A280DD06FF02F023078A0F13003092B63
:105EE00009D807EB870302EB4303C718761CF3E7D7
:105EF00059F8047B761C30786C280FD006DC4C28CF
:105F000017D068280DD06A2814D104E0742810D066
:105F10007A280FD10DE044F400140AE044F4801410
:105F200001E044F440147278824202D104F58014F6
:105F3000761C761C307866280BD013DC582877D076
:105F400009DC002875D04528F6D04628F4D047282B
:105F50001AD19DE118E0632835D0642879D06528EE
:105F600012D195E1702873D008DC6728F1D0692838
:105F70006FD06E280DD06F2806D1B5E073282CD0D5
:105F8000752875D0782874D05A46179990476D1C9B
:105F900075E1C4F30250022809D003280DD0D9F8C6
:105FA000001004280DD00D6009F1040967E1D9F84B
:105FB0000010EA17C1E90052F6E7D9F800100D8089
:105FC000F2E70D70F0E719F8041B8DF800100020BF
:105FD0008DF80100EA46012003E059F804AB4FF0C8
:105FE000FF3061074FF0000102D40DE008F101011C
:105FF0008846B9420FDA8045F8DB1AF80810002904
:10600000F4D108E008F1010188468142FADB1AF870
:1060100008100029F6D105985B46A0EB0807214639
:106020003846179A00F094FA284400EB080507E078
:106030004DE029E10DE01AF8010B5A4617999047F7
:10604000B8F10108F7D25B4621463846179A13E1AA
:1060500042E00A220092C4F302524FF0000A022AE0
:1060600008D059F804CB032A4FEAEC710AD00DE0AE
:1060700029E02AE009F1070121F00702F2E802C154
:10608000914609E00FFA8CFC4FEAEC71042A03D127
:106090004FFA8CFC4FEAEC71002907DA0A4600211E
:1060A000DCF1000C61EB02012D2202E0220504D597
:1060B0002B228DF80420012203E0E20701D02022E8
:1060C000F7E7904659E00A2102E010220DE0102186
:1060D0004FF0000A00910BE010224FF0000A44F04C
:1060E00004040827009203E008224FF0000A0092FF
:1060F000C4F30252022A05D059F804CB0021032A26
:1061000008D009E009F1070121F00702F2E802C115
:10611000914605E01FFA8CFC042A01D10CF0FF0C1B
:106120004FF00008220728D5702806D0009B83F086
:10613000100353EA0A0305D00EE040228DF8042034
:10614000012208E05CEA010206D030228DF804202A
:106150008DF8050002229046009B83F0080353EA65
:106160000A030AD15CEA010201D1620705D5302297
:106170008DF804204FF001087F1E582804D034A069
:1061800003900EA802900DE036A0F9E75346604652
:10619000009AFAF72FF884460398825C0298401E12
:1061A000029002705CEA0100F0D1029806A9081A78
:1061B00000F1200A600702D524F4803400E00127B2
:1061C000574502DDA7EB0A0000E0002000EB0A01C2
:1061D000009005984144401A0590E00306D45B46C0
:1061E0002146179A059800F0B3F90544002706E008
:1061F00001A85A46C05D179990476D1C7F1C474502
:10620000F6DBE0030CD55B462146179A059800F0B3
:106210009FF9054404E030205A46179990476D1CB9
:106220000099481E00900029F5DC08E002980299C8
:106230005A460078491C0291179990476D1CBAF193
:106240000001AAF1010AF1DC65E100000928010062
:1062500030313233343536373839616263646566DC
:10626000000000003031323334353637383941429E
:10627000434445460000000000F058F90544761CF0
:10628000307800287FF4ECAD19B02846BDE8F08FD7
:10629000620700D4062709F1070222F0070CFCE888
:1062A0000223E14603F000485FEA080C02D00FF237
:1062B000702C0DE05FEA045C02D50FF2682C07E059
:1062C0005FEAC47C02D00FF2602C01E0AFF2700CE8
:1062D0004FF0FF3823F00043CDF850C065280CD0B4
:1062E00006DC452809D046281DD047283DD13DE091
:1062F000662818D067287ED138E00021112F01DBF5
:10630000112000E0781CCDE9000106A90EA8FFF7D6
:10631000D5FCDDE90F010E9A03910021009207F1EF
:10632000010A04914DE04FF000400097CDE90110C3
:1063300006A90EA8FFF7C2FCDDE90F0203920E9B2F
:1063400011990022DDF80CA00093049211B9791C78
:1063500000EB010AB7EB0A0004D4C0F1FF3007F1EB
:10636000010A0490AAEB0700019044E0012F00DA33
:1063700001270021112F01DD112000E03846CDE971
:10638000000106A90EA8FFF799FCDDE90F010E9A9E
:106390000391002104910092BA4621070CD403997D
:1063A000514500DA8A46BAF1010F05DD009AAAF1DB
:1063B0000101515C302908D0B84202DA10F1040F13
:1063C00006DA0121CDE9011015E0AAF10101E9E7A2
:1063D000002805DC049901440491AAEB000102E0C5
:1063E000411C514500DD8A460499401A401C019029
:1063F0004FF000400290200704D40198504501DB83
:10640000CDF8048000208DF84F0002980DF14F0761
:10641000B0F1004F25D02B200E9002984FF00208CB
:1064200000280CDA404202902D200E9007E00A214D
:106430000298F9F7F6FF3031029007F8011DB8F124
:106440000001A8F10108F2DC02980028EFD1791EC2
:106450000E980870307800F0200040F0450007F8F2
:10646000020D12A8C01B00F107081498007800B1B3
:10647000012000EB0A01019801EBE071059841440D
:10648000401A401E0590E00306D45B462146179A49
:10649000059800F05DF805441498007818B15A4644
:1064A000179990476D1CE00324D55B462146179A47
:1064B000059800F04DF805441CE00498002807DB1F
:1064C000DDE90301884203DD0098405C179901E093
:1064D000179930205A469047049805F10105401C51
:1064E00004900198401E019004D12E205A4617991D
:1064F00090476D1CBAF10001AAF1010ADDDC05E04C
:1065000017F8010B5A46179990476D1CB8F1000116
:10651000A8F10108F4DC5B462146179A0598ABE622
:106520002D0000002B000000200000002DE9F041AC
:10653000044600251E461746880404D405E0394663
:106540002020B0476D1C641EF9D52846BDE8F081B7
:106550002DE9F041044600251E469046C80301D5AA
:10656000302700E02027880404D505E0414638465E
:10657000B0476D1C641EF9D52846BDE8F0810A6855
:10658000531C0B60107070472DE9F0410D46074613
:1065900081009046012005F0DFFC0646002405FB43
:1065A00008F506E02946012005F0D6FC46F824004F
:1065B000641CBC42F6DB3046BDE8F0812DE9F041B9
:1065C00080462DED028B14460E469FED258A9000E5
:1065D00004F026F80546002714E058F82700F9F7DC
:1065E000F1FE41EC100BFFF7B7F851EC100BF9F787
:1065F000FCFE00EE100A05EB87007F1C30EE088AD7
:1066000080ED000AA742E8DB00200AE005EB8001EC
:1066100091ED000A06EB8001401CC0EE080AC1EDB6
:10662000000AA042F2DB0027D6ED000A01200CE0B0
:1066300006EB800191ED000AB4EEE00AF1EE10FAEB
:1066400002DDF0EE400A0746401CA042F0DB28467F
:106650007F1C03F035FCBDEC028B3846BDE8F081B1
:106660000000000070B590ED000A9FED1F1A049D18
:10667000B0EEC00A82ED000AF0EE410A002413E0F9
:1066800000EB8406D2ED001A96ED000AB0EEC00AC7
:10669000F4EEC01AF1EE10FA01D282ED000A40EEDB
:1066A000000A31EE001A641C8C42E9DB00EE101A7D
:1066B000F8EEC01A81EE210A01EE101AF8EEC11AA6
:1066C00080EEA11A83ED000A00EE401A11EE100AC6
:1066D000F9F778FE41EC100BFFF7EAF951EC100BDB
:1066E000F9F783FE286070BD000000002DE9F04737
:1066F0000746C06A891E00EB1136C1F3C80501F0D8
:1067000007014FF0010A0AFA01F098469146C4B217
:106710003146761C384605F055FB10B10120BDE826
:10672000F08752464FF40073791991F8340010EA5B
:10673000040C01D04FF0010CC44501D10220EEE75A
:10674000604081F83400B9F10100FA708146E6D06A
:10675000600010F0FF04E7D101246D1C9D42E3D3DB
:10676000D6E7000070B504460020E070401E2063AC
:10677000204605F027FB08B1042070BD04F232204A
:1067800003F034FEA0F52A41553901D0032070BD35
:1067900004F16A0003F0F4FD0B4DB5EB002F06D0B9
:1067A00004F1860003F0ECFDB5EB002F01D10020D1
:1067B00070BD082205A104F1370003F067FF08B19E
:1067C000022070BD012070BD00464154455846412D
:1067D000542020200000000070B500240C4E12E070
:1067E00000EB8405D2ED000A95ED000A93ED001A46
:1067F00070EE600A80EE810A10EE105AB54201DD9B
:10680000012070BD641C8C42EADB002070BD0000DA
:106810000000A04100E0401C02780AB18A42FAD18F
:10682000D0B2704770B515460168846C680A4A8911
:1068300040EAC350590A0023241DF9F7DBFC02CCBF
:1068400021B1884204D3401A241DF8E7002070BD0E
:106850002168084470BD8269891E921E8A4201D84F
:1068600000207047C26A408901FB00207047000089
:106870002DE9F05F8146884601F11A0003F0B6FD6C
:1068800088BB98F80000012700F03F00401E00EB95
:106890008001DFF85CA001EBC00400254FF6FF7B10
:1068A0001AF8051001EB080003F0A0FD06466FB1D1
:1068B000FF2C18D203F058F8074639F81400641C6E
:1068C00003F052F887420ED1374601E05E450AD107
:1068D0006D1C0D2DE4D398F80000400606D52FB1AD
:1068E00039F8140010B10020BDE8F09F0120FBE74B
:1068F000B8D300082DE9F04FA1B09FEDFE0A49F68C
:1069000040478DED190A8DED1A0A8DED1B0A002402
:106910003946012005F020FBF74D1C90F7A069686F
:10692000FEF7BAFEA8680068F9F74CFD41EC100BC1
:10693000002153EC102BFCA0FAF74AFBA868406832
:10694000F9F740FD41EC100B012153EC102BF6A0A0
:10695000FAF73EFBA8688068F9F734FD41EC100BAC
:10696000022153EC102BF0A0FAF732FBA868D0F804
:10697000AC04F9F727FD41EC100B40F22B1153EC5E
:10698000102BE9A0FAF724FBA868D0F8B004F9F7B7
:1069900019FD41EC100B4FF4967153EC102BE2A053
:1069A000FAF716FBA868D0F8B404F9F70BFD41EC30
:1069B000100B40F22D1153EC102BDBA0FAF708FB63
:1069C000DD4EA8683044D0F83403F9F7FBFC41EC05
:1069D000100BDA4953EC102BD3A0FAF7F9FAA86898
:1069E0003044D0F83803F9F7EDFC41EC100BD349F3
:1069F00053EC102B491CCCA0FAF7EAFAA8683044F3
:106A0000D0F83C03F9F7DEFC41EC100BCB4953EC1A
:106A1000102B891CC4A0FAF7DBFA1BA80090D5E95B
:106A200002011AAB19AAFFF71DFED5E902011BAB43
:106A30001AAAFFF7D1FE012826D0C1A0FEF72CFE2E
:106A40001998F9F7BFFC41EC100BBFA053EC102BC9
:106A5000FEF722FE1A98F9F7B5FC41EC100BBEA028
:106A600053EC102BFEF718FE1B98F9F7ABFC41EC2A
:106A7000100BBEA053EC102BFEF70EFEC1490020F8
:106A8000087021B0BDE8F08FBFA0FEF705FED5E984
:106A900002011C9A9DED190A03F094FA394601206F
:106AA00005F05AFA002142F20F731D9001EBC1026A
:106AB000002002EB011200EB82061C9D401C05EB3E
:106AC00086051E1B95ED000A1D9D641C05EB8605C1
:106AD000642885ED000AEEDB491C6429E6DBACA0E6
:106AE000FAF776FA4AF29021012005F035FA0246CB
:106AF000189064211D98FAF73DFF42F210790422A4
:106B00004C4649462020FFF73FFD07460422214618
:106B10002020FFF739FD0646042221462020FFF7FA
:106B200033FD054600244FF0200A4FF0180B4FF0BC
:106B30001C089B480323816804EBC40001EB80021E
:106B400092ED000A042202EB80020A448DED080A4D
:106B500092ED000A082202EB80020A448DED090A38
:106B600092ED000A0C2202EB80020A448DED0A0A23
:106B700092ED000A102202EB80020A448DED0B0A0E
:106B800092ED000A142202EB80020A448DED0C0AF9
:106B900092ED000A0BEB80020A448DED0D0A92ED96
:106BA000000A08EB80020A448DED0E0A92ED000AFD
:106BB0000AEB800008448DED0F0A90ED000A08AA48
:106BC0008DED100A57F82400009066211898FAF706
:106BD000A1F9641C202CACDB0024724856F8242058
:106BE0004946806800EB840090ED000A57F82400C5
:106BF000FAF73FF9641C202CEFDB0024494655F8D6
:106C0000242056F82400FDF789FA641C202CF5DBBB
:106C1000042240F6C4112020FFF7B6FC8146002470
:106C2000022359F82400009055F824001A466421E4
:106C3000FDF714FA641C202CF2DB5BA0FAF7C8F90C
:106C40000120189905F07CF92021304603F060F905
:106C50002021384603F05CF92021284603F058F93A
:106C600004224FF429612020FFF78EFC0646002401
:106C7000322156F8242059F82400FAF77BFE641CD0
:106C8000202CF5DB40F6C414042221462020FFF717
:106C90007BFC2090042221464020FFF775FC1F90CA
:106CA000042221464020FFF76FFC1E90042221465B
:106CB0004020FFF769FC07460025C346002405EB8A
:106CC000C5083D4804EBC40101EB4811806800EBA6
:106CD000810292ED000A042202EB810202448DED52
:106CE000080A92ED000A082202EB81028DED090AE2
:106CF000024463E00000000028C20220434E4EC45C
:106D0000A3D0CDD5FDD4DAD4CBD0D0A3A1A3A1A359
:106D1000A10D0A44617461CAFDBEDDBCAFCEAAA359
:106D2000BA25730D0A000000646174615B25645D1F
:106D30003A2025660D0A000000484C00CD121300D1
:106D40004E6F0D0A000000006D617876616C75650C
:106D50002069733A256609006D65616E76616C7510
:106D6000652069733A256609000000007374645F4A
:106D700064657676616C75652069733A2566090DE0
:106D80000A0000009102002053746172740D0A0021
:106D9000BFAACABCB5DAD2BBB2E3A3A10D0A0000F8
:106DA00074C1022060C10220B5DAD2BBB2E3CDEAE1
:106DB000B1CFA3A10D0A00009CC1022092ED000AF0
:106DC0000C2202EB810202448DED0A0A92ED000AC8
:106DD000102202EB810202448DED0B0A92ED000AB3
:106DE000142202EB810202448DED0C0A92ED000A9E
:106DF000182202EB810202448DED0D0A92ED000A89
:106E00000BEB810202448DED0E0A92ED000A0AEBB3
:106E1000810108448DED0F0A90ED000A03238DEDEA
:106E2000100A209808AA342150F82400009056F83F
:106E30002400FAF76FF8641C202CFFF642AF1F986D
:106E40003222202150F825302098FAF725F86D1CC1
:106E5000402DFFF633AFDFF8EC83002440F6C41575
:106E6000D8F80800294600EB840090ED000A1E982F
:106E700050F824201F9850F82400F9F7FAFF641CFA
:106E8000402CEDDB00241E9857F82420294650F8AA
:106E90002400FDF743F9641C402CF4DB042240F28B
:106EA00071214020FFF770FB80460024022358F830
:106EB0002400009057F824001A463221FDF7CEF83E
:106EC000641C402CF2DBE0A0FAF782F82021304667
:106ED00003F01EF82021484603F01AF820212098DC
:106EE00003F016F840211E9803F012F840211F9875
:106EF00003F00EF84021384603F00AF8042240F26D
:106F0000D9214020FFF740FB07460024192157F8FC
:106F1000242058F82400FAF72DFD641C402CF5DBE2
:106F200040F27124042221464020FFF72DFB1E90E1
:106F3000042221468020FFF727FB06460422214633
:106F40008020FFF721FB1F90042221468020FFF7BD
:106F50001BFB0025209000244FF0040A4FF0200B6B
:106F600005EBC509BC4804EBC40101EB891180683D
:106F7000032300EB810292ED000A0AEB8102024436
:106F80008DED080A92ED000A082202EB810202440C
:106F90008DED090A92ED000A0C2202EB81020244F7
:106FA0008DED0A0A92ED000A102202EB81020244E2
:106FB0008DED0B0A92ED000A142202EB81020244CD
:106FC0008DED0C0A92ED000A182202EB81020244B8
:106FD0008DED0D0A92ED000A1C2202EB81020244A3
:106FE0008DED0E0A92ED000A0BEB810108448DED48
:106FF0000F0A90ED000A08AA8DED100A1E981B21B9
:1070000050F82400009057F82400F9F783FF641C1F
:10701000402CA7DB56F82530192240211E98F9F79D
:107020003BFF6D1C802D96DBDFF83092002440F290
:107030007125D9F80800294600EB840090ED000A7C
:107040001F9850F8242056F82400F9F712FF641C0A
:10705000802CEEDB00242098294650F824201F982D
:1070600050F82400FDF75AF8641C802CF3DB04224E
:1070700090218020FFF788FA81460024022359F8E6
:107080002400009056F824001A461921FCF7E6FF68
:10709000641C802CF2DB4FF490352946012004F06B
:1070A0005BFF034608900C2280214846FAF740FC1B
:1070B0006BA0F9F78DFF4021384602F029FF4021EF
:1070C000404602F025FF40211E9802F021FF80215A
:1070D0001F9802F01DFF8021304602F019FF802129
:1070E000209802F015FF62A0F9F772FF4FF40078C4
:1070F00044464146012004F02FFF06462146F9F799
:10710000C3F8DFF87CA1DFF87CB100242946012018
:1071100004F022FF0746DAF8080004EBC40100EB94
:1071200041312A463846F9F796F8DBF808003A4626
:1071300000EB84004FF4904190ED000A0898F9F7B5
:10714000D1FEFDF705F806EB8400394680ED000A14
:10715000012004F0F5FE641C802CD7DB4AA0F9F76F
:1071600037FF8021484602F0D3FE1C2101A8F9F721
:107170008BF84546DFF82081DFF8209100240DF1DF
:10718000040A2946012004F0E7FE0746D8F8080063
:107190002A4600EB44213846F9F75DF8D9F8080093
:1071A0003A4600EB8400802190ED000A3046F9F762
:1071B00099FE0AEB8400394680ED000A012004F0B4
:1071C000BFFE641C072CDCDB35A0F9F701FF0722AA
:1071D00011A901A8FFF7F2F904460722114601A8F8
:1071E000FCF778FF0722114611A8FCF773FF11A8DE
:1071F00000EB8400DFED2E0A10ED010A20EE200ADC
:1072000010EE100AF9F7DEF841EC100B29A053EC50
:10721000102B0094FEF740FA0120089904F090FE2C
:107220003146012004F08CFE01201D9904F088FEF7
:107230000120189904F084FE01201C9904F080FEBE
:10724000FFF7FEBB88C10220B5DAB6FEB2E3CDEA95
:10725000B1CFA3A10D0A0000C4C10220B0C1022019
:10726000B5DAC8FDB2E3CDEAB1CFA3A10D0A0000A3
:10727000BFAACABCB5DACBC4B2E3A3A10D0A000011
:10728000ECC10220D8C10220B5DACBC4B2E3CDEA0A
:10729000B1CFA3A10D0A000014C2022000C2022037
:1072A000B5DACEE5B2E3CDEAB1CFA3A10D0A000075
:1072B0000000C84225662C204C6162656C20256464
:1072C000090000002DE9F04705685FEA010807465C
:1072D00026D04146384602F0C5FE022841D3411C63
:1072E0001CD0A969814219D8464628784FF0FF3949
:1072F00004281CD03446A869641CA04202D8022489
:10730000022E0AD32146384602F0ACFE40B30128D3
:1073100004D0411C02D0B442EDD10020BDE8F0877A
:107320002E6916B1A869B042DFD80126DDE7012237
:107330003146284602F06FFB040039D0601C37D07C
:1073400001231A4621462846FFF7D0F9022808D023
:10735000012808D0B8F1000F07D0F879022806D02C
:107360000DE00120DAE74846D8E7022006E0701C6D
:10737000844204D0B868301AB8610320F8712878C4
:10738000042802D1F879022814D04E464A462146F4
:10739000284604F02FFE40B9B8F100000AD001469B
:1073A0002246284604F026FE20B101280FD00124F1
:1073B0002046B3E72C61D5E90501891E884201D238
:1073C000401E6861287940F001002871F0E73446DA
:1073D000EEE700002DE9F35F0E6800980024884670
:1073E000D0F840B02546705D6D1C202823D32F288F
:1073F00021D05C281FD0FF2C46D2A0F181017D292D
:107400000BD8715D6D1C01EB0020A1F1400280B230
:107410003F2A02D380397F2936D2012102F076FA41
:10742000070031D0802F12D201466BA0FFF7F2F98E
:1074300050BB0CE06D1C715D2F29FBD05C29F9D08D
:107440007219C8F80020202805D204250EE02BF878
:107450001470641CC7E7002508E00BEB440030F80B
:10746000020C202801D02E2802D1641E002CF4D159
:1074700000212BF814103CB100980B222021806BC6
:1074800003F019F9002703E00620BDE8FC9F7F1CEC
:107490003BF817002028FAD02E28F8D01FB145F06D
:1074A000030500E0641E2CB10BEB440030F8020C25
:1074B0002E28F7D14FF00008C1464FF0080A3BF8DC
:1074C00017607F1C06B3202E03D02E2E04D1A742B6
:1074D00002D045F00305F2E7D04501D2A74219D109
:1074E000BAF10B0F0ED0A74201D045F003050BD81F
:1074F0004FEA896027464FF008084FF00B0A4FEA21
:107500001069DCE745F003050098806B0178E529F8
:107510003DD03EE0802E08D3304602F025FA00210F
:1075200002F0F4F9064645F00205FF2E0FD9AAF144
:107530000100804503D345F00305D046BFE700981E
:10754000310A826B02F8081008F1010818E026B130
:10755000314624A0FFF75EF918B15F2645F0030518
:107560000EE0A6F14100192802D849F0020907E00F
:10757000A6F16100192803D8203E49F00109B6B2EE
:107580000098816B01F8086008F1010897E7052170
:107590000170BAF1080F03D14FEA89604FEA106910
:1075A000C9F38100032803D06FEA0901890701D1DB
:1075B00045F00205A90709D409F00301012901D109
:1075C00045F01005012801D145F008050098806BB1
:1075D000C572002059E70000222A3A3C3E3F7C7FDA
:1075E000000000002B2C3B3D5B5D00002DE9F05FAF
:1075F000894606464022002103F05DF88520307060
:10760000C02086F82000484605F09DFE014606F1A0
:10761000240004F03EFE402400254FF001084746B8
:10762000AA464FF0C10B06F804B0641C06F804A08B
:10763000641C27B139F815700FB16D1CEDB230190B
:10764000394604F026FEA41CE006F2D108F1010040
:1076500000F0FF0839F815000028E4D186F823501F
:1076600086F80180BDE8F09F10B504460420FBF7C2
:1076700058FD0148046010BD1800002070B5054693
:1076800000244FF47A7603E0304600F005F8641CDD
:10769000AC42F9D370BD000070B54FF0E025002179
:1076A0006C69094AAB6912685043AA699A42FCD0D6
:1076B00002D2A3EB020302E0A4EB02063344194416
:1076C00013468142F1D370BD180000202DE9F0412E
:1076D0000F4604460021066800F005FBE8B90025C6
:1076E0003046216B04F06EFBB8B931780429616B28
:1076F000097803D0E52905D021B107E041F3C01195
:10770000491C03D06D1CBD420AD000E000250121B8
:10771000204600F0A5F80028E2D0042800D1072078
:10772000BDE8F0812DE9F05F04460021D0F800901B
:1077300000F0D9FA00284BD199F8000004280CD0A9
:10774000FF254FF0FF382F46C4F83C804846216B98
:1077500004F038FB06004CD13CE0206C05F0F3FD52
:1077600082462DE0D9F80C00243002F03FFE50454F
:1077700026D1D9F80C0040254FF0000890F823607E
:1077800016E0E80600D1AD1CD9F80C00284402F040
:107790002DFE02F0E9F8216C074631F8180002F0DE
:1077A000E3F8874207D1761EF6B208F10108AD1C56
:1077B000002EE6D100E01EB9216C31F8180030B17E
:1077C0000021204600F0CEF85FEA000BCAD05846F0
:1077D000BDE8F09F616B087850B1CA7AE52802F0E5
:1077E0003F02A27130D0130704D50F2A2CD105E037
:1077F000042633E00F2A01D0C5B11CE0226C32B35D
:10780000430605D54F7B20F04000A36A0546E3639D
:10781000A84208D1487BB84205D11046FFF728F8A6
:1078200008B16D1E00E0FF25EDB210E0084604F03F
:107830006AFDB84212D0A16BC87AC00704D10B22EE
:10784000606B02F023FF48B1FF25C4F83C800021A3
:10785000204600F005F806003FF478AF3046B7E761
:107860002DE9F04705460468806A894600F1200842
:10787000286B30B12178042906D04FF4001141451E
:1078800005D80420BDE8F0874FF08051F7E75FEAA4
:10789000C8515ED1401C2863E96A002729B160897C
:1078A000401E10EA582F05D053E02189B1EB581F34
:1078B00021D94EE0284602F0D5FB064601281ED904
:1078C000701C34D0A069B0423DD8B9F1000F12D07D
:1078D0002846E96AFFF7F6FC06000ED0012E0ED00E
:1078E000701C24D0E87940F00400E871204604F0D0
:1078F0005BFDE0B905E02F63C3E70720C2E7022084
:10790000C0E74FF40072002104F1340002F0D3FE0E
:10791000002731462046FEF79EFF4FF00109206305
:107920000BE084F80390204604F03EFD08B10120EE
:10793000A8E7206B401C7F1C20636089B842F0D808
:10794000206BC01B206331462046EE62FEF783FFAA
:107950002863C8F3080020443430C5F828806863E1
:1079600000208FE72DE9F0470426FF2589460446CD
:107970002F46D0F800805FE0404604F023FA06006E
:107980005ED1616B0878A0B198F80020042A12D06B
:10799000CA7AE52802F03F02A27108D02E2806D04C
:1079A00022F02003082B1CD000234B451BD0FF25C1
:1079B00032E0042644E0B9F1000F02D0832841D020
:1079C0002AE0852828D1A06AE063204602F02FFD36
:1079D000060035D1D8F80C00007900F03F00A07106
:1079E00030E00123E1E70F2A01D00DBB1BE0420686
:1079F00005D54F7B20F04000A26A0546E263A8420D
:107A000008D1487BB84205D1206C04F0BBFA08B11C
:107A10006D1E00E0FF25EDB200212046FFF720FF9C
:107A2000060009D00CE0084604F06DFCB84209D00D
:107A30004FF0FF30E06305E0216B00299CD10EB1CF
:107A4000002020633046BDE8F08700002DE9F04FAC
:107A5000876B0446D0F80090D0F84080F87A95B053
:107A600010F0A00F03D0062015B0BDE8F08F002560
:107A700000E06D1C38F815000028FAD199F80000D4
:107A8000042817D00C22394612A802F00BFE9DF8EC
:107A90005300C0076AD00020F872012620643346E4
:107AA000424612A9384602F047FA2046FFF73AFE4E
:107AB000E8BB4FE00F200E35B5FBF0F5AD1C2946B5
:107AC0002046FFF703FE0028CED169422022A06A9B
:107AD00002EB41110844E063E079410733D500F03F
:107AE0000300E071B9F80A00D4E9043142029A189F
:107AF00041F10001C4E90421204601F075FF00288E
:107B0000B2D12146684602F076FC0028ACD1D4E917
:107B10000423D9F80C00383004F096FBD4E9042390
:107B2000D9F80C00283004F08FFBE07900E014E075
:107B300040F00101D9F80C0080F82110684604F0EB
:107B4000ACFB002890D14146D9F80C00FFF74EFD60
:107B5000002089E7761C642EA1D3642E10D004285F
:107B600082D19DF85300F872C4F840809DF853000C
:107B7000800707D50D200C35B5FBF0F6761C02E02A
:107B8000072071E7012631462046FFF79FFD0500DB
:107B900075D1761E5FEA060B58D0A16ACBF10000C2
:107BA00001EB4011204600F09EF8050067D1A06B64
:107BB00004F0A9FB01904846216B04F003F905008D
:107BC0005DD1206C0090666B01980BF0FF0A70731A
:107BD0000F20F07200203073014606F11A0004F005
:107BE00058FBAAF1010000EB800101EBC00800275F
:107BF00001E0854204D0009830F8185008F10108DF
:107C000020482946C05D304404F043FB0DB94FF6CF
:107C1000FF757F1C0D2F4FF6FF70EAD3854203D00E
:107C2000009830F8180008B94AF0400A86F800A019
:107C3000012089F8030000212046FFF711FE05000E
:107C40001DD1ABF101005FEA000BB4D14846216BB6
:107C500004F0B8F8050012D120220021606B02F078
:107C60002AFDD4E90D010B2202F01CFDA06B616B13
:107C7000C07A00F018000873012089F80300284634
:107C8000F2E60000B8D300082DE9F041C16B0446CC
:107C9000866A0568481C02D0204600F024F80028B7
:107CA0001AD1E5274FF001082846216B04F08AF825
:107CB00078B929780429616B10D00F7085F803809A
:107CC000A16AB14208D200212046FFF7C9FD002871
:107CD000EAD0042800D10220BDE8F0810A7802F041
:107CE0007F020A70EAE72DE9F041076806460D4673
:107CF0003878042806D04FF40010A8423CD9E80692
:107D00003AD102E04FF08050F7E7B562B46834B979
:107D10003878032807D30020BC6AF0711CB1788939
:107D20004FEA402812E03889B0EB551F24D9B86AD1
:107D300012E0304602F096F90446401C1AD0022C9C
:107D40001AD3B869A04217D9A5EB080545452146C5
:107D5000EFD23846FEF77FFDC6E90B4060B100EB7D
:107D600055203063C5F30800384434307063002078
:107D7000BDE8F0810120FBE70220F9E710B520B152
:107D8000012805D0022809D105E0FCF77BFC04E0BE
:107D9000FDF716FB04E0F9F729FC08B1012010BD3E
:107DA000002010BD30B54FF4007428B101281CD05C
:107DB000022827D0012030BD39B11F4801290BD03E
:107DC000022904D003290ED103E0002030BD146045
:107DD000FBE7B0F8500020E0816CB0F84C00C30520
:107DE00043EA512025E0042030BD0029EDD00129CF
:107DF00005D0022913D00329F5D108200DE04FF456
:107E0000484016E00029E0D00C4D01296B8808D0CD
:107E1000022904D00329E6D1580A1080D5E714803E
:107E2000D3E7E889A97948435843C11700EBD150FB
:107E300040121060C9E7000040040020281700200D
:107E40002DE9F0411C0015460E4607D048B14FF40D
:107E50000072012811D0022821D11BE00420BDE8C6
:107E6000F0811A4602E0FCF70DFC22462946304616
:107E7000FCF7FAFD0028F6D113E0174669023A46EE
:107E80003046FDF7DBFA641E05F1010506F50076C4
:107E9000F4D106E029463046F9F726FC08B1012066
:107EA000DDE70020DBE7002070472DE9F0411C00F2
:107EB00015460E4607D048B14FF4007201280ED087
:107EC00002281ED118E00420BDE8F081E2B2294664
:107ED0003046FCF779FEB0B1FCF7D4FBF6E7174665
:107EE00069023A463046FDF723FB641E05F10105A1
:107EF00006F50076F4D106E029463046F9F78CFC09
:107F000008B10120E0E70020DEE77CB50D46002146
:107F10001446009101AA694600F059F800280AD1D8
:107F200001998A694B89921E00995A434B43510823
:107F30002960590821607CBD70B5164D00244FF4AE
:107F40000D763146002004F007F845F8240018B1FA
:107F5000641CE4B2032CF4D34FF4147631460020B1
:107F600003F0FAFF0C4D31462860002003F0F4FFC7
:107F700068604FF40071002003F0EEFFA860032C4E
:107F800006D1296821B1696811B108B1002070BD1E
:107F9000012070BDE8BF02207C02002038B50446F5
:107FA00001F09CFA002807D16946204605F096F9B1
:107FB000002801D10021216038BD38B5044669464A
:107FC00005F08CF9002801D10021216038BD2DE990
:107FD000F7478DB014468A46002269460DA801F085
:107FE00063FD5FEA00097AD1009820600098D0E92B
:107FF0000516B21E914202D8CAF800106FE001784F
:108000000024012904D004291AD0D0F824803BE0B0
:1080100002250290294602A802F024F8411C03D050
:10802000012803D028B105E0012000E002208146AC
:108030004DE0641C00986D1C80698542EAD346E0DF
:108040000025B61EC76A00E045B939467F1C009876
:1080500003F0B8FE5FEA000939D1009A08205119EF
:1080600091F8341007E0CB0700D1641C4908401E8A
:10807000A6F1010601D0002EF5D16D1CC5F308054F
:10808000002EE1D123E065B9414608F101080098CE
:1080900003F098FE5FEA000919D1009F4FF40075C4
:1080A0003437009800780228384604D002F068F986
:1080B000000107D007E002F099F900B9641CAD1E79
:1080C000BF1C02E0641C2D1F3F1D761EDBD1CAF8C9
:1080D000004000984461017941F00101017110B044
:1080E0004846BDE8F0872DE9F74793B091460D4625
:1080F000002212A913A801F0D7FC060064D1F5B341
:108100001298B04600904146CDF808806846FFF7C7
:10811000EAFD060019D101216846FFF723FC06009D
:1081200013D112980078042813D0002002460D992C
:10813000095CA954401C521C0B2AF8D34046A85491
:108140001AB1521EA95C2029F9D0042E23D0B6B151
:108150003AE0002427464FF0020A13E00D990AEB9B
:108160004700084402F042F9002101F0CFFB80B142
:10817000FF2802D9010A2955641C285500E00DE0AA
:10818000641C7F1C0D984078B842E7D805F804803D
:10819000DBE73F20F1E785F800800026B9F1000F0A
:1081A00012D01298016A03F00DFE06000CD112994C
:1081B000087803280ED004280AD027200844343039
:1081C00002F0DEF8C9F8000016B03046BDE8F087CE
:1081D0006420F3E74320F1E72DE9FC4100259046B8
:1081E000074604464E1E0FE001AB01226946404699
:1081F00000F0CEFE0198012808D19DF800006D1C0A
:1082000004F8010B0A2801D0B542EDDB00202070F4
:1082100015B13846BDE8FC810020FBE72DE9F04FA1
:1082200087B017469946044602A905F057F85FEA59
:10823000000A6FD194F82900B0F1000AF9D1D4F8FE
:10824000488004F14C004FF0010B0190B8F1000F91
:1082500076D0F94371EA090135D0D4E90410CB1B7B
:1082600070EB090201D20F468146C4E90C7957EA46
:1082700009004FD07F1E49F1FF331D463A46204684
:10828000FEF7D0FA0146A0630298FEF7E4FA002850
:108290007ED002997A0A42EAC5524B895B1E1A4087
:1082A0001518208EC005E4D0E26BAA42E1D094F804
:1082B0002800400638D5487801230199FFF7F5FDDD
:1082C000002866D12AE058F8049BA1680226D1B1A3
:1082D0000025B61C00910F4620466D1C01F0C2FE21
:1082E0000146012854D9481C53D0781C8142F2D051
:1082F0004E4504D848F8045B009848F8040B0298EF
:1083000080698842E4D8A06C4E45066003D80020FE
:10831000C8F80000DEE04FF0110ADBE094F8280016
:1083200020F0400084F82800029801232A46407873
:108330000199FFF785FD00282BD1E563CAE0FFE72F
:10834000D4E90410CB1B70EB090205D294F8282065
:10835000920701D40F468146D4E90C01CDE904010E
:1083600000200090C4E90C0057EA09005FD0029891
:1083700040894FEA4028DDE90401084325D0781EF2
:1083800049F1FF3142460023F7F734FF054601E08B
:1083900078E08CE00E46DDE90401401E41F1FF313A
:1083A000424600230490F7F725FF281A8E410CD38C
:1083B000A8F10101CA430498002110403F1AC4E902
:1083C0000C0169EB0109A16B0CE0A16849B900211E
:1083D0002046FEF777FF0146012854D0481C66D09E
:1083E000A160A16319B30026B8EB0700354676EB10
:1083F00009000AD294F82800800720462AD5FEF703
:1084000061FF010029D14746B146D4E90C32DB199E
:1084100042EB0902C4E90C32F80508D00298FEF7D5
:108420001AFA78B3790A41EAC95108440090208EBB
:10843000C00542D0E26B009882423ED094F82800FA
:1084400040062CD50298012301994078FFF72DFDB5
:1084500068BB1EE001F006FE0146481C27D001293A
:1084600011D90298806988420DD9A163D4E90C30F2
:1084700013EB08026841C4E90C20B7EB080769EB6D
:108480000509B1E7FFE7022084F8290007B0BDE83D
:10849000F08F94F8280020F0400084F8280002981B
:1084A000DDE9002140780123FFF7CAFC18B184F808
:1084B00029B00120EAE70098E063D4E90C01D4E98F
:1084C0000423121A8B4105D2E4E90401207E40F016
:1084D000200020765046D9E72DE9F14F9AB00222CC
:1084E00001A91AA801F0E0FA0400019804907CD1D7
:1084F0004FF48C6001F030FA5FEA000910D016A842
:1085000004991290CDF8509009F50070C86004A845
:108510001A9901F071FC040006D0042C06D088E002
:1085200011201BB0BDE8F08F082482E0002104A8D0
:10853000FEF7C8FE5FEA000801984FF000021446FB
:1085400041894FEA4121CDE9081203D0B8F1010F6A
:1085500002D002E0072400E00224B8F1FF3F01D07E
:1085600014B104E0012402E003F01EFF044601F010
:108570000CFE0090D4BB41460198FEF76CF9019EB9
:10858000074634364FF400720021304602F093F86B
:1085900001984FF0100A007804282AD00B222021DD
:1085A000304602F088F82E25357086F80BA006F1CB
:1085B0001600009903F040FE42463146019803F050
:1085C00027FE06F1200020223146044602F06AF818
:1085D00086F821500198069A0178032903D1816A0F
:1085E000914200D10022214601E025E01CE003F089
:1085F0000FFE01984FF0010B458985B10198076383
:1086000080F803B07F1C03F0CFFE04000CD14FF4C0
:1086100000720021304602F04EF86D1EEED104A823
:10862000FFF714FA040009D00022414604A803F021
:108630007BFD484601F094F9204672E701980178E5
:10864000042914D0119C009904F1160003F0F4FDE4
:1086500042462146019803F0DBFD84F80BA0019906
:1086600081F803B0019803F05BFE0446E1E7C068BF
:1086700000990C3003F0E0FD01984146C0683430A9
:1086800003F0DAFD01980899C068383003F0D4FD92
:1086900001980899C068283003F0CEFD01980321A5
:1086A000C26882F82110C06880F804A004A803F012
:1086B000F4FDD7E72DE9F74F88B017460998012850
:1086C00003D913200BB0BDE8F08F08A801F0E2FD3C
:1086D000002801DA0B20F5E7FD4951F820504DB193
:1086E00000212970C0B20190FFF748FBC10703D0F9
:1086F0000320E7E70C20E5E7400701D50A20E1E782
:1087000003AA01210198FFF74DFB00287DD10398B2
:1087100080287AD3099909B1002100E03F218946D8
:10872000A0EB0901781E0742039100D17FB94FF4F5
:10873000FA60B1FBF0F20020E64B00E0401C33F899
:1087400010409442FAD8E34A163232F81070B7F566
:10875000007F00D37F0A87B1802F00D98027B1FB2B
:10876000F7F0012640F6F672904200D302264FF64B
:10877000F672904203D3032621E00127EFE7032E90
:108780001DD0012E25D04000001D00F2FF104FEA41
:1087900050284FF0010A2020834609EB0A0004907C
:1087A000404400EB0B04E219A2EB0900884247D8D1
:1087B00002AA03210198FFF7F5FAA8B90FE040F2E9
:1087C000072202EB80004FEA50284FF0200A0020D9
:1087D000E2E700EB4000401C4008C01CD5E70298CF
:1087E00010B1B0F5004F01D9012002902118401EB0
:1087F000491E8143081B0290032E13D08044039826
:10880000A0EB0A02A2EB080200E0D8E0A2EB0B0109
:10881000B1FBF7F10591022E09D0032E0CD0012EE9
:1088200012D016E00499824408440490E7E740F629
:10883000F672914204D30CE04FF6F670814201D2F9
:108840000E203FE70C200AE0B0F5803F06D2012061
:1088500005E0B0F5803F01D2042000E0062006903C
:10886000099808B1F02038E005F134004FF40072A7
:108870000021009001F01FFF05F5F97401206070E0
:10888000A0700020E07006982071FE2060710399AE
:1088900009EB010043F6C161B0FBF1F03F2141EA71
:1088A00090010290A171E0713F2104F1080003F0F2
:1088B000C3FC04F10C00039903F0BEFC4AF65521F9
:1088C00005F2322003F0E5FCDDE90010012300226F
:1088D000FFF7EBFA002872D1F82005F134044FF4C9
:1088E000007500902A460021204601F0E4FE0B228C
:1088F00079A1204601F0D6FE294604F10B0003F0D1
:10890000C8FC67731FFA8AF104F10E0003F0C1FC82
:1089100001202074032E0ED0410204F1110003F057
:10892000B8FC0399B1F5803F07D289B204F1130076
:1089300003F0AFFC05E00021EFE704F1200003F0B5
:108940007BFC009860753F2104F1180003F0A1FC46
:10895000FF2104F11A0003F09CFC494604F11C00BD
:1089600003F06AFC01F011FC802501464FF0290A52
:108970000290032E24D004F1270003F05DFC1FFABF
:1089800088F104F1160003F084FC84F8245084F884
:1089900026A0132253A104F12B0001F083FE04F55D
:1089A000FF704AF65521069003F073FC01234A46F6
:1089B00021460198FFF779FA002800D121E085E0EF
:1089C00004F1430003F038FC414604F1240003F0B5
:1089D00033FC022104F12C0003F02EFC012104F1F0
:1089E000300003F056FC062104F1320003F051FC84
:1089F00084F8405084F842A013223FA104F14700BC
:108A0000CBE7032E06D1012309F106022146019886
:108A1000FFF74BFA049D4FF0000A4FF4007200215B
:108A2000204601F048FE00980290032E13D0012E3C
:108A30000FD06FF0FF0101432046029103F0FCFBD1
:108A40002A466D1C012321460198FFF72EFAE8BB48
:108A500011E02E49EFE760F0FF012046029103F09C
:108A6000EBFB4FF0FF31201D03F0E6FB6FF0704190
:108A700004F10800E2E74FF400720021204601F003
:108A80001AFE012009E02A466D1C012321460198A7
:108A9000FFF70BFAD0B90298401C02904045F2D380
:108AA0000AF101005FEA000AB7D0032E00D05F464A
:108AB0002A466D1C012321460198FFF7F6F928B9D3
:108AC0007F1EF5D1032E4BD1114923E050E0000069
:108AD000DCBF0220D6D30008EBFE904D53444F5329
:108AE000352E30004E4F204E414D4520202020464F
:108AF00041542020202020004E4F204E414D452043
:108B000020202046415433322020200000FFFF0067
:108B100052526141204603F08FFB164904F5F27072
:108B200003F08AFB059904F5F470491E03F084FBF9
:108B3000022104F5F67003F07FFB4AF655210698F2
:108B400003F0A7FB012309F1010221460198FFF779
:108B5000ACF9012309F1070221460198FFF7A5F9B5
:108B6000002211460198FFF71DF900283FF4B3AD2C
:108B70000120A7E57272416117B581B014460298D1
:108B80000090684601F086FB002802DA0B2004B052
:108B900010BD0B4B002253F8201001B10A7001994F
:108BA000002900D00A7043F8201001D0012C01D018
:108BB0000020ECE7002201A902A800F075FFE6E71B
:108BC000DCBF02202DE9F74F98B004000DD04FF024
:108BD000000802F01F06324601A919A8C4F8008057
:108BE00000F062FF050004D006E109201BB0BDE8DB
:108BF000F08F019802904FF48C6000F0ADFE0700FA
:108C00000DD014A802991090129707F50070C86053
:108C100002A8199901F0F0F8050002D006E0112031
:108C2000E4E71098C07A000600D5062516F01C0F60
:108C30007ED04DB1042D03D102A8FEF707FF0546F3
:108C400046F008064DB1D4E09DF80E0010F0110F6B
:108C50006FD1700701D50825CBE030076AD501F048
:108C600094FA814601984FF0200A4FF0010B0178E9
:108C700004292AD00F9849460E3003F0DDFA0F98E8
:108C80004946163003F0D8FA0F9981F80BA00F99D6
:108C9000019801F062FB814600220F99019803F0D0
:108CA000B7FA0F9800211C3003F0C6FA0198B9F109
:108CB000000180F803B078D0D0F830A0002202A8DC
:108CC00003F032FA050055D093E020600198C068A7
:108CD000343001F055FBA0600198C068383001F0D5
:108CE0005AFBC4E904010198C16891F8211001F010
:108CF0000201E171C0684946083003F09DFA01980D
:108D00004546C16881F81480C06849460C3003F0BC
:108D100093FA0198C1684D75C268002182F804A0D9
:108D2000C068343003F088FA01980022C06802E07D
:108D30002BE036E03BE01346383003F085FA01982B
:108D400000221346C068283003F07EFA019902A879
:108D5000C96881F821B003F0A0FA050049D1A168E3
:108D6000D1B10022204603F0DFF90546A068019941
:108D7000401E07E05146019803F024F8054601998A
:108D8000A9F10100086175B133E095BB9DF80E00B3
:108D9000C10602D504252CE007E0B10703D5C007C2
:108DA00001D0072525E0300701D546F020060198BF
:108DB000016B21640F996164017804291ED00F9919
:108DC00001F0CBFAA0600F981C3001F0D9FAC4E989
:108DD0000408C4F8488084F829800021C4F83C8045
:108DE000C4E90C1184F82860019820600198C088BB
:108DF000A080384600F0B4FD2846F7E6C06834305D
:108E000001F0BEFAA0600198C068383001F0C3FAE2
:108E1000C4E904010198C06890F8210000F0020044
:108E2000E0710498E06106989DF80F1020F0FF00B3
:108E30000843206211986062CBE773B584B00400E8
:108E400007D00022694605A800F02EFE050003D0D9
:108E500055E0092006B070BD00994FF48C60216088
:108E600000F07AFD06000DD001A92664A1632168F7
:108E700006F50070C8602046059900F0BDFF0500AA
:108E800002D036E01120E5E7A06BC07A000628D4B6
:108E9000A079C00637D500980178042904D0616B09
:108EA00001F05BFAA0601CE0A268E2612169E2794E
:108EB00021F0FF0111432162E26B6262C06834302D
:108EC00001F05EFAA0600098C068383001F063FAE3
:108ED000C4E904010098C06890F8210000F0020184
:108EE000E1710098C188A18020460021FEF7FBFEB9
:108EF0000546304600F034FD042D06D00DB10020AB
:108F000020602846A6E70525F3E70525F7E700B525
:108F100095B00291002103910491014602A803F04B
:108F2000E4F8039800280DDB024601AB05A902987E
:108F300000F002FC30B901990398884202D10498EC
:108F400015B000BD4FF0FF30FAE710B596B00446FB
:108F50000020CDE90210049003E002A8641C03F095
:108F6000C4F821780029F8D1039800280DDB0246C7
:108F700001AB05A9029800F0DFFB30B90199039815
:108F8000884202D1049816B010BD4FF0FF30FAE7C6
:108F90002DE9FC5F894600259A4616460446694637
:108FA0001D6004F09BF900281AD194F829000028CC
:108FB00016D194F82800C00711D0D4E90C02D4E9E6
:108FC0000431181A04F14C0361EB02010193831B75
:108FD0004FF0010B71F1000100D206468EE0072030
:108FE000BDE8FC9F208EC0056CD1D4E90C2300980D
:108FF000550A45EAC3554089401E054013D152EA3F
:10900000030005D0A06C28B12046FDF70BFC05E05D
:10901000A06803E02046A16B01F024F8022819D3D0
:10902000411C49D0A063A16B0098FDF714FC88B1E6
:1090300000EB0508770A23D00098EA1941898A4293
:1090400000D94F1B40783B4642464946FEF7F8FEA2
:1090500090BB03E0022084F82900C1E794F82800BF
:1090600040060BD5E16BA1EB0800B84206D209EB34
:1090700040204FF40072019901F014FB7D022FE0B3
:10908000E26B42451CD094F8280040060CD50098AD
:10909000012301994078FEF708FF68B994F8280089
:1090A00020F0400084F828000098012342464078D0
:1090B0000199FEF7C5FE18B184F829B001208FE7A9
:1090C000C4F83C80208EC0F30800C0F50075B5429E
:1090D00000D9354601192A4648464C3101F0E2FADA
:1090E000D4E90C20521940F10000C4E90C20DAF850
:1090F0000000A9444119761BCAF80010002E7FF425
:1091000071AF00206CE72DE9FF410F46064603A929
:1091100004F0E4F804002FD1AFB14FF48C6000F0FC
:109120001BFC050015D0C6F838D03564316805F54C
:109130000070C86000213046FEF714FC0446042885
:109140000BD054B115E000213046FEF7CCFD0446AB
:1091500012E0112004B0BDE8F0813946304601F03C
:1091600016F800213046FEF77BFB0446042800D1A8
:109170000024284600F0F4FB2046EBE7F3B5B9B035
:109180003AA801F087F80222694639A800F08CFC61
:10919000040072D1009814904FF48C6000F0DCFB56
:1091A00005000DD036A814992290249505F500707D
:1091B000C86014A8399900F01FFE040003D09FE096
:1091C00011203BB0F0BD2298C07A10F0A00F01D062
:1091D000062495E000980178042913D021991522DE
:1091E00026A80B3101F05EFA482214A902A801F06A
:1091F00059FA02A83A9900F0FFFD040015D0042C9A
:109200003CD038E0C168402226A801F04BFA482241
:1092100014A902A801F046FA02A83A9900F0ECFD60
:10922000040002D0042C02D025E0082468E002A843
:10923000FEF70CFC040063D10098C068467890F8F3
:109240002340243001F0D2F807460098402226A996
:10925000C06801F027FA0098C06846700098C1689D
:1092600081F82340C0683946243003F012F802A880
:1092700003F013F804467CB342E044E002A8FEF792
:10928000E5FB04003CD10F9C13220DF19A0104F17F
:109290000D0001F007FA9DF89800012640F020002B
:1092A000E0720098C670E17AC90620D5049A169932
:1092B00091421CD0214601F050F801460098FDF77C
:1092C000CAFA010009D0009802F07CFD0400009861
:1092D00000F1540103D013E009E0022410E04A78C1
:1092E0002E2A04D1049A02F093FF0098C67014A8A5
:1092F000FEF7CAFC040003D1009803F011F80446FD
:10930000284600F02DFB20465BE700002DE9F143E5
:109310009AB0022218A91AA800F0C6FB002875D13D
:10932000189A002400921A9800E0641C015D20291C
:10933000FBD211784FF000090DF14808042930D113
:1093400000252E4628E01A99485D6D1CA0F1810287
:109350007D2A0ED8A5420BD2495DA1F140023E2ADA
:1093600002D9403A7E2A03D841EA00206D1C00E071
:109370000020012100F0CAFA07007DD001465648BE
:10938000FDF748FA002877D1162E75D008EB0600B5
:10939000394602F07EFFB61CA542D4D3344650E0D5
:1093A000641EA4B3011911F8011C2029F8D000256E
:1093B0008DF848902E461A99885D761CA0F181029E
:1093C0007D2A10D80A2D0DD2A6420BD2895DA1F1BB
:1093D00040023E2A02D9403A7E2A03D841EA0020C0
:1093E000761C00E00020012100F090FA00F0BCFAA9
:1093F000002100F08BFA07004BD001463648FDF7FC
:1094000009FAC8BBFF2F03D90A2002E042E018E0A6
:109410000B20A8423DD9FF2F03D9390A08F80510BF
:109420006D1C404608F805706D1CA642C3D3202170
:109430000B2D02D241556D1CFAE79DF84800E52836
:1094400027D000216846CDF80890FEF74CFC002894
:1094500020D101216846FEF785FA0125E8B10428EC
:1094600018D10020002C15D001216846FEF72EF9F6
:1094700000280FD1202200E00BE000210D9801F020
:109480001AF918980078042822D00D990820C8727B
:1094900008E006201BB0BDE8F08318980078042887
:1094A00004D06CB10B2212A90D9806E00D9960084A
:1094B000224648700D9812A9801C01F0F3F802E0D2
:1094C0000D99E52008701898C57002F029FFE1E7B2
:1094D0000D9983200870E9E7C5D30008F0B593B073
:1094E000044612A903F0FAFE050023D194F82800DF
:1094F00081061FD5400611D51298E26B01234078F2
:1095000004F14C01FEF7D1FC10B1012013B0F0BD05
:1095100094F8280020F0400084F8280000F035FE80
:10952000064612980178042905D0216C02F04AFC05
:10953000050055D079E0204600F056FA050074D1B8
:109540004FF4187000F008FA070008D0129821466E
:10955000C760684600F04FFF050002D03CE01120D4
:10956000D4E71298C1680A7942F020020A71E179C1
:10957000C26841F0010182F82110C068A16834304E
:1095800002F05AFED4E904231298C068383002F081
:109590005BFED4E904231298C068283002F054FE20
:1095A00012983146C0680C3002F046FE1298002135
:1095B000C2685175C068103002F03EFE684602F085
:1095C0006CFE050008D1129802F0AAFE054614F8B8
:1095D000280F20F020002070384600F0C1F924E068
:1095E000656C2946E87A40F02000E872A26820689D
:1095F00002F00EFE05F11C00216902F01DFE31464D
:1096000005F1160002F018FE002105F1120002F02B
:1096100040FE12980121C17002F082FE054694F8C6
:10962000280020F0200084F8280028466EE771B555
:10963000B3B002222EA933A800F036FA04002E9807
:10964000009077D14FF48C6000F086F905000DD0C2
:109650002FA800990E90109505F50070C860684617
:10966000339900F0C9FB040003D060E0112034B04E
:1096700070BD0E98C07A000601D5062457E09DF80B
:109680000600C00701D0072451E02E9824900178ED
:1096900004290ED00D9900F060FE06469DF80600E4
:1096A000C00633D52E98149612900078042816D050
:1096B0001DE0C068343000F063FE064626902E9808
:1096C000C068383000F067FECDE928012E98C068E8
:1096D00090F8210000F002008DF89700DEE7DDE948
:1096E0002801CDE916019DF897008DF84F00002163
:1096F00012A8FEF7F8FA040019D1002112A8FEF70B
:1097000031F90400BFD0042C00D084B96846FEF7BC
:10971000BBFA04000BD136B10022314624A802F076
:1097200003FD040003D12E9802F0FAFD04462846FA
:1097300000F016F920469AE72DE9FC5F89464FF0C4
:10974000000B9A46164604466946C3F800B003F07B
:10975000C5FD002808D194F82900002804D194F808
:109760002800800702D40720BDE8FC9F00980178FC
:1097700004F14C000190042907D1D4E90C108A1996
:1097800040EB0B03511A834102D3206B811901D3A3
:10979000206BC643B0E0208EC0057FD1D4E90C23F6
:1097A0000098550A45EAC3554089401E05401AD124
:1097B00052EA030005D0A06C38B12046FDF732F81C
:1097C00007E0A06838B9002100E0A16B2046FDF752
:1097D00079FD00287DD001282ED0411C57D0A063F0
:1097E000A16801B9A06094F8280040060DD5009842
:1097F000E26B012340780199FEF757FBA0BB94F878
:10980000280020F0400084F82800A16B0098FDF7A4
:1098100022F888B100EB0508770A26D00099EA19EA
:109820004889824200D9471B48783B464246494610
:10983000FEF73BFBC0B903E0022084F8290093E760
:10984000E16BA1EB0800B8420CD209EB40214FF4C8
:109850000072019800F026FF94F8280020F04000E4
:1098600084F828007D022DE011E0E16B414513D022
:10987000D4E90413D4E90C20511A98410CD2009871
:109880000123424640780199FEF7DAFA20B101201F
:1098900084F8290068E701E0C4F83C80208EC0F31A
:1098A0000800C0F50075B54200D9354620442A4667
:1098B00049464C3000F0F6FE94F8280040F0400095
:1098C00084F82800D4E90C134A19A94443EB0B038C
:1098D00000E014E0C4E90C23D4E904108F1A70EB03
:1098E000030701D211461846C4E90410DAF8000053
:1098F0004119761BCAF80010002E7FF44CAF14F803
:10990000280F40F02000207000202DE770B580283F
:109910001BD345F2205409B10D4D00E00D4D00233D
:109920001022E11A01EBD17103EB610135F82160DE
:10993000864206D001D20B4600E00C46521EF0D102
:1099400004E01AB105EB8100408870BD002070BDB5
:109950008628020802D400080146002002F0FCBA62
:109960000146002002F0ECBA30B5B0F5805F01D2BC
:109970001B4900E01B4931F8022B002A15D0904208
:1099800013D331F8023B1C0ADDB252FA83F383424F
:1099900021D9092C09D2DFE804F005090E111315AD
:1099A00017191B00801A31F8100030BD811A01F020
:1099B0000101401A00E0103880B230BD2038FBE7CA
:1099C0003038F9E71A38F7E70830F5E75038F3E7A9
:1099D000A0F5E350F0E7002CCDD101EB4501CAE73B
:1099E0000A7D0308FC7E030870B50646C07903288B
:1099F0000FD1B569B46808E0621C2146306802F0F6
:109A0000F9FA002806D1641C6D1E002DF4D1002047
:109A1000F071002070BD2DE9F047064680698F1E69
:109A2000801E9246B84200D800273C46B846002522
:109A3000F06A00EB1431304602F0C4F918B14FF06F
:109A4000FF30BDE8F08704F0070201209040B269C2
:109A5000C4F3C801C0B24FF480534FF40079921E92
:109A600006EB010C641C9CF834C00CEA000C4006A8
:109A7000000E944202D3002420461946BCF1000F88
:109A800005D0A0460025BC4207D10020D9E76D1CB7
:109A90005545F8D108F10200D3E70028E0D10120B4
:109AA000491C4945DCD3C3E72DE9FF5F00279046F9
:109AB0000E460F6000F0EEFB050003D50B2004B04E
:109AC000BDE8F09FC84850F825409CB1346020782C
:109AD00028F0010620B16078FEF7E5F9C1070BD048
:109AE0002770E8B2B8466070FEF748F9C10708D0A1
:109AF0000320E4E70C20E2E70EB1400704D4002085
:109B0000DDE71EB1400701D50A20D8E70025294628
:109B10002046FCF727FE022820D16E4604EB0510F4
:109B200090F8F61100F5F97019B1083000F028FC32
:109B300000E0002046F825006D1C042DEED3002720
:109B400056F8275025B129462046FCF70BFE00E0C9
:109B50000320022802D37F1C042FF1D3042879D0DC
:109B6000022879D24FF0FF3A4FF4007601280CD04A
:109B700004F13F0000F03AFCB0426DD104F14A001C
:109B800000F034FC002868D083E00B2002E0401C89
:109B9000402806D2211891F834100029F7D0402827
:109BA0005AD304F19C0000F021FCB0F5807F53D122
:109BB00094F8A000012707FA00F0B34658454BD1AE
:109BC00004F17C0000F0E7FBC14610EB050841EB17
:109BD0000906012E40D204F1880000F0D1FBE061BB
:109BE00094F8A200A070012836D194F8A100874013
:109BF0003804000C60812FD004F1900000F0C0FB0D
:109C00000746801CA061B0F1004F25D204F18C0002
:109C1000256200F0B5FB2844E06204F1840000F006
:109C2000AFFB284460626189E06A07FB0101B8EB81
:109C3000010176EB09060FD304F1940000F0A0FBBC
:109C40000146A0622046FCF706FE0146204602F0CF
:109C5000B9F818B1012032E766E016E000255E464B
:109C6000601990F83410812904D1483000F088FB45
:109C7000022802D02035B542F2D3B54263D0C4F8F1
:109C800014A00426C4F810A0A7E004F1580000F0C6
:109C900077FBE06194F84470A770012F01D0022F88
:109CA00051D1474394F841006081E8B3411E084216
:109CB00049D104F1450000F099FB2081000742D111
:109CC00004F1470000F092FB060004D104F15400B7
:109CD00000F056FB064604F1420000F087FB01004D
:109CE00031D02389C81900EB131296422BD3B01A36
:109CF0006689B0FBF6F0B8B1012640F6F67C604507
:109D000000D302264FF6F67C604500D30326801C64
:109D10002A44E2622944A061C4E90851032E14D008
:109D200013B13944A16200E00DE0022E1ED000F014
:109D3000010100EB400001EB5000E16900F2FF106F
:109D4000B1EB502F14D20D20B9E604F15E0000F003
:109D50004DFB0028F7D120890028F4D104F16000E0
:109D600000F00EFBA062A0698000E6E74000E4E797
:109D7000C4F814A08020C4F810A02071032E2CD1A8
:109D800004F1640000F032FB012826D1691C204652
:109D900002F018F808BB84F8048004F2322000F0C6
:109DA00025FBA0F52A41553917D104F1340000F004
:109DB000E7FA0E49884210D104F5067000F0E0FA87
:109DC0000B49884209D104F5077000F0D9FA6061A7
:109DD00004F5087000F0D4FA20610649267008885E
:109DE000401C0880E0808AE6DCBF022052526141BC
:109DF000727241617802002073B5044605680198CB
:109E000001E0401C019001782F29FAD05C29F8D09C
:109E10000021A16001980078202807D2A16B802042
:109E2000C87200212046FDF75EFF7CBD01A92046D7
:109E3000FDF7D0FA0028F8D12046FDF773FCA16B9E
:109E4000C97A28B10428F0D14907EED405207CBD99
:109E50004907FCD4A079C006F8D52878042809D091
:109E6000208DC0F3080041192846343100F075FAFE
:109E7000A060DBE7A168E1612069E17920F0FF00E3
:109E800008432062E16B6162E868343000F078FAE0
:109E9000A060E86890F8210000F00201E171E86834
:109EA000383000F078FAC4E90401BFE703490A68D2
:109EB0005206FCD5C2B24A60704700000010014053
:109EC00010B5002821D0114B0022001F196803E0B3
:109ED000814203D80A4649680029F9D152B1136872
:109EE000841A9C4204D1006818441060104602E0B5
:109EF000506000E0186039B102680B1A934203D138
:109F00000B681A4402604968416010BD9402002049
:109F100070B50E460546002405E055F824100120D2
:109F200002F00EF8641CB442F7DB2946BDE870402D
:109F3000012002F005B800007CB516461C46054617
:109F40000B2200F0AFFB052C11D91D4A0CE00021BB
:109F5000B61C2346044663F35F044008E30300D5C0
:109F60005440491C1029F4D330880028EFD107222F
:109F70006B4604F00F003030392800D9C01D9854CA
:109F8000521E2409F5D17E2000219854541E06E06B
:109F900081387D2802D8A14206D0491C491C914233
:109FA00002D2685C2028F3D1082A02D2985C521CA5
:109FB00000E020206854491C0829F5D37CBD00002E
:109FC00021100100F0B5DFED250A002404EBC405E3
:109FD000002305EB041503EB850602EB86065B1CEC
:109FE000C6ED000A642BF6DB641C642CEEDB6423F4
:109FF0009FED1B1A91FBF3F6C0EE010A00232AE045
:10A0000000EB830494ED000AB0EEC00AB5EEC00A7E
:10A01000F1EE10FA1ED093FBF6F4642C00DB6324FF
:10A0200080EE201ABDEEC10A10EE105AD5F163057C
:10A0300000D5002505EBC50707EB051504EB8504E6
:10A0400002EB8404B7EE001A94ED000A30EE010A28
:10A0500084ED000A5B1C8B42D2DBF0BD00000000E7
:10A060000000C8422DE9F04104680D46022972D370
:10A07000A169A9426FD921784FF0FF36012909D093
:10A0800002292CD0F20D02EA8507032936D00429D3
:10A0900077D141E0606A05EB550700EB5721204678
:10A0A00001F090FE00286DD1C7F3080020447F1C0A
:10A0B00090F83480606A00EB5721204601F082FE60
:10A0C00048BBC7F30800204490F8341048EA012048
:10A0D000E90701D0060955E0C0F30B0652E0606ABB
:10A0E00000EB1521204601F06DFEA0B9E8B204EBAB
:10A0F0004000343000F07AF9064643E0606A00EB35
:10A10000D511204601F05EFE28B93819343000F030
:10A1100037F920F0704635E0D0E9041351EA030224
:10A120002FD08268AA1A491E43F1FF33490A41EA37
:10A13000C3516389B1FBF3F3C17902290CD0032920
:10A1400013D002291DD0606A00EBD511204601F022
:10A1500039FEB8B90EE014E09A4212D802D16FF07D
:10A1600000460FE005F101060CE080699042EAD953
:10A170006E1C07E03819343000F002F920F0004678
:10A1800000E001263046BDE8F081002070472DE94F
:10A19000F0474FF00009064681F81A90006B0C4614
:10A1A000002875D030680178042905D0F06B401C78
:10A1B00020D00025376C16E0C0682146BDE8F04786
:10A1C00000F086B80021FFF7A1FB38B1FF2803D9C2
:10A1D000010A62196D1C9176FF2D01D3002506E05E
:10A1E00061196D1C887637F8020B0028EAD16119D5
:10A1F00081F81A900021A37E0A464FF02E0C706B56
:10A20000805C521C202822D0052800D1E520092A94
:10A2100007D113B9651885F81AC06518491C85F867
:10A220000DC0651868738BB9A0F14107192F0CD8C0
:10A23000776B092A97F80C8001D3102700E00827D4
:10A2400018EA070F01D02030C0B2A876491C0B2AAB
:10A25000D5D333B9621882F81A90706B007B00B9BD
:10A26000002160184D4680F80D90706BC07A207305
:10A27000706B1C3000F084F8C4E90005706B183076
:10A2800000F0B4F82081706B163000F0AFF86081F8
:10A29000BDE8F08710B503464FF0FF301C68002C76
:10A2A00013D0214600E0491C0A78202A0ED33A2A0E
:10A2B000F9D114F8012B303A0A2A06D28C4204D183
:10A2C000032A02D2491C1046196010BD002010BD9F
:10A2D0002DE9F041402700260C460546B04617E020
:10A2E000F80600D1BF1CE81900F080F80021FFF744
:10A2F0000DFB90B1FF2803D9010AA219761C9176B3
:10A30000FF2E0AD2A119761C887608F10108BF1C1D
:10A3100095F823104145E3D816B93F20A0760126D1
:10A32000A11900208876607328792073C00602D5B1
:10A330000020014603E005F1380000F02CF8C4E9E4
:10A34000000105F10C0000F051F8608105F10E00EC
:10A3500000F04CF82081BDE8F08170B506460D464E
:10A3600001F11A0000F042F804463078032805D1C4
:10A3700005F1140000F03AF844EA0044204670BDAC
:10A38000C178827842EA01214278007842EA0121CC
:10A3900040EA0120704710B5C17982790B0E42EA7C
:10A3A00001211A02437942EA116243EA01211302B0
:10A3B000027943EA116342EA01211A02C37842EAB0
:10A3C000116243EA0121130243EA116382781B02FE
:10A3D00042EA012143EA11630A02417800780A4304
:10A3E000190241EA126140EA022010BD417800786A
:10A3F00040EA0120704710B5044608682060C8692B
:10A40000A06091F82000E071086A002220F0FF00AF
:10A41000C4E90402496A2046E163FDF764FC0028B0
:10A4200004D12046BDE8104000F001B810BD2DE970
:10A43000F04104460068216BC66801F0C3FC0028A7
:10A4400022D1616B0878852842D12022304600F065
:10A4500029F97778002120467F1CFDF701FA0028B2
:10A4600012D1216B206801F0ADFC00280CD1616B8A
:10A470000878C0282CD1202206F1200000F012F923
:10A48000F81E112802D30420BDE8F08140257F0189
:10A4900000212046FDF7E4F90028F5D1216B206862
:10A4A00001F090FC0028EFD1616B0878C1280FD132
:10A4B0007019202200F0F6F82035BD42E8D330466E
:10A4C00002F027FF0446B01CFFF790FF844201D042
:10A4D0000220D9E70020D7E71CB5F7F783FB082354
:10A4E000022219214FF4B470FAF74EFCB420FDF7A4
:10A4F000BBF84FF4165001F081FFF9F783FEF9F72E
:10A500009DF8002001F0A4FC012001F0A1FC00F066
:10A5100087FD42F2273141F28730FAF7A9FC28483B
:10A5200041685A208847FAF7ADF8264D040010D04C
:10A5300025A0FBF7B1F84FF4FA763046FDF79EF808
:10A54000D5F88402002837D00021C5F88412002CE9
:10A55000F3D1F7F74BF8FDF7EFFC2048012220A1DB
:10A560000068FEF709FB4FF40071012001F0F4FCD4
:10A570001C4901AA0860694619A0FDF7C6FC040041
:10A580000DD019A0FBF788F86420FDF777F8D5F80F
:10A59000840298B10021C5F88412002CF4D118A0CF
:10A5A00000F06AFF17A0FBF777F81C4C2078002812
:10A5B000FCD0FCF79FF9F9E70121C6E70121EAE7A2
:10A5C0008401002000804042534420436172642093
:10A5D0004572726F72210D0A00000000E8BF022070
:10A5E000303A00008402002053442043617264200A
:10A5F0004661746673204572726F7221000000001C
:10A60000616C6C00E5889DE5A78BE58C96E5AE8CCA
:10A61000E68890EFBC810D0A000000009102002046
:10A62000F0B50B30154D20F007010024144A0FE05F
:10A6300003688B420BD38B4205D95E1A43184768D7
:10A64000C3E9006700E04368136002C004E0021D34
:10A6500010680028ECD12046002802D1286808B1F3
:10A660000020F0BD064A07481060074A121A22F07F
:10A670000702C0E9002401202860D7E798020020E3
:10A68000940200207CC2022078C4022010B510F889
:10A69000013B11F8014B1B1B521E01D0002BF6D0C1
:10A6A000184610BD002A05D011F8013B00F8013B07
:10A6B000521EF9D17047C9B200F8011B521EFBD1DE
:10A6C00070470000034810B50068FDF767FC0020E4
:10A6D00010BD00007C0200200148FDF76EBC0000A8
:10A6E00018C10220FDF7E6BF10B586B00446002071
:10A6F000059005AA69462046FDF7F5FC010004D047
:10A7000007A0FAF7C9FF06B010BD6A4621460AA0A5
:10A71000FAF7C2FF21460EA0059AFAF7BDFFF2E74D
:10A720000D0ABBF1C8A1CAA7B0DCA3ACB4EDCEF34F
:10A73000C2EB3A25580D0A000D0AB4C5C5CC2573E5
:10A7400020B5C4C5CCB7FBCEAA3A25730D0A0000CC
:10A75000B4C5C5CC257320B5C4D0F2C1D0BAC53AB2
:10A7600025580D0A0D0A000010B50146074A084891
:10A7700012680068FDF730FD01460078002804D01B
:10A78000BDE8104003A0FAF787BF10BD7C0200208F
:10A79000840200200D0A54686520537472696E6744
:10A7A000205265616465642049733A25730D0A007F
:10A7B0000246024800230068FDF730BD7C020020FD
:10A7C000FDF78ABE034603480A4619464068FEF76D
:10A7D000D3B90000E8BF02200A46014601480068DC
:10A7E000FEF7F0B97C02002001460148FEF725BBC8
:10A7F00018C10220034910B50968FEF788FBC0B2F2
:10A8000010BD00007C020020034910B50968FEF766
:10A810009CFBC0B210BD00007C0200202DE9F05F5F
:10A8200080460026354632A0FAF736FF0027DFF8CB
:10A83000D8A0DFF8D8B026E03548344B4FF400728A
:10A84000D146DAF800100068FEF7A2FB060004D03B
:10A85000014630A0FAF720FF18E0BBF80010CA4606
:10A8600029448DB20024D94607E0DAF80000015DE2
:10A870002CA0FAF711FF641CA4B2D9F8000084429E
:10A88000F3D37F1CBFB2B7EB582FD5D35FEAC850C4
:10A8900022D01F48C8F308021C4BD046DAF800103B
:10A8A0000068FEF775FB060004D001461EA0FAF70B
:10A8B000F3FE11E0BBF800005F46284485B2002497
:10A8C00007E0D8F80000015D16A0FAF7E5FE641C69
:10A8D000A4B238688442F4D31DB1294617A0FAF710
:10A8E000DBFE1CA0FAF7D8FE3046BDE8F09F000062
:10A8F0000D0A526561642066696C6520646174614B
:10A900002069733A0D0A00008402002088020020AA
:10A910007C02002052656164204572726F723A2594
:10A92000640D0A00256300000D0A5265616420452C
:10A9300072726F723A25640D0A0000000D0A5265AA
:10A94000616465642064617461206C656E3A25649D
:10A950000D0A0000526561642064617461206F76A5
:10A9600065720D0A0000000010B525492548FEF764
:10A97000CAFB002842D124A0FAF78EFE214C26A063
:10A98000A16AFAF789FEA18827A0FAF785FE2AA016
:10A99000A168FAF781FED4E904232CA0FAF77CFE23
:10A9A00030A0616AFAF778FE33A0E16AFAF774FE24
:10A9B00035A0216BFAF770FE37A0E16BFAF76CFE59
:10A9C00014A0FAF769FE0E4938A01A31FAF764FEAE
:10A9D0000B4C3BA0D4E90023FAF75EFE21893DA091
:10A9E000FAF75AFE618940A0FAF756FE217B43A090
:10A9F000FAF752FE07A0FAF74FFE002010BD000044
:10AA0000F8BF022018C102200D0A204449522069D3
:10AA10006E666F3A0D0A00006469722E647074727B
:10AA20003A25640D0A0000006469722E6F626A2E76
:10AA300069643A25640D0A006469722E6F626A2E99
:10AA400073636C7573743A25640D0A006469722E21
:10AA50006F626A2E6F626A73697A653A256C6C64FC
:10AA60000D0A00006469722E6F626A2E635F6F6662
:10AA7000733A25640D0A00006469722E636C757365
:10AA8000743A25640D0A00006469722E736563745C
:10AA90003A25640D0A0000006469722E626C6B5FD7
:10AAA0006F66733A25640D0A0000000046696C6504
:10AAB000204E616D652069733A25730D0A00000010
:10AAC00046696C652053697A652069733A256C6C18
:10AAD000640D0A0046696C652064617461206973C5
:10AAE0003A25640D0A00000046696C652074696DA2
:10AAF000652069733A25640D0A00000046696C659B
:10AB000020417474722069733A25640D0A000000B4
:10AB1000FEF734BB70B5064601460F48FEF78DF9C7
:10AB2000002817D10DA0FAF7B7FD0D4C04F11A0556
:10AB30000B490948FEF7E7FA00280BD1A17E00294E
:10AB400008D0314607A0FAF7A7FD294606A0FAF774
:10AB5000A3FDEDE770BD000018C102200D0A000042
:10AB6000F8BF022025732F0025730D0A0000000096
:10AB700010B50446FEF7CAFB010004D003A0BDE8EF
:10AB80001040FAF789BD214608A0F8E70D0AB4C5C0
:10AB9000C5CCC5CCB7FBC9E8D6C3CAA7B0DCA3AC4B
:10ABA000B4EDCEF3C2EB3A25580D0A000D0AB4C538
:10ABB000C5CCC5CCB7FBC9E8D6C3B3C9B9A63A253D
:10ABC000730D0A001CB5034600200446009001AA3C
:10ABD00069461846FDF7FBF990B9019988694C89D7
:10ABE000801E009960434C43B0F5A04F03D2620829
:10ABF000410804A002E0C10AE20A0CA0FAF74CFDE9
:10AC000020461CBD0D0AB4C5C5CCD7DCC8DDC1BF0C
:10AC10003A2564204B420D0ABFC9D3C3BFD5BCE45B
:10AC20003A2564204B420D0A000000000D0AB4C50D
:10AC3000C5CCD7DCC8DDC1BF3A2564204D420D0A22
:10AC4000BFC9D3C3BFD5BCE43A2564204D420D0A29
:10AC50000000000001480068006970477C02002085
:10AC600001480068006B70477C020020FEF7DFBCE3
:10AC700070B505460C460EA0FAF70EFD214612A04F
:10AC8000FAF70AFD1648154B224629460068FEF7DA
:10AC900053FD040002D0014612A002E00F480168F3
:10ACA00015A0FAF7F9FC1AA0FAF7F6FC204670BDD9
:10ACB0000D0A426567696E2057726974652066697E
:10ACC0006C652E2E2E0D0A00577269746520646122
:10ACD0007461206C656E3A25640D0A008C020020B8
:10ACE0007C0200205772697465204572726F723A57
:10ACF00025640D0A000000005772697465642064C1
:10AD0000617461206C656E3A25640D0A00000000D4
:10AD100057726974652064617461206F7665722E64
:10AD20000D0A000010B504462EA1F5F7CBFA002855
:10AD300037D02FA12046F5F7C5FA002833D030A12F
:10AD40002046F5F7BFFA002830D030A12046F5F7AD
:10AD5000B9FA00282DD031A12046F5F7B3FA002822
:10AD60002AD031A12046F5F7ADFA40B332A12046F2
:10AD7000F5F7A8FA30B333A12046F5F7A3FA20B3CC
:10AD800033A12046F5F79EFA10B334A12046F5F71B
:10AD900099FA00B334A12046F5F794FAF0B10020F7
:10ADA00010BD334810BD3248143010BD3048283033
:10ADB00010BD2F483C3010BD2D48503010BD2C48E0
:10ADC000643010BD2A48783010BD29488C3010BD41
:10ADD0002748A03010BD2648B43010BD2448C830E4
:10ADE00010BD0000636F6E76315F626961730000B1
:10ADF000636F6E76315F7765696768740000000085
:10AE0000636F6E76325F626961730000636F6E76A6
:10AE1000325F77656967687400000000636F6E7663
:10AE2000335F626961730000636F6E76335F7765CD
:10AE300069676874000000006663315F626961736E
:10AE4000000000006663315F776569676874000021
:10AE50006663325F62696173000000006663325F9F
:10AE600077656967687400006461746100000000C0
:10AE700060C102200248416802A0FAF70DBC000040
:10AE800028C202200D0A64617461736574206973BD
:10AE90003A2025730D0A000010B5044620A1F5F7ED
:10AEA00011FA00281AD02046FFF73CFF002814D0E2
:10AEB0002046FFF737FF044601681AA0FAF7ECFBBB
:10AEC0001EA0A168FAF7E8FB24A0E168FAF7E4FB0A
:10AED00029A02169FAF7E0FB012010BD2DA0FFF7A2
:10AEE000DBFF2FA0FFF7D8FF31A0FFF7D5FF33A07E
:10AEF000FFF7D2FF35A0FFF7CFFF37A0FFF7CCFF5A
:10AF000039A0FFF7C9FF3BA0FFF7C6FF3CA0FFF742
:10AF1000C3FF3EA0FFF7C0FF3FA0FFF7BDFFDBE789
:10AF2000616C6C000D0A6D6F64656C2E6E616D65F1
:10AF30002069733A2025730D0A0000006D6F646567
:10AF40006C2E61727261792E616464726573732014
:10AF500069733A20305825580D0A00006D6F6465FA
:10AF60006C2E6D61786C656E6774682069733A2029
:10AF700025640D0A000000006D6F64656C2E72651B
:10AF8000616C656E6774682069733A2025640D0AE8
:10AF900000000000636F6E76315F626961730000CC
:10AFA000636F6E76315F77656967687400000000D3
:10AFB000636F6E76325F626961730000636F6E76F5
:10AFC000325F77656967687400000000636F6E76B2
:10AFD000335F626961730000636F6E76335F77651C
:10AFE00069676874000000006663315F62696173BD
:10AFF000000000006663315F776569676874000070
:10B000006663325F62696173000000006663325FED
:10B01000776569676874000064617461000000000E
:10B0200070B5324C2EA0206000F048FDA0602020BA
:10B03000E06014342EA0206000F040FDA0604FF4CA
:10B040009070E06014342EA0206000F037FDA06006
:10B050004020E06014342DA0206000F02FFDA0609F
:10B060004FF49040E06014342CA0206000F026FDE6
:10B070008025C4E9020514342BA0206000F01EFDD9
:10B08000A0604FF49030E06014342BA0206000F0FA
:10B0900015FDC4E9020514342AA0206000F00EFD5D
:10B0A000A0604FF41010E060143429A0206000F07C
:10B0B00005FDA0600720E060143428A0206000F0A7
:10B0C000FDFCA0604FF46070E060143426A02060A6
:10B0D00000F0F4FCA0602648E06023A0606070BD32
:10B0E000636F6E76315F62696173000060C1022038
:10B0F000636F6E76315F7765696768740000000082
:10B10000636F6E76325F626961730000636F6E76A3
:10B11000325F77656967687400000000636F6E7660
:10B12000335F626961730000636F6E76335F7765CA
:10B1300069676874000000006663315F626961736B
:10B14000000000006663315F77656967687400001E
:10B150006663325F62696173000000006663325F9C
:10B1600077656967687400006461746100000000BD
:10B17000D01213002DE9FC5F8A469B469046044698
:10B1800048A1F5F79FF890B12046FFF7CBFD0500E9
:10B190004FD0B8F1000F4CD02869504549D34045F5
:10B1A00047D3002845D00026A8EB0A0960E05B469B
:10B1B000424651463CA0FFF7DDFF5B464246514602
:10B1C0003CA0FFF7D7FF5B46424651463DA0FFF744
:10B1D000D1FF5B46424651463DA0FFF7CBFF5B46A1
:10B1E000424651463EA0FFF7C5FF5B4642465146E8
:10B1F0003EA0FFF7BFFF5B46424651463FA0FFF728
:10B20000B9FF5B46424651463FA0FFF7B3FF5B469E
:10B21000424651463FA0FFF7ADFF5B4642465146CE
:10B220003FA0FFF7A7FF5B46424651463FA0FFF70E
:10B23000A1FF0020BDE8FC9F06EB0A07A868A74213
:10B2400002D200EB870004E06FF0030101EB840100
:10B2500008440068F5F7B6F8A742CDE9000101D22D
:10B260003A4600E0621E33A02968FAF715FA5E44F8
:10B270002C69444501D2204607E0B9FBFBF20BFBE9
:10B28000129008B1022000E00120444501D221467D
:10B2900000E049460844B042CED82CA0FAF7FCF9A9
:10B2A0000120C7E7616C6C00636F6E76315F626985
:10B2B00061730000636F6E76315F776569676874EC
:10B2C00000000000636F6E76325F62696173000098
:10B2D000636F6E76325F776569676874000000009F
:10B2E000636F6E76335F626961730000636F6E76C1
:10B2F000335F776569676874000000006663315FDB
:10B3000062696173000000006663315F7765696799
:10B31000687400006663325F626961730000000058
:10B320006663325F776569676874000064617461A1
:10B33000000000000D0A25735F666C6F6174417236
:10B340007261795B25645D3A202566000D0A000074
:10B350002DE9F0410646F4F7AEFFC4B204F108004F
:10B360000746FFF75DF905461848806810B118A038
:10B3700000F0BCFA324618A12846FAF79DF91948A0
:10B38000012229460068FDF71DFC10B1314616A0C8
:10B3900014E0304600F070F8314670B119A0FAF7A9
:10B3A0007BF92B463A4621461DA0F5F711FE2846AB
:10B3B000FEF786FD0120BDE8F08127A0F5F708FE25
:10B3C0002846FEF77DFD0020F5E7000028C2022098
:10B3D0006461746100000000303A2F25732E747888
:10B3E000740000007C0200200D0A44617461CAFDF3
:10B3F000BEDDBCAF5B25735DB2BBB4E6D4DA0D0A2B
:10B400000000000044617461CAFDBEDDBCAF5B2575
:10B41000735DC7D0BBBBB3C9B9A6A3A10D0A000019
:10B42000646174615F6E616D65B5C4B3A4B6C8CE66
:10B43000AAA3BA25640D0A5F70617468B5C4B3A489
:10B44000B6C8CEAAA3BA25640D0A5F70617468CE2F
:10B45000AAA3BA25730D0A0044617461CAFDBEDD5A
:10B46000BCAF5B25735DC7D0BBBBCAA7B0DCA3A1D3
:10B47000A3A10D0A000000002DE9F04F9FB0814606
:10B4800092A1F4F71FFFD8B10027B8463D464846C1
:10B49000F4F711FFC0B22630FFF7C2F81C907021FC
:10B4A0006846F4F7F1FE4846FFF73CFC884E04007E
:10B4B0002DD088A14846F4F705FF002827D03FE0AB
:10B4C00086A0FFF7D9FF88A0FFF7D6FF8AA0FFF775
:10B4D000D3FF8CA0FFF7D0FF8EA0FFF7CDFF90A089
:10B4E000FFF7CAFF92A0FFF7C7FF94A0FFF7C4FFC2
:10B4F00095A0FFF7C1FF97A0FFF7BEFF73A0FFF76E
:10B50000CBFCF8F7F1FE00201FB0BDE8F08F4A46F3
:10B5100093A11C98FAF7D0F801221C993068FDF726
:10B5200051FB38B191A0F5F753FD1C98FEF7C8FC0C
:10B53000C720E9E767A0FFF7F5FB0446C0F80490D1
:10B54000606898B986A122681C98FAF7B5F80122BC
:10B550001C993068FDF736FB40B18FA01C99F5F7B8
:10B5600037FD1C98FEF7ACFC0420CDE7A06820B99D
:10B57000206800F0A3FA002813D08EA02168F5F708
:10B5800027FD616811B192A0F5F722FD97A0E1684F
:10B59000F5F71EFD9EA02169F5F71AFD616851B906
:10B5A00008E0A3A02168F5F713FD1C98FEF788FCBE
:10B5B000C820A9E72168A8A0FAF76EF8DFF8C4A2AE
:10B5C0004348AF4B6E22DAF800100068FDF7E0FC4C
:10B5D000060008D00146ACA0F5F7FAFC1C98FEF76F
:10B5E0006FFC304690E70026DFF894B20FE0DAF8FF
:10B5F0000000825D0D2A1ED02D2A37D0A9A11DA8DA
:10B60000FAF75AF81DA96846F4F749FE761CDBF8EC
:10B6100000008642EBD3E068B0F5903F47D30A21A3
:10B62000B0FBF1F101FB08F14246A9423FD8A84224
:10B630001ED8642024E06846FAF772F851EC100B2B
:10B64000F4F7D3FE00EE100A0FB1B1EE400AA06885
:10B65000002700EB85006D1C80ED000A8DF800705E
:10B660002561E068761CA842D5D9CFE70127CDE750
:10B67000100000F1010101F0FF0801D009F10A00FA
:10B68000814689A0F5F7A4FC002609EBD97AB6EB30
:10B690006A0F01DA85A000E085A0F5F799FC761C19
:10B6A000B6B2322EF3D3494682A0F5F791FCE0689A
:10B6B000A84283D82269616801B921687FA0F5F7A3
:10B6C00087FC1C98FEF7FCFB01201DE7616C6C00F9
:10B6D0007C0200206461746100000000636F6E767C
:10B6E000315F626961730000636F6E76315F776509
:10B6F0006967687400000000636F6E76325F62698C
:10B7000061730000636F6E76325F77656967687496
:10B7100000000000636F6E76335F62696173000042
:10B72000636F6E76335F7765696768740000000049
:10B730006663315F62696173000000006663315FB8
:10B7400077656967687400006663325F6269617378
:10B75000000000006663325F776569676874000007
:10B76000303A2F25732E7478740000000D0ACAE455
:10B77000C8EBC1CBD2BBB8F6CEDED0A7B5C4C4A34C
:10B78000D0CDBBF244617461CAFDBEDDBCAFB5C4AF
:10B79000C3FBD7D60D0A0000D4A4C9E8C0EFC3BBD1
:10B7A000D3D0D5E2B8F6C4A3D0CDA3BA5B25735DE0
:10B7B0000D0A0000D0B4C8EBB5C4C4A3D0CDB2CE3E
:10B7C000CAFDC3FBD7D6CAC7A3BA25730D0A0000AA
:10B7D000D0B4C8EBB5C444617461CAFDBEDDBCAF72
:10B7E000CAC7A3BA25730D0A00000000D0B4C8EB85
:10B7F000C4A3D0CDB2CECAFDCAFDD7E9B5C4D7EE39
:10B80000B4F3B3A4B6C8CEAAA3BA25640D0A000047
:10B81000C4BFC7B0CAFDD7E9B4E6BBEEB5C4D4AA6D
:10B82000CBD8CAFDC1BFCEAAA3BA256400000000D0
:10B83000CEDEB7A8B4B4BDA8C4A3D0CDB2CECAFDE5
:10B840005B25735DB5C4CAFDD7E9B5BD534452410C
:10B850004DC0EF0D0A0000000D0AD5FDD4DAD0B4BA
:10B86000C8EBC4A3D0CDB2CECAFD27257327A3ACA5
:10B87000C7EBC9D4BAF32E2E2E2E2E2E0D0A0000A1
:10B880008802002084020020B6C1CEC4BCFEB3F6FC
:10B89000B4EDA3ACB4EDCEF3C2EBCEAAA3BA25644B
:10B8A0000D0A0000256300000D0A5B003D0000004A
:10B8B000200000005D202564252500000D0AC4A39A
:10B8C000D0CDB2CECAFD5B25735DD2D1D0B4C8EB6A
:10B8D000B5BDC4DAB4E6D6D02120C4A3D0CDB3A47C
:10B8E000B6C8CEAA2025640D0A00000070B54E4DE2
:10B8F00006460024A86828B14CA13046F4F7E2FCC3
:10B90000002865D0484D1435A86828B14AA13046B2
:10B91000F4F7D8FC00285BD0434D2835A86828B13F
:10B9200049A13046F4F7CEFC002851D03E4D3C35BD
:10B93000A86828B147A13046F4F7C4FC002847D0D6
:10B94000394D5035A86828B146A13046F4F7BAFC05
:10B9500000283DD0344D6435A86828B144A1304654
:10B96000F4F7B0FC002833D02F4D7835A86820B10B
:10B9700043A13046F4F7A6FC50B32B4D8C35A86894
:10B9800020B142A13046F4F79DFC08B3264DA03506
:10B99000A86820B140A13046F4F794FCC0B1224D14
:10B9A000B435A86820B13FA13046F4F78BFC78B1DC
:10B9B0001D4DC835A86820B13DA13046F4F782FC82
:10B9C00030B13DA13046F4F77DFC48B1002070BD98
:10B9D0000120A96800F0B4FAAC6001202C6170BDB0
:10B9E00012A0FFF783FF14A0FFF780FF16A0FFF758
:10B9F0007DFF18A0FFF77AFF1AA0FFF777FF1CA0C2
:10BA0000FFF774FF1EA0FFF771FF20A0FFF76EFF86
:10BA100021A0FFF76BFF23A0FFF768FF24A0FFF72B
:10BA200065FF022070BD000060C10220636F6E766A
:10BA3000315F626961730000636F6E76315F7765B5
:10BA40006967687400000000636F6E76325F626938
:10BA500061730000636F6E76325F77656967687443
:10BA600000000000636F6E76335F626961730000EF
:10BA7000636F6E76335F77656967687400000000F6
:10BA80006663315F62696173000000006663315F65
:10BA900077656967687400006663325F6269617325
:10BAA000000000006663325F7765696768740000B4
:10BAB0006461746100000000616C6C002DE9F14F5D
:10BAC0009A4CA06820B99AA10098F4F7FBFB20B12A
:10BAD000964D1435A86838B10BE08021012000F0A4
:10BAE0003BFAA060BDE8F88F94A10098F4F7EAFB58
:10BAF00020B18E4E2836B06838B10BE04FF490611B
:10BB0000012000F029FAA860ECE790A10098F4F772
:10BB1000D9FB20B1854F3C37B86838B10BE04FF402
:10BB20008071012000F018FAB060DBE78AA100986C
:10BB3000F4F7C8FB38B1DFF8F4A10AF1500ADAF8DB
:10BB4000080038B10BE04FF49031012000F004FA06
:10BB5000B860C7E784A10098F4F7B4FB20B173483C
:10BB60006430806840B10CE04FF40071012000F0B7
:10BB7000F3F9CAF80800B5E77EA10098F4F7A2FB34
:10BB800020B16A487830806840B10CE04FF49021D1
:10BB9000012000F0E1F9654964314EE079A1009897
:10BBA000F4F790FB38B1DFF8848108F18C08D8F8FD
:10BBB000080040B10CE04FF40071012000F0CCF916
:10BBC0005A49783139E072A10098F4F77BFB38B11B
:10BBD000DFF858B10BF1A00BDBF8080040B10CE026
:10BBE0004FF41001012000F0B7F9C8F8080079E718
:10BBF0006AA10098F4F766FB20B14C48B430806825
:10BC000038B10BE01C21012000F0A6F9CBF80800A8
:10BC100068E765A10098F4F755FB38B1DFF80C919F
:10BC200009F1C809D9F8080048B10DE04FF4606186
:10BC3000012000F091F93D49B431886052E75DA1DF
:10BC40000098F4F73FFB28B15CA10098F4F73AFBA9
:10BC500038B169E05A49012000F07EF9C9F80800BE
:10BC600040E7A06820B98021012000F075F9A060AC
:10BC7000A86828B94FF49061012000F06DF9A86020
:10BC8000B06828B94FF48071012000F065F9B06008
:10BC9000B86828B94FF49031012000F05DF9B86020
:10BCA000DAF80800544628B94FF40071012000F07A
:10BCB00053F9A0601D4C6434A06828B94FF490215A
:10BCC000012000F049F9A060184C7834A06828B928
:10BCD0004FF40071012000F03FF9A060D8F808008F
:10BCE000444628B94FF41001012000F035F9A06056
:10BCF000DBF808005C4620B91C21012000F02CF97B
:10BD0000A0600A4CB434A06828B94FF460610120E7
:10BD100000F022F9A060D9F808004C4620B9284963
:10BD2000012000F019F9A0600020DBE660C10220CC
:10BD3000636F6E76315F626961730000636F6E7668
:10BD4000315F77656967687400000000636F6E7625
:10BD5000325F626961730000636F6E76325F776590
:10BD60006967687400000000636F6E76335F626914
:10BD700061730000636F6E76335F7765696768741F
:10BD8000000000006663315F6269617300000000BB
:10BD90006663315F77656967687400006663325F68
:10BDA00062696173000000006663325F77656967EE
:10BDB000687400006461746100000000616C6C00D4
:10BDC000404B4C0070B50446006B0E460025B04257
:10BDD0000FD0204600F0E8FA05000AD16078012370
:10BDE000324604F13401FCF72BF808B16E1E012530
:10BDF0002663284670BD000070B5134A131893F8E7
:10BE0000203093B1114B53F820308B421AD90F4B8D
:10BE100002EB80020C3B53F820305069B1FBF3F188
:10BE200050F821400020034608E0116888470120AF
:10BE300070BD55690E18401C45F82630A042F8DB4D
:10BE4000002070BD022070BD2C000020ACD3000883
:10BE500030B504460748084D002150F82400820000
:10BE600005EB8400406900F087F80120291981F86A
:10BE7000200030BD94D300082C0000202DE9F041B3
:10BE80001E4E0546002470190F4690F8200010B988
:10BE90003168284688474FF0FF326FB3184B53F88C
:10BEA0002510B7FBF1F0B7FBF1FC01FB1C7101B1F0
:10BEB000401C13490C3951F82510491E1CD406EBBF
:10BEC0008506776957F821C0BCF1000F04D0002423
:10BED00084420FD1002206E0641CF9E774698F18D0
:10BEE000521C44F827008242F8D353F825004843F7
:10BEF000BDE8F081491EE5D51046F9E72C00002089
:10BF0000A0D3000810B50C4B0C4C002253F8203085
:10BF1000114604EB800005E0446954F8214004B167
:10BF2000521C491C8B42F7D84FF47A704243B2FB43
:10BF3000F3F080B210BD000094D300082C00002064
:10BF4000002906D0034A02EB80029268891AFFF7A3
:10BF500053BF70472C00002010B50446FFF78EFF3A
:10BF6000411C05D0034901EB84018968084410BDD8
:10BF7000002010BD2C00002001E000F8011B521E23
:10BF8000FBD270472DE9F04780460F4601F11A00B9
:10BF9000FEF72CFA20BB3878012600F03F00401E47
:10BFA00000EB8001DFF8489001EBC00400254FF65C
:10BFB000FF7A19F805003844FEF718FA36B1FF2C5D
:10BFC0000ED228F814000646641C01E0504507D143
:10BFD0006D1C0D2DEDD33878400607D5FF2C02D30C
:10BFE0000020BDE8F087002128F814100120F8E7B0
:10BFF000B8D300082DE9F047022617460D4604463F
:10C0000002296FD3A069A8426CD920784FF00109AA
:10C01000012806D0022838D0032846D0042861D150
:10C0200043E0616A05EB550801EB58212046FFF714
:10C03000C9FE060056D1C8F308002044343008F188
:10C040000108E90704D00178FAB262F31F1100E099
:10C050003946017084F80390616A204601EB58214B
:10C06000FFF7B0FE06003DD1C8F30800204434308D
:10C07000E90702D0C7F3071105E00178C7F30322EF
:10C0800001F0F001114301702AE0606A00EB152114
:10C090002046FFF797FE060024D1E8B204EB4000EB
:10C0A000B9B2343000F0F5F81AE0606A00EBD5114F
:10C0B0002046FFF787FE060014D140F2FF1000EA89
:10C0C0008500217805193435042905D02846FEF766
:10C0D00057F967F31B0007462846394600F0ACF8CD
:10C0E00084F803903046BDE8F08738B545680446CB
:10C0F000002D16DB60196D1C01733D2D0DDB6B46A9
:10C100002A4604F10C012068FDF716FB0098A842AE
:10C1100001D1002501E04FF0FF356560A068401CAB
:10C12000A06038BD006870472DE9F0478946046873
:10C13000924680460F464E46022936D3A069B84241
:10C1400033D9BAF1000F0ED02078042803D198F823
:10C150000700022807D04FF0FF3251462046FFF774
:10C1600049FF002822D139464046FDF77BFF0500F4
:10C1700033D0012D19D0681C1AD02078042806D09D
:10C18000002239462046FFF735FF00280ED16069AE
:10C19000411C05D0401C6061207940F001002071F5
:10C1A000701CA84206D12E4613E00220BDE8F0879D
:10C1B0000120FBE72078042809D1A6EB090200231F
:10C1C00049462046521CFAF791FA0028EED12E4635
:10C1D000B146A0692F46B842C5D82078042815D1A9
:10C1E000BAF1000F04D098F80700032802D00DE040
:10C1F000002109E0D8F80800504507D8D8F81810F1
:10C200000144514502D3022188F807100020CDE7F0
:10C2100070B50C460646154691B204F11A0000F0BE
:10C2200038F83078032806D1290C04F11400BDE851
:10C23000704000F02EB870BD0170090A4170090A03
:10C240008170090AC170704710B5110A027041EA85
:10C25000036141701A0A090A41EA02618170120AF7
:10C26000090A41EA0261C170120A090A41EA02613F
:10C270000171120A090A41EA02614171120A090AAE
:10C2800041EA0261120A8171090A41EA0261C1713F
:10C2900010BD0170090A417070472DE9F041044654
:10C2A0000068C568284601F034F80146A81CFFF76D
:10C2B000F0FF6F7820467F1CE16BFBF714FD06460C
:10C2C0004FF001080FE020222946606BFEF7EAF9E3
:10C2D00021687F1E81F803800DD000212046203583
:10C2E000FBF7BEFA06463EB9216B2068FFF76AFDF0
:10C2F0000600E8D000E026B1012E02D00220BDE801
:10C30000F0813046FBE7014600200B22430803EB97
:10C31000C01011F8013B521E1844C0B2F6D170474C
:10C3200070B5044600F040F8050036D120780328A7
:10C330002CD12079012829D1420204F134000021B6
:10C340000646FEF7B8F94AF6552104F23220FFF707
:10C35000A0FF13493046FFF76FFF124904F506703E
:10C36000FFF76AFF04F507706169FFF765FF04F5E1
:10C3700008702169FFF760FF226A0123521C2263C3
:10C3800060783146FBF791FD002020710022607833
:10C390001146FBF707FD00B10125284670BD0000DE
:10C3A00052526141727241612DE9F0410446C078F8
:10C3B0000027F8B1266B04F134016078012332467E
:10C3C0008846FBF772FD08B1012713E00020E070FA
:10C3D000606AE169301A88420CD2A57808E0E06909
:10C3E00001230644607832464146FBF75EFD6D1E30
:10C3F000022DF4D23846BDE8F08100000749064A14
:10C40000C1E9002000208860C860086188610C20B4
:10C4100048610846F7F730B8001001406803002073
:10C4200070B594B0064613AB11AA694600F0D8F96E
:10C43000002824D18DF840001D4C042514E020680C
:10C4400005EBC10113AB405812AA08A900F0C8F9C6
:10C45000002814D1694608A800F0E2FB88B19DF8D5
:10C460004000401C8DF84000207D9DF8401088421F
:10C47000E5D8207D9DF8401088420ED1042014B0EC
:10C4800070BD9DF848009DF84410884201D90220F3
:10C49000F5E79DF84000A075EBE710A9304600F0E5
:10C4A00053FA0028EBD19DF8400060750020E6E7C4
:10C4B000840100202DE9F0417E4E9AB0B57D307D9B
:10C4C000A8427CD90421306801EBC50119AB405862
:10C4D00018AA10A900F084F910A977A0F9F7DCF8E0
:10C4E00000240DF1180832E0308B0121A1400842F0
:10C4F00017D0222172A0F9F7CFF8204600F08CFA6D
:10C50000811970A02431F9F7C7F822216CA0F9F73E
:10C51000C3F8204600F080FA3044243048F8240064
:10C520000BE0204600F078FA3044416A48F82410C5
:10C53000F07D00B364A0F9F7AFF89DF86000401EED
:10C54000844202D062A0F9F7A7F8641CE4B29DF817
:10C5500060008442C8D35FA0F9F79EF800F0A2FA09
:10C56000707D0B2814D2DFE800F0080D3138404808
:10C57000525E6B78890058A0DDE7306850F83500CE
:10C58000804704E0306850F8351006988847074621
:10C5900000F054FA9DF8640001286ED04FA0F9F71E
:10C5A0007BF896F8EC0000280DD0D6F8F0000A21B0
:10C5B000B0FBF1F201FB1202B0FBF1F100E002E08E
:10C5C00047A0F9F769F81AB0BDE8F081306850F873
:10C5D0003520DDE906019047D9E7306806AC50F810
:10C5E000353094E807009847D1E7306806AF50F837
:10C5F000354097E80F00A047C9E70A9800903068D7
:10C6000006AF50F8354097E80F00A047BFE7DDE9D7
:10C610000A01CDE90001306806AF50F8354097E8CF
:10C620000F00A047B3E70AAB06AF93E807008DE819
:10C630000700306850F8354097E80F00A047A6E79C
:10C640000AAC06AF94E80F008DE80F00306850F890
:10C65000354097E80F00A04799E70BAC06AF94E888
:10C660000F0001AC84E80F000A980090306850F881
:10C67000354097E80F00A04789E711E00CAC06AF02
:10C6800094E80F0002AC84E80F00DDE90A01CDE96F
:10C690000001306850F8354097E80F00A04776E772
:10C6A000F07D394618B116A0F8F7F6FF79E717A024
:10C6B000FAE70000840100200D0A2573280000001D
:10C6C0002563000025730000305825580000000045
:10C6D0002C00000029000000256C64003B0D0A00BE
:10C6E00046756E6374696F6E2052756E2054696D65
:10C6F000653A25642E2531646D730D0A0000000033
:10C700003D305825583B0D0A000000003D256C7552
:10C710003B0D0A00F0B500252E462F462C46037827
:10C720002C2B03D0292B04D01BB103E014B9012614
:10C7300000E05CB317B1222B26D026E0A3F1300C29
:10C74000BCF1090F15D9A3F1610CBCF1050F10D98B
:10C75000A3F1410CBCF1050F0BD9582B09D0782B54
:10C7600007D0222B0CD0202B1ED02C2B1CD0FF2727
:10C770000CE05EB9612B00D3203B01F8013B13E0D4
:10C7800026B901273C460FE0002426B1002008709E
:10C7900017702846F0BD3CB15C2B02D16D1CEDB288
:10C7A000401C037801F8013B6D1CEDB2401CB6E75C
:10C7B00030B5002515700AE001F8014B1478401CD3
:10C7C000641CE4B214709C4201D3012030BD047893
:10C7D000202C01D0002CEFD10D70002030BD0000C6
:10C7E0002DE9FF4F002482B089469846A24627468D
:10C7F000012526462246EB46029915E0202810D056
:10C8000002F07F03052B0CD202B9802202F07F03D5
:10C81000042B01D12A280AD1521C0BF80300D2B2F2
:10C8200001E0852A04D0491C08780028E6D16AB1C5
:10C8300002F07F0200200BF8020041A1584600F0F0
:10C84000EFF938B1012188F8001000224FF00008FC
:10C85000029B15E0002088F80000F6E708F10100CF
:10C8600000F0FF0813F8010F202801D02A2807D173
:10C87000184600F07DF9282802D02A2800D0C246A8
:10C880001878282801D00028E8D10299BAF1000FC1
:10C8900001D05144491C4FF000084346087888B144
:10C8A000282804D0292806D0222810D011E083B9E6
:10C8B000641CE4B20DE063B924B1641E14F0FF04FB
:10C8C00002D00DE04FF00108012F27D02FE04BB12F
:10C8D00000234CB12C280CD0202816D0282814D0A6
:10C8E0005AB110E00123F4E7202815D009F8010B14
:10C8F00012E00125521CD2B207E0052E03D20BF83C
:10C900000600761CF6B26D1CEDB2012C04D1022D8E
:10C9100002D103257F1CFFB2491CBFE700200BF8A2
:10C92000060007A1684600F07BF900B900270498CB
:10C930000770002089F8000006B04046BDE8F08F7F
:10C94000766F6964000000002DE9F04300248946F9
:10C95000304DB5B0214622466B18491CC9B29A76B3
:10C960000A29F9D302E010F8011F99B101782829AA
:10C97000F9D1461C4FF0010833AA69463046FFF74B
:10C98000C9FE06449DF8CC0040B1012824D0FF2800
:10C9900036D10BE0012035B0BDE8F0839DF80000F2
:10C9A00070B334A9684600F0EBF808B10220F2E752
:10C9B000204600F031F8284434994162298B08FA66
:10C9C00004F081432983042029198876641CE4B289
:10C9D0000A2C15D90320DEE7684600F036F9471C1B
:10C9E000204600F019F841196846243100F024F976
:10C9F000298B08FA04F00143281929838776E5E793
:10CA00003078292801D00028B6D189F800400020CC
:10CA1000C1E7000084010020024610B50020014655
:10CA2000054B05E05C18491CA47EC9B22044C0B285
:10CA30009142F7D310BD000084010020094800682E
:10CA40000169C943CA070849D1F8F02004D14FF65B
:10CA5000FF731A44C1F8F020406A1044C1F8F00096
:10CA600070470000A0BF02208401002000EBC0013D
:10CA700001EB00104FF0FF3101EB800010B581B2E7
:10CA80004FF47A70F8F784FA01490120C87510BD97
:10CA9000840100200346012000E05843491EC9B22A
:10CAA000FBD2704707486FF001010268116102680C
:10CAB000090CD162C1600068002141620248C0F8DF
:10CAC000F0107047A0BF0220840100202DE9F04142
:10CAD000164E3088010426D51549C0B2154F0025E1
:10CAE0000D54B9681248884704000FD0104800F070
:10CAF000B5F8012801D0040014D0012C09D0022C73
:10CB000009D0032C09D0042C0CD108E0F868804728
:10CB100008E009A004E00BA002E00DA000E00FA0D7
:10CB2000F8F7BAFD3580BDE8F08100001C00002058
:10CB3000A002002084010020BAAFCAFDB4EDCEF3FC
:10CB4000210D0A00B2CECAFDB4EDCEF3210D0A00CC
:10CB5000B2CECAFDCCABB6E0210D0A00CEB4D5D220
:10CB6000B5BDC6A5C5E4B5C4BAAFCAFD210D0A005E
:10CB700010F8011F202901D10028F9D1C8B270474F
:10CB80002DE9F0410024884605460A260C6001780C
:10CB9000A1F13002092A0DD9113A052A0AD95829DA
:10CBA00005D011F0FF0F0CD00120BDE8F081012C61
:10CBB00002D0F9E7412900D31026641CE4B2401CDE
:10CBC000E5E7102E01D084B112E0032C01D202203F
:10CBD000EBE72878302802D16878582801D0032064
:10CBE000E3E7A41EE4B2AD1C01E00420DDE70CB1D4
:10CBF000641EE4B22F783846303F092F01D9A0F1E6
:10CC0000370721463046FFF745FFD8F8001007FBED
:10CC10000011C8F8001015F8010F0028E7D1C4E78B
:10CC200002780B789A4201D00120704712B1401C63
:10CC3000491CF5E70020704702780A700278002A44
:10CC400002D0401C491CF7E77047002102781AB156
:10CC5000491CC9B2401CF9E708467047F0B58DB0D1
:10CC600004461E2308AA6946FFF7A2FD0990002882
:10CC700072D19DF82000271800253E4C8DF82050D9
:10CC80009DF8200054F820106846FFF7C9FF38B11E
:10CC90009DF82000401CC0B28DF820000728EFD37B
:10CCA0009DF820000426344C072855D2DFE800F018
:10CCB0000404395A605F5E0030A0F8F7EDFC30A044
:10CCC000F8F7EAFC3EA0F8F7E7FC4DA0F8F7E4FC23
:10CCD0005BA0F8F7E1FC6AA0F8F7DEFC78A0F8F7B3
:10CCE000DBFC86A0F8F7D8FC8BA0F8F7D5FC93A066
:10CCF000F8F7D2FC97A0F8F7CFFC9CA0F8F7CCFC93
:10CD0000A1A0F8F7C9FCA7A0F8F7C6FCB3A0F8F7F4
:10CD1000C3FCC0A0F8F7C0FCCBA0F8F7BDFCD7A0BF
:10CD20001BE016A0F8F7B8FCE4A0F8F7B5FC8DF806
:10CD300020500BE0216806EBC0000958EFA0F8F77F
:10CD4000ABFC9DF82000401C8DF82000217D9DF853
:10CD500020008142EED856E257E2F8F79DFC002011
:10CD60000DB0F0BD05A0F8F797FCCBE12CE20CE28A
:10CD7000EBE1000050000020840100200D0A0000BB
:10CD80002D2D2D2D2D2D2D2D2D2D2D2D2D2D2D2DD3
:10CD90002D2D2D2D2D2D2D2D55534D4152542056D9
:10CDA000332E332D2D2D2D2D2D2D2D2D2D2D2D2DA6
:10CDB0002D2D2D2D2D2D2D2D2D2D2D200D0A00004D
:10CDC0002020202055534D415254CAC7D3C9414C4D
:10CDD00049454E54454BBFAAB7A2B5C4D2BBB8F61D
:10CDE000C1E9C7C9B5C4B4AEBFDAB5F7CAD4BBA5EB
:10CDF000BDBBD7E9BCFE2CCDA8B9FD200D0A0000B3
:10CE0000CBFC2CC4E3BFC9D2D4CDA8B9FDB4AEBF0E
:10CE1000DAD6FACAD6B5F7D3C3B3CCD0F2C0EFC3D3
:10CE2000E6B5C4C8CEBACEBAAFCAFD2CB2A2D6B44B
:10CE3000D0D02ED2F2B4CB2CC4E3BFC90D0A00006F
:10CE4000D2D4CBE6D2E2B8FCB8C4BAAFCAFDB5C4FE
:10CE5000CAE4C8EBB2CECAFD28D6A7B3D6CAFDD75E
:10CE6000D62831302F3136BDF8D6C62CD6A7B3D64A
:10CE7000B8BACAFD29A1A2D7D6B7FBB4AE0D0A0035
:10CE8000A1A2BAAFCAFDC8EBBFDAB5D8D6B7B5C84C
:10CE9000D7F7CEAAB2CECAFD292CB5A5B8F6BAAF3F
:10CEA000CAFDD7EEB6E0D6A7B3D63130B8F6CAE49D
:10CEB000C8EBB2CECAFD2CB2A2D6A7B3D60D0A00DB
:10CEC000BAAFCAFDB7B5BBD8D6B5CFD4CABE2ED679
:10CED000A7B3D6B2CECAFDCFD4CABEBDF8D6C6C996
:10CEE000E8D6C3B9A6C4DC2CD6A7B3D6BDF8D6C63F
:10CEF000D7AABBBBB9A6C4DC2E0D0A00BCBCCAF5C0
:10CF0000D6A7B3D63A7777772E6F70656E6564765D
:10CF10002E636F6D0D0A000055534D415254D3D00E
:10CF200037B8F6CFB5CDB3C3FCC1EE28B1D8D0EB3E
:10CF3000D0A1D0B4293A0D0A000000003F3A2020C9
:10CF400020202020BBF1C8A1B0EFD6FAD0C5CFA2D7
:10CF50000D0A000068656C703A202020BBF1C8A162
:10CF6000B0EFD6FAD0C5CFA20D0A00006C69737479
:10CF70003A202020BFC9D3C3B5C4BAAFCAFDC1D0BF
:10CF8000B1ED0D0A0A00000069643A20202020203B
:10CF9000BFC9D3C3BAAFCAFDB5C44944C1D0B1ED0E
:10CFA0000D0A0A006865783A20202020B2CECAFD1A
:10CFB0003136BDF8D6C6CFD4CABE2CBAF3B8FABF44
:10CFC000D5B8F12BCAFDD7D6BCB4D6B4D0D0BDF8F5
:10CFD000D6C6D7AABBBB0D0A0A0000006465633A37
:10CFE00020202020B2CECAFD3130BDF8D6C6CFD425
:10CFF000CABE2CBAF3B8FABFD5B8F12BCAFDD7D642
:10D00000BCB4D6B4D0D0BDF8D6C6D7AABBBB0D0A27
:10D010000A00000072756E74696D653A312CBFAA02
:10D02000C6F4BAAFCAFDD4CBD0D0BCC6CAB13B306F
:10D030002CB9D8B1D5BAAFCAFDD4CBD0D0BCC6CAF2
:10D04000B13B0D0A0A000000C7EBB0B4D5D5B3CC94
:10D05000D0F2B1E0D0B4B8F1CABDCAE4C8EBBAAFFF
:10D06000CAFDC3FBBCB0B2CECAFDB2A2D2D4BBD8FB
:10D07000B3B5BCFCBDE1CAF82E0D0A002D2D2D2D37
:10D080002D2D2D2D2D2D2D2D2D2D2D2D2D2D2D2DD0
:10D090002D2D2D2D2D2D414C49454E54454B2D2DDB
:10D0A0002D2D2D2D2D2D2D2D2D2D2D2D2D2D2D2DB0
:10D0B0002D2D2D2D2D2D2D200D0A00002D2D2D2D4A
:10D0C0002D2D2D2D2D2D2D2D2D2D2D2D2D2D2D2D90
:10D0D0002D2D2D2D2DBAAFCAFDC7E5B5A52D2D2DB2
:10D0E0002D2D2D2D2D2D2D2D2D2D2D2D2D2D2D2D70
:10D0F0002D2D2D2D2D2D2D2D200D0A0025730D0AE2
:10D100000000000042A0F8F7C7FA8DF8205016E0A2
:10D11000216806EBC0000BAB08580AAA6946FFF766
:10D120005FFB9DF82010206850F83120694648A028
:10D13000F8F7B2FA9DF82000401C8DF82000217D00
:10D140009DF820008142E3D85DE0AFF2D030F8F7DF
:10D15000A3FA08AA69463846FFF7DCFA9DF82000D2
:10D16000002843D109A96846FFF70AFD8DF8200081
:10D1700010B104283AD102E03AA009991CE03CA081
:10D18000F8F78AFA0120E0753DE038A0F8F784FA54
:10D1900008AA69463846FFF7BDFA9DF8200028BB6B
:10D1A00009A96846FFF7ECFC8DF8200010B10428AF
:10D1B0001CD104E033A00999F8F76EFA23E034A0FB
:10D1C000F8F76AFAE5751EE028A0F8F765FA08AAEC
:10D1D00069463846FFF79EFA9DF8200030B909A944
:10D1E0006846FFF7CDFC8DF8200008B10220B7E5B6
:10D1F000099810F0FF0084F8EC0001D029A000E0AD
:10D200002FA0F8F749FA19A0A7E50120A8E500002A
:10D210002D2D2D2D2D2D2D2D2D2D2D2D2D2D2D2D3E
:10D220002D2D2D2D2D2D2D2D2DBAAFCAFD2049448C
:10D23000202D2D2D2D2D2D2D2D2D2D2D2D2D2D2D2B
:10D240002D2D2D2D2D2D2D2D2D2D2D2D200D0A008B
:10D2500025732069642069733A0D0A3058253038E7
:10D26000580D0A004845583A305825580D0A000014
:10D270003136BDF8D6C6B2CECAFDCFD4CABE210D56
:10D280000A0000004445433A256C750D0A00000071
:10D290003130BDF8D6C6B2CECAFDCFD4CABE210D3C
:10D2A0000A00000052756E2054696D652043616C60
:10D2B00063756C6174696F6E204F4E0D0A0000003B
:10D2C00052756E2054696D652043616C63756C61A5
:10D2D00074696F6E204F46460D0A000070B50D460A
:10D2E00004000CD0206850B1017841B1C188A288F7
:10D2F000914204D14078FAF7D6FDC00703D0002050
:10D300002860092070BD20682860002070BD016081
:10D31000704730B5034640784FF400454401002083
:10D32000014620340AE002290BD0C20700D02A4669
:10D3300002EB50005A5C104480B2491CA142F2D367
:10D3400030BD0321F9E770B5054600244FF40046CF
:10D3500011E0FCF709FBE10700D0314601EB540175
:10D36000C2B2114489B2CA0700D0324602EB510161
:10D3700001EB102084B235F8020B0028E9D12046D9
:10D3800070BD00000000010203040102030406074F
:10D3900008090000000A0000000F0700C003000099
:10D3A000400000004000000040000000008002003B
:10D3B00000C0C30100F0000001030507090E1012B0
:10D3C0001416181C1E222A2B2C2E3A3B3C3D3E3FA5
:10D3D0005B5D7C7F000000040002000180004000D3
:10D3E000200010000800040002000000008000403F
:10D3F0000020001000080040002000100008000479
:10D400000002A400E8A1A700ECA1A800A7A1B00019
:10D41000E3A1B100C0A1B700A4A1D700C1A1E00061
:10D42000A4A8E100A2A8E800A8A8E900A6A8EA002C
:10D43000BAA8EC00ACA8ED00AAA8F200B0A8F300CE
:10D44000AEA8F700C2A1F900B4A8FA00B2A8FC0087
:10D45000B9A80101A1A81301A5A81B01A7A82B0128
:10D46000A9A84401BDA84801BEA84D01ADA86B0103
:10D47000B1A8CE01A3A8D001ABA8D201AFA8D40116
:10D48000B3A8D601B5A8D801B6A8DA01B7A8DC01BF
:10D49000B8A85102BBA86102C0A8C702A6A1C902D0
:10D4A000A5A1CA0240A8CB0241A8D90242A8910373
:10D4B000A1A69203A2A69303A3A69403A4A69503F0
:10D4C000A5A69603A6A69703A7A69803A8A69903C0
:10D4D000A9A69A03AAA69B03ABA69C03ACA69D0390
:10D4E000ADA69E03AEA69F03AFA6A003B0A6A10360
:10D4F000B1A6A303B2A6A403B3A6A503B4A6A6032C
:10D50000B5A6A703B6A6A803B7A6A903B8A6B103F4
:10D51000C1A6B203C2A6B303C3A6B403C4A6B5038F
:10D52000C5A6B603C6A6B703C7A6B803C8A6B9035F
:10D53000C9A6BA03CAA6BB03CBA6BC03CCA6BD032F
:10D54000CDA6BE03CEA6BF03CFA6C003D0A6C103FF
:10D55000D1A6C303D2A6C403D3A6C503D4A6C603CB
:10D56000D5A6C703D6A6C803D7A6C903D8A6010463
:10D57000A7A71004A1A71104A2A71204A3A713042C
:10D58000A4A71404A5A71504A6A71604A8A7170402
:10D59000A9A71804AAA71904ABA71A04ACA71B04CF
:10D5A000ADA71C04AEA71D04AFA71E04B0A71F049F
:10D5B000B1A72004B2A72104B3A72204B4A723046F
:10D5C000B5A72404B6A72504B7A72604B8A727043F
:10D5D000B9A72804BAA72904BBA72A04BCA72B040F
:10D5E000BDA72C04BEA72D04BFA72E04C0A72F04DF
:10D5F000C1A73004D1A73104D2A73204D3A7330482
:10D60000D4A73404D5A73504D6A73604D8A7370441
:10D61000D9A73804DAA73904DBA73A04DCA73B040E
:10D62000DDA73C04DEA73D04DFA73E04E0A73F04DE
:10D63000E1A74004E2A74104E3A74204E4A74304AE
:10D64000E5A74404E6A74504E7A74604E8A747047E
:10D65000E9A74804EAA74904EBA74A04ECA74B044E
:10D66000EDA74C04EEA74D04EFA74E04F0A74F041E
:10D67000F1A75104D7A710205CA9132043A81420B8
:10D68000AAA1152044A81620ACA11820AEA11920EB
:10D69000AFA11C20B0A11D20B1A1252045A82620A6
:10D6A000ADA13020EBA13220E4A13320E5A135204B
:10D6B00046A83B20F9A1AC2080000321E6A105216A
:10D6C00047A8092148A81621EDA1212159A96021C7
:10D6D000F1A26121F2A26221F3A26321F4A26421EA
:10D6E000F5A26521F6A26621F7A26721F8A26821BA
:10D6F000F9A26921FAA26A21FBA26B21FCA2702186
:10D70000A1A27121A2A27221A3A27321A4A27421B9
:10D71000A5A27521A6A27621A7A27721A8A2782189
:10D72000A9A27921AAA29021FBA19121FCA1922179
:10D73000FAA19321FDA1962149A897214AA89821F1
:10D740004BA899214CA80822CAA10F22C7A11122D7
:10D75000C6A115224DA81A22CCA11D22D8A11E2295
:10D76000DEA11F224EA82022CFA123224FA82522CE
:10D77000CEA12722C4A12822C5A12922C9A12A22DB
:10D78000C8A12B22D2A12E22D3A13422E0A135227E
:10D79000DFA13622C3A13722CBA13D22D7A1482247
:10D7A000D6A14C22D5A1522250A86022D9A1612233
:10D7B000D4A16422DCA16522DDA1662251A86722E2
:10D7C00052A86E22DAA16F22DBA1952292A899229B
:10D7D000D1A1A522CDA1BF2253A81223D0A160249C
:10D7E000D9A26124DAA26224DBA26324DCA264242D
:10D7F000DDA26524DEA26624DFA26724E0A26824FD
:10D80000E1A26924E2A27424C5A27524C6A27624EA
:10D81000C7A27724C8A27824C9A27924CAA27A24EC
:10D82000CBA27B24CCA27C24CDA27D24CEA27E24BC
:10D83000CFA27F24D0A28024D1A28124D2A282248C
:10D84000D3A28324D4A28424D5A28524D6A286245C
:10D85000D7A28724D8A28824B1A28924B2A28A247C
:10D86000B3A28B24B4A28C24B5A28D24B6A28E249C
:10D87000B7A28F24B8A29024B9A29124BAA292246C
:10D88000BBA29324BCA29424BDA29524BEA296243C
:10D89000BFA29724C0A29824C1A29924C2A29A240C
:10D8A000C3A29B24C4A20025A4A90125A5A90225E1
:10D8B000A6A90325A7A90425A8A90525A9A9062580
:10D8C000AAA90725ABA90825ACA90925ADA90A2550
:10D8D000AEA90B25AFA90C25B0A90D25B1A90E2520
:10D8E000B2A90F25B3A91025B4A91125B5A91225F0
:10D8F000B6A91325B7A91425B8A91525B9A91625C0
:10D90000BAA91725BBA91825BCA91925BDA91A258F
:10D91000BEA91B25BFA91C25C0A91D25C1A91E255F
:10D92000C2A91F25C3A92025C4A92125C5A922252F
:10D93000C6A92325C7A92425C8A92525C9A92625FF
:10D94000CAA92725CBA92825CCA92925CDA92A25CF
:10D95000CEA92B25CFA92C25D0A92D25D1A92E259F
:10D96000D2A92F25D3A93025D4A93125D5A932256F
:10D97000D6A93325D7A93425D8A93525D9A936253F
:10D98000DAA93725DBA93825DCA93925DDA93A250F
:10D99000DEA93B25DFA93C25E0A93D25E1A93E25DF
:10D9A000E2A93F25E3A94025E4A94125E5A94225AF
:10D9B000E6A94325E7A94425E8A94525E9A946257F
:10D9C000EAA94725EBA94825ECA94925EDA94A254F
:10D9D000EEA94B25EFA9502554A8512555A852254D
:10D9E00056A8532557A8542558A8552559A8562553
:10D9F0005AA857255BA858255CA859255DA85A2523
:10DA00005EA85B255FA85C2560A85D2561A85E25F2
:10DA100062A85F2563A8602564A8612565A86225C2
:10DA200066A8632567A8642568A8652569A8662592
:10DA30006AA867256BA868256CA869256DA86A2562
:10DA40006EA86B256FA86C2570A86D2571A86E2532
:10DA500072A86F2573A8702574A8712575A8722502
:10DA600076A8732577A8812578A8822579A88325AB
:10DA70007AA884257BA885257CA886257DA887256E
:10DA80007EA8882580A8892581A88A2582A88B253B
:10DA900083A88C2584A88D2585A88E2586A88F250A
:10DAA00087A8932588A8942589A895258AA8A025C4
:10DAB000F6A1A125F5A1B225F8A1B325F7A1BC25B2
:10DAC0008BA8BD258CA8C625F4A1C725F3A1CB251D
:10DAD000F0A1CE25F2A1CF25F1A1E2258DA8E32565
:10DAE0008EA8E4258FA8E52590A80526EFA1062697
:10DAF000EEA1092691A84026E2A14226E1A100302C
:10DB0000A1A10130A2A10230A3A10330A8A1053038
:10DB1000A9A1063065A9073096A90830B4A109303B
:10DB2000B5A10A30B6A10B30B7A10C30B8A10D30A9
:10DB3000B9A10E30BAA10F30BBA11030BEA1113077
:10DB4000BFA1123093A81330FEA11430B2A115303A
:10DB5000B3A11630BCA11730BDA11D3094A81E3052
:10DB600095A8213040A9223041A9233042A9243070
:10DB700043A9253044A9263045A9273046A9283095
:10DB800047A9293048A94130A1A44230A2A443307A
:10DB9000A3A44430A4A44530A5A44630A6A447308D
:10DBA000A7A44830A8A44930A9A44A30AAA44B305D
:10DBB000ABA44C30ACA44D30ADA44E30AEA44F302D
:10DBC000AFA45030B0A45130B1A45230B2A45330FD
:10DBD000B3A45430B4A45530B5A45630B6A45730CD
:10DBE000B7A45830B8A45930B9A45A30BAA45B309D
:10DBF000BBA45C30BCA45D30BDA45E30BEA45F306D
:10DC0000BFA46030C0A46130C1A46230C2A463303C
:10DC1000C3A46430C4A46530C5A46630C6A467300C
:10DC2000C7A46830C8A46930C9A46A30CAA46B30DC
:10DC3000CBA46C30CCA46D30CDA46E30CEA46F30AC
:10DC4000CFA47030D0A47130D1A47230D2A473307C
:10DC5000D3A47430D4A47530D5A47630D6A477304C
:10DC6000D7A47830D8A47930D9A47A30DAA47B301C
:10DC7000DBA47C30DCA47D30DDA47E30DEA47F30EC
:10DC8000DFA48030E0A48130E1A48230E2A48330BC
:10DC9000E3A48430E4A48530E5A48630E6A487308C
:10DCA000E7A48830E8A48930E9A48A30EAA48B305C
:10DCB000EBA48C30ECA48D30EDA48E30EEA48F302C
:10DCC000EFA49030F0A49130F1A49230F2A49330FC
:10DCD000F3A49B3061A99C3062A99D3066A99E3057
:10DCE00067A9A130A1A5A230A2A5A330A3A5A43005
:10DCF000A4A5A530A5A5A630A6A5A730A7A5A830A0
:10DD0000A8A5A930A9A5AA30AAA5AB30ABA5AC306F
:10DD1000ACA5AD30ADA5AE30AEA5AF30AFA5B0303F
:10DD2000B0A5B130B1A5B230B2A5B330B3A5B4300F
:10DD3000B4A5B530B5A5B630B6A5B730B7A5B830DF
:10DD4000B8A5B930B9A5BA30BAA5BB30BBA5BC30AF
:10DD5000BCA5BD30BDA5BE30BEA5BF30BFA5C0307F
:10DD6000C0A5C130C1A5C230C2A5C330C3A5C4304F
:10DD7000C4A5C530C5A5C630C6A5C730C7A5C8301F
:10DD8000C8A5C930C9A5CA30CAA5CB30CBA5CC30EF
:10DD9000CCA5CD30CDA5CE30CEA5CF30CFA5D030BF
:10DDA000D0A5D130D1A5D230D2A5D330D3A5D4308F
:10DDB000D4A5D530D5A5D630D6A5D730D7A5D8305F
:10DDC000D8A5D930D9A5DA30DAA5DB30DBA5DC302F
:10DDD000DCA5DD30DDA5DE30DEA5DF30DFA5E030FF
:10DDE000E0A5E130E1A5E230E2A5E330E3A5E430CF
:10DDF000E4A5E530E5A5E630E6A5E730E7A5E8309F
:10DE0000E8A5E930E9A5EA30EAA5EB30EBA5EC306E
:10DE1000ECA5ED30EDA5EE30EEA5EF30EFA5F0303E
:10DE2000F0A5F130F1A5F230F2A5F330F3A5F4300E
:10DE3000F4A5F530F5A5F630F6A5FC3060A9FD3067
:10DE400063A9FE3064A90531C5A80631C6A807310B
:10DE5000C7A80831C8A80931C9A80A31CAA80B3116
:10DE6000CBA80C31CCA80D31CDA80E31CEA80F31E6
:10DE7000CFA81031D0A81131D1A81231D2A81331B6
:10DE8000D3A81431D4A81531D5A81631D6A8173186
:10DE9000D7A81831D8A81931D9A81A31DAA81B3156
:10DEA000DBA81C31DCA81D31DDA81E31DEA81F3126
:10DEB000DFA82031E0A82131E1A82231E2A82331F6
:10DEC000E3A82431E4A82531E5A82631E6A82731C6
:10DED000E7A82831E8A82931E9A82032E5A22132B3
:10DEE000E6A22232E7A22332E8A22432E9A22532B6
:10DEF000EAA22632EBA22732ECA22832EDA2293286
:10DF0000EEA231325AA9A33249A98E334AA98F33DE
:10DF10004BA99C334CA99D334DA99E334EA9A133E7
:10DF20004FA9C43350A9CE3351A9D13352A9D2330A
:10DF300053A9D53354A9004EBBD2014EA1B6024E0F
:10DF40004081034EDFC6044E4181054E4281064E9C
:10DF50004381074EF2CD084EC9D5094EFDC80A4E81
:10DF6000CFC90B4EC2CF0C4EA2D80D4EBBB20E4E37
:10DF7000EBD30F4E4481104EA4D8114EF3B3124E82
:10DF80004581134EA8D7144ED2C7154EA7D8164EAA
:10DF9000C0CA174E4681184EF0C7194EFBB11A4E33
:10DFA000B5D21B4ED4B41C4EABB61D4EBFCB1E4ECD
:10DFB000A9D81F4E4781204E4881214E4981224ECB
:10DFC000AAB6234E4A81244EBDC1254ECFD1264E3E
:10DFD0004B81274EA5C9284EADD8294E4C812A4EDB
:10DFE000F6B82B4EBED12C4EDCE32D4ED0D62E4EA5
:10DFF0004D812F4E4E81304EE1B7314E4F81324E22
:10E00000AEB4334E5081344ED9C1354E5181364E67
:10E01000BCD8374E5281384EE8CD394EA4B53A4E71
:10E02000AACE3B4EF7D63C4E53813D4EF6C03E4EF7
:10E03000D9BE3F4EAFD8404E5481414E5581424EDD
:10E040005681434ECBC4444E5781454EC3BE464EC7
:10E050005881474EB1D8484EB4C3494EE5D24A4ED6
:10E0600059814B4EAED64C4EDACE4D4EA7D54E4EC4
:10E07000F5BA4F4EA6B7504ED6C0514E5A81524EA9
:10E08000B9C6534ED2C5544EC7C7554E5B81564E86
:10E09000D4B9574E5C81584ECBB3594ED2D25A4E5A
:10E0A0005D815B4E5E815C4EBFD85D4EC5BE5E4EEF
:10E0B000F2C65F4EB2D2604EB0CF614EE7CF624E35
:10E0C0005F81634E6081644E6181654E6281664E00
:10E0D000E9CA674E6381684E6481694EC0D86A4E52
:10E0E00065816B4E66816C4E67816D4E68816E4EA8
:10E0F00069816F4E6A81704EF2C2714ED2C2724E09
:10E100006B81734EE9C8744E6C81754E6D81764E8D
:10E110006E81774E6F81784E7081794E71817A4E23
:10E1200072817B4E73817C4E74817D4E75817E4EF3
:10E13000ACC77F4E7681804E7781814E7881824E4A
:10E140007981834E7A81844E7B81854E7C81864E97
:10E15000CBC1874E7D81884EE8D3894EF9D58A4E52
:10E160007E818B4EC2CA8C4EFEB68D4EA1D88E4E8D
:10E17000DAD38F4EF7BF904E8081914EC6D4924E27
:10E18000A5BB934EC1D8944EE5CE954EAEBE964EED
:10E190008181974E8281984EA8D8994E83819A4E5C
:10E1A000C7D19B4EA9D09C4E84819D4E85819E4EA9
:10E1B00086819F4EBDD8A04EEFD9A14EF6CDA24E7E
:10E1C000BABFA34E8781A44EBBBDA54EA5BAA64E2D
:10E1D000E0D2A74EFAB2A84EE0BAA94EB6C4AA4EF3
:10E1E0008881AB4EEDCFAC4EA9BEAD4EA4CDAE4EA8
:10E1F000C1C1AF4E8981B04E8A81B14E8B81B24E82
:10E20000D7C7B34EF1D9B44E8C81B54EF4D9B64EC2
:10E210008D81B74E8E81B84E8F81B94E9081BA4EA6
:10E22000CBC8BB4EE9D8BC4E9181BD4E9281BE4E4B
:10E230009381BF4EDAD2C04EB2CAC14ECAC8C24ED6
:10E24000ECD8C34EEAD8C44EC6D8C54EF6BDC64EAD
:10E25000CDC6C74EF0B3C84E9481C94EEBD8CA4E56
:10E26000F1BDCB4EE9BDCC4E9581CD4ED4C8CE4E3E
:10E27000D3B4CF4E9681D04E9781D14ED8C2D24ED4
:10E280009881D34ED6B2D44ED0D7D54ECBCAD64E27
:10E29000FBCBD74ECCD5D84EB6B8D94EC9CFDA4E77
:10E2A0009981DB4E9A81DC4E9B81DD4EDAD9DE4EC0
:10E2B000F0D8DF4EAAC7E04E9C81E14EEED8E24E88
:10E2C0009D81E34EFAB4E44EEEC1E54ED4D2E64E63
:10E2D0009E81E74E9F81E84EEDD8E94EA081EA4E3F
:10E2E000C7D2EB4EEFD8EC4EC7C3ED4EA181EE4E38
:10E2F000A281EF4EA381F04EF6D1F14EA481F24EF1
:10E30000D9D6F34EF2D8F44EA581F54EF5D8F64E97
:10E31000FEBCF74EDBBCF84EA681F94EA781FA4E43
:10E32000A881FB4ECEC8FC4EA981FD4EDDB7FE4E46
:10E33000AA81FF4EC2B7004FAB81014FF3C6024F17
:10E34000AC81034FAD81044FAE81054FAF81064FC5
:10E35000B081074FB181084FB281094FF8D80A4FF9
:10E36000C1D20B4FB3810C4FB4810D4FE9CE0E4F8C
:10E37000BFBC0F4FFCB7104FA5B7114FDDD0124FE8
:10E38000B581134FB681144FB781154FB881164F21
:10E39000B981174FDAD6184FC5D3194FEFBB1A4FB3
:10E3A000E1BB1B4FF1D81C4FBA811D4FBB811E4FE3
:10E3B000A1C91F4FB0CE204FABB4214FBC81224F1B
:10E3C000F3D8234FBD81244FCBC9254FF6D8264F14
:10E3D000D7C2274FF7D8284FBE81294FBF812A4F78
:10E3E000B1CE2B4FF9D82C4FC0812D4FC1812E4F6C
:10E3F000C2812F4FAEB2304FC0B9314FC381324FBF
:10E40000A3D9334FC481344FE9B0354FC581364F5E
:10E41000E6C1374FC681384FECC9394FC7813A4FF3
:10E42000C5CB3B4FC8813C4FC6CB3D4FA4D93E4FD7
:10E43000C9813F4FCA81404FCB81414FCC81424F70
:10E44000CD81434FE8B5444FCE81454FCF81464FF4
:10E45000ABB5474FD081484FD181494FD2814A4F08
:10E46000D3814B4FD4814C4FD5814D4FBBCE4E4FB6
:10E47000CDB54F4FA1D7504FF4D7514FD3D3524FB3
:10E48000D681534FE5CC544FD781554FCEBA564F16
:10E49000D881574FA2D9584FDCD9594FE0D35A4FA2
:10E4A000FDD85B4FF0B75C4FF7D75D4FFED85E4F9E
:10E4B000FAD85F4FA1D9604FE3C4614FD981624F51
:10E4C000DA81634FB6D3644FF4D8654FDDD9664F18
:10E4D000DB81674FFBD8684FDC81694FE5C56A4F28
:10E4E000DD816B4FDE816C4FD0C06D4FDF816E4F91
:10E4F000E0816F4FF0D1704FDBB0714FE181724F0F
:10E50000E281734FD1BC744FA6D9754FE381764F2A
:10E51000A5D9774FE481784FE581794FE6817A4F2D
:10E52000E7817B4FACD97C4FAED97D4FE8817E4FE0
:10E53000ABD97F4FB9CA804FE981814FEA81824FC1
:10E54000EB81834FA9D9844FB6D6854FEC81864F96
:10E55000ED81874FEE81884FDEB3894FA8D98A4F6E
:10E56000EF818B4FFDC08C4FF0818D4FCCCA8E4F09
:10E57000F1818F4FAAD9904FF281914FA7D9924F35
:10E58000F381934FF481944FB0D9954FF581964F15
:10E59000F681974FB1B6984FF781994FF8819A4F0E
:10E5A000F9819B4FA9B99C4FFA819D4FC0D29E4FD4
:10E5B000FB819F4FFC81A04FC0CFA14FFD81A24F97
:10E5C000FE81A34FC2C2A44F4082A54FC4BDA64F37
:10E5D000ECD5A74FE0B2A84FC8C7A94FEBBFAA4FD1
:10E5E000ADD9AB4F4182AC4FAFD9AD4F4282AE4FA8
:10E5F000EACEAF4FEEBAB04F4382B14F4482B24F32
:10E600004582B34F4682B44F4782B54FD6C7B64F07
:10E610004882B74F4982B84F4A82B94F4B82BA4FAE
:10E620004C82BB4F4D82BC4F4E82BD4F4F82BE4F7E
:10E630005082BF4FE3B1C04F5182C14F5282C24F8F
:10E640005382C34FD9B4C44FEDB6C54FB4D9C64FEA
:10E650005482C74F5582C84F5682C94F5782CA4FFE
:10E66000A1BFCB4F5882CC4F5982CD4F5A82CE4F4B
:10E67000DED9CF4FCEC7D04FFEC0D14FB8D9D24F81
:10E680005B82D34F5C82D44F5D82D54F5E82D64F82
:10E690005F82D74FD7CBD84FFDB7D94F6082DA4FC3
:10E6A000B5D9DB4F6182DC4FB7D9DD4FA3B1DE4F67
:10E6B000E1D3DF4FB9D9E04F6282E14FC5D0E24FDD
:10E6C0006382E34FB6D9E44F6482E54F6582E64F3B
:10E6D000B1D9E74F6682E84FB2D9E94FA9C1EA4FF5
:10E6E000B3D9EB4F6782EC4F6882ED4FF3BCEE4F2E
:10E6F000DED0EF4FA9B8F04F6982F14FE3BEF24F81
:10E700006A82F34FBDD9F44F6B82F54F6C82F64F9E
:10E710006D82F74F6E82F84FBAD9F94F6F82FA4F78
:10E72000B3B0FB4F7082FC4F7182FD4F7282FE4F7F
:10E73000C2D9FF4F7382005074820150758202501B
:10E740007682035077820450788205507982065091
:10E750007A8207507B8208507C8209507D820A5061
:10E760007E820B5080820C50C4D90D50B6B10E5031
:10E7700081820F50BFD91050828211508382125073
:10E78000B9B5135084821450F3BE155085821650CB
:10E790008682175087821850C8CC1950F2BA1A5086
:10E7A000D0D21B5088821C50C3D91D5089821E5064
:10E7B0008A821F50E8BD20508B822150ABB322507B
:10E7C0008C8223508D8224508E822550C5D92650AC
:10E7D000EBBE27508F822850C6D92950BBD92A506A
:10E7E000DFC42B5090822C50BED92D50C1D92E5051
:10E7F000C0D92F5091823050928231509382325042
:10E800009482335095823450968235509782365098
:10E8100098823750998238509A8239509B823A5068
:10E82000AED53B509C823C50B5D63D509D823E506B
:10E83000E3C73F509E8240509F824150A082425089
:10E84000A1824350C8D94450A2824550A382465069
:10E85000A4824750D9BC4850CAD94950A5824A50D1
:10E86000A6824B50A7824C50BCD94D50A8824E5026
:10E87000CBD94F50ABC65050A9825150AA825250AA
:10E88000AB825350AC825450AD825550C9D95650CA
:10E89000AE825750AF825850B0825950B1825A5010
:10E8A000F6D75B50B2825C50A3CD5D50B3825E5010
:10E8B000B4825F50B5826050B6826150B7826250B8
:10E8C000B8826350B9826450BA826550A1BD665067
:10E8D000BB826750BC826850BD826950BE826A505C
:10E8E000BF826B50C0826C50CCD96D50C1826E50CB
:10E8F000C2826F50C3827050C4827150C582725000
:10E90000C6827350C7827450C8827550C9827650CF
:10E91000BCC57750B5CD7850CA827950CB827A5039
:10E92000CC827B50CDD97C50CD827D50CE827E5022
:10E93000C7D97F50A5B38050FEBF8150CF8282508F
:10E94000D0828350D1828450D2828550B5B886500F
:10E95000D3828750D4828850FCC08950D5828A5097
:10E96000D6828B50D7828C50D8828D50F8B08E5082
:10E97000D9828F50DA829050DB829150DC829250A3
:10E98000DD829350DE829450DF829550E082965073
:10E99000E1829750E2829850E3829950E4829A5043
:10E9A000E5829B50E6829C50E7829D50E8829E5013
:10E9B000E9829F50EA82A050EB82A150EC82A250E3
:10E9C000ED82A350F6B4A450EE82A550CED9A65045
:10E9D000EF82A750CFD9A850A2B4A950D0D9AA503D
:10E9E000F082AB50F182AC50DFB4AD50F282AE5049
:10E9F000F382AF50F482B050F582B150F682B2503B
:10EA0000C1B0B350F782B450F882B550F982B65015
:10EA1000FA82B750FB82B850FC82B950FD82BA50DE
:10EA2000D1D9BB50B5C9BC50FE82BD504083BE5049
:10EA30004183BF504283C0504383C1504483C2507E
:10EA40004583C3504683C4504783C5504883C6504E
:10EA50004983C7504A83C8504B83C9504C83CA501E
:10EA60004D83CB504E83CC504F83CD505083CE50EE
:10EA70005183CF50F1CFD0505283D1505383D250D5
:10EA80005483D3505583D4505683D5505783D65092
:10EA9000D2D9D7505883D8505983D9505A83DA5095
:10EAA000C5C1DB505B83DC505C83DD505D83DE5091
:10EAB0005E83DF505F83E0506083E1506183E2500A
:10EAC0006283E3506383E4506483E5506583E650DA
:10EAD000D6D9E750AEC9E8506683E9506783EA505B
:10EAE0006883EB506983EC50D5D9ED50D4D9EE5002
:10EAF000D7D9EF506A83F0506B83F1506C83F2509A
:10EB00006D83F350DBCBF4506E83F550A9BDF65006
:10EB10006F83F7507083F8507183F9507283FA5005
:10EB20007383FB50A7C6FC507483FD507583FE5061
:10EB30007683FF50778300517883015179830251A6
:10EB40007A8303517B8304517C8305517D83065175
:10EB5000D3D90751D8D908517E83095180830A51EE
:10EB600081830B51D9D90C5182830D5183830E516E
:10EB700084830F51858310518683115187831251ED
:10EB8000E5C8135188831451898315518A8316511E
:10EB90008B8317518C8318518D8319518E831A5191
:10EBA0008F831B5190831C5191831D5192831E5161
:10EBB00093831F519483205195832151DCC02251AE
:10EBC0009683235197832451988325519983265105
:10EBD0009A8327519B8328519C8329519D832A51D5
:10EBE0009E832B519F832C51A0832D51A1832E51A5
:10EBF000A2832F51A3833051A4833151A583325175
:10EC0000A6833351A7833451A8833551A983365144
:10EC1000AA833751AB833851AC833951AD833A5114
:10EC2000AE833B51AF833C51B0833D51B1833E51E4
:10EC3000B2833F51F9B64051A3D84151CAD4425191
:10EC4000B3834351AAD44451D6D04551E4B346517D
:10EC5000D7D54751B4834851C8CF4951E2B94A5139
:10EC6000B5834B51CBBF4C51B6834D51E2C34E518E
:10EC7000B7834F51B8835051B9835151D2B65251D5
:10EC8000BA835351BB835451C3CD5551EED956511C
:10EC9000F0D95751BC835851BD835951BE835A5145
:10ECA000B3B55B51BF835C51B5B65D51C0835E5156
:10ECB000C1835F51C2836051C3836151C483625178
:10ECC000A4BE6351C5836451C6836551EBC86651C8
:10ECD000C7836751C8836851ABC86951C9836A51FA
:10ECE000CA836B51CBB06C51ABB96D51F9C16E5148
:10ECF000E2D96F51CB837051BCC07151B2B972511E
:10ED0000CC837351D8B97451CBD07551F8B17651C9
:10ED1000E4C67751DFBE7851E4B57951C8D77A514E
:10ED2000CD837B51F8D17C51E6BC7D51DECA7E514A
:10ED3000CE837F51CF838051BDBC8151E6D98251B2
:10ED4000E7D88351D0838451D1838551DAC4865169
:10ED5000D2838751D3838851D4B88951BDC88A5191
:10ED6000D4838B51D5838C51E1B28D51D9D48E513E
:10ED7000D6838F51D7839051D8839151D9839251A3
:10ED8000B0C39351DA839451DB839551E1C396511B
:10ED9000A2DA9751DFC89851DC839951B4D09A51C7
:10EDA000DD839B51FCBE9C51A9C59D51DE839E51C4
:10EDB000DF839F51E083A051DAB9A151E183A251D1
:10EDC000A3DAA351E283A451A9D4A551A4DAA65190
:10EDD000E383A751E483A851E583A951E683AA51AF
:10EDE000E783AB51FBD9AC51ACB6AD51E883AE5122
:10EDF000E983AF51EBB7B051F9B1B151FCD9B25180
:10EE0000E5B3B351F6BEB451EA83B551F6BFB6517E
:10EE1000B1D2B751E4C0B851EB83B951EC83BA51C8
:10EE2000ED83BB51B3B6BC51FED9BD51FDD9BE5126
:10EE3000EE83BF51EF83C051BBBEC151F083C251BD
:10EE4000F183C351F283C451E0C6C551F383C65167
:10EE5000BCD7C751A1DAC851F483C951B9C1CA514D
:10EE6000F583CB51F2B5CC51E8C1CD51F683CE51EB
:10EE7000F783CF51F5BCD051F883D151D5B4D251DD
:10EE8000F983D351FA83D451FB83D551FC83D651F6
:10EE9000FD83D751FE83D8514084D9514184DA5142
:10EEA0004284DB51DDC1DC514384DD51FDC4DE51C0
:10EEB0004484DF514584E051B8BCE151B2B7E2511E
:10EEC0004684E3514784E451EFB7E5514884E65165
:10EED0004984E7514A84E8514B84E9514C84EA5112
:10EEE0004D84EB51ECD9EC514E84ED51BEC6EE5140
:10EEF0004F84EF51ADBFF051CBBBF1515084F25173
:10EF00005184F351CAB5F4515284F551C9DBF6511D
:10EF1000D7D0F7515384F851B9CDF951BCB0FA515B
:10EF2000F6B3FB51F7BBFC51CADBFD51AFBAFE5142
:10EF30005484FF51E4D40052B6B50152F3B50252E5
:10EF4000D6D80352D0C8045255840552568406526E
:10EF5000D6B70752D0C70852D7D8095257840A5299
:10EF6000AFBF0B5258840C5259840D52BBDB0E526A
:10EF7000D8D80F525A8410525B841152CCD01252FE
:10EF8000AEBB13525C8414525D8415525E841652DB
:10EF9000BEEB1752D0C11852F5C11952F2D41A5211
:10EFA000D5B81B52B4B41C525F841D52F5B31E5227
:10EFB00060841F5261842052BEC921526284225251
:10EFC0006384235264842452D0C52552658426521A
:10EFD0006684275267842852D9C52952FBC02A5219
:10EFE00068842B52F0B12C5269842D52D9D82E52FC
:10EFF000CEB92F526A843052BDB531526B84325231
:10F000006C843352DAD834526D8435526E84365261
:10F01000C6D63752A2CB3852AFC83952B2C93A52CB
:10F02000CCB43B52CCBF3C526F843D52F4B93E52FB
:10F0300070843F52DBD84052DCD84152E7B642528E
:10F04000C1BC4352EACC4452718445527284465248
:10F0500073844752748448527584495276844A5264
:10F06000F7CF4B5277844C52DDD84D52B0C74E5239
:10F0700078844F5279845052D0B95152A3BD525224
:10F080007A8453527B845452DECC55527C8456523F
:10F09000CAC657527D8458527E84595280845A522F
:10F0A00081845B5282845C52E0D85D5283845E52DC
:10F0B000DED85F528484605285846152DFD8625208
:10F0C000868463528784645288846552FEB0665297
:10F0D00089846752E7BE68528A846952A3CA6A5219
:10F0E000F4BC6B528B846C528C846D528D846E5246
:10F0F0008E846F52B1B870528F8471529084725264
:10F10000EEB87352918474529284755293847652FD
:10F1100094847752958478529684795297847A525F
:10F1200098847B5299847C529A847D52E2D87E5294
:10F130009B847F52CBBD80529C848152E4D8825202
:10F14000E3D883529D8484529E8485529F84865244
:10F15000A0848752A1848852FCC58952A2848A5215
:10F16000A3848B52A4848C52A5848D52A6848E5283
:10F17000A7848F52A8849052E5D89152A9849252C4
:10F18000AA849352E6D89452AB849552AC8496529A
:10F19000AD849752AE849852AF849952B0849A52FB
:10F1A000B1849B52A6C19C52B2849D52B0C89E525B
:10F1B000ECB09F52A6B9A052D3BCA152F1CEA2523C
:10F1C000BDDBA352D3C1A452B384A552B484A652CA
:10F1D000B584A752B684A852AFB6A952FAD6AA529D
:10F1E000ACC5AB52D9BDAC52BEDBAD52BFDBAE52EB
:10F1F000B784AF52B884B052B984B152F8C0B25299
:10F20000A2BEB352CDC0B452BA84B552BB84B6527A
:10F21000BC84B752BD84B852BE84B952BF84BA52BE
:10F22000C084BB52C184BC52C284BD52C384BE528E
:10F23000C0DBBF52C6CAC052C484C152C584C252C8
:10F24000C684C352AAB2C452C784C552C884C65227
:10F25000C984C752C2D3C852CA84C952E3C3CA526E
:10F26000CB84CB52ABD1CC52CC84CD52CD84CE52B8
:10F27000CE84CF52CF84D052C2DBD152D084D2526E
:10F28000D5C0D352D184D452D284D552D384D6524D
:10F29000C3DBD752D484D852B1BFD952D584DA5205
:10F2A000D684DB52D784DC52D884DD52D984DE5236
:10F2B000DA84DF52BCC4E052DB84E152DC84E252E7
:10F2C000DD84E352DE84E452DAC7E552DF84E6529D
:10F2D000E084E752E184E852E284E952E384EA52AE
:10F2E000E484EB52E584EC52E684ED52E784EE527E
:10F2F000E884EF52E984F052C4DBF152EA84F2521E
:10F30000EB84F352EC84F452ED84F552EE84F65221
:10F31000EF84F752F084F852F184F952E8D9FA52A6
:10F32000D7C9FB52F284FC52F384FD52F484FE529E
:10F33000B4B9FF52F0CE0053C8D40153F584025340
:10F34000F6840353F7840453F8840553FCB0065342
:10F35000D2B40753F9840853D9D00953FA840A5315
:10F36000FB840B53FC840C53FD840D53E9D90E53DD
:10F37000FE840F53CBDE1053EBD91153408512534B
:10F38000418513534285145343851553B0D8165302
:10F39000AFBB1753B1B1185344851953D7B31A53A0
:10F3A000CED81B5345851C5346851D53D1D41E53BF
:10F3B00047851F5348852053B3BD2153EFBF2253C8
:10F3C00049852353BBCF24534A8525534B85265368
:10F3D000D0D827534C8528534D8529534E852A5321
:10F3E000CBB72B534F852C5350852D5351852E531E
:10F3F000D1D82F53528530535385315354853253CE
:10F400005585335356853453578535535885365370
:10F41000598537535A8538535B853953A5C63A53B6
:10F42000F8C73B53BDD23C535C853D535D853E538D
:10F43000D2D83F53E4C440535E854153AECA4253D1
:10F440005F854353A7C7445360854553A6D84653A9
:10F4500061854753FDC94853E7CE4953DCBB4A5346
:10F46000EBB04B5362854C5363854D5364854E53CB
:10F47000AABB4F53ADD0505365855153B0B15253D1
:10F48000E4D75353BFD7545366855553A5B5565348
:10F49000F4C25753CFC458536785595368855A539C
:10F4A000A9B25B5369855C53B7B25D536A855E53FD
:10F4B000E5B15F53B2DF6053BCD56153A8BF62535F
:10F4C000ACC26353D5D86453B1C265536B856653E0
:10F4D000D4D86753D4CE68536C856953E0DA6A5345
:10F4E0006D856B53C0CE6C536E856D536F856E53B7
:10F4F000B4D86F53AEC37053A1D37153A3CE72531C
:10F5000070857353B4BC7453B4C87553D1C2765369
:10F5100071857753EDBE7853B6D0795372857A539F
:10F52000E1DA7B5373857C5374857D5375857E53F7
:10F5300076857F53E4C780537785815378858253DE
:10F54000A7B3835379858453F2B68553FCCC865395
:10F55000FAC087537A8588537B858953F7C08A53CD
:10F560007C858B53B9D18C53E1D18D53C7D88E5341
:10F570007D858F537E8590538085915381859253ED
:10F58000828593538385945384859553DEB2965335
:10F590008585975386859853E5C0995387859A53F7
:10F5A000F1BA9B5388859C5389859D53C8D89E5337
:10F5B0008A859F53ADD4A0538B85A1538C85A253CC
:10F5C000E1CFA353C9D8A4538D85A553CAD8A65358
:10F5D000C3CFA7538E85A853F8B3A953C7BEAA5368
:10F5E0008F85AB539085AC539185AD539285AE53C7
:10F5F000CBD8AF539385B0539485B1539585B2530F
:10F600009685B3539785B4539885B5539985B6536A
:10F61000CCDBB7539A85B8539B85B9539C85BA53B5
:10F620009D85BB53A5C8BC539E85BD539F85BE53C6
:10F63000A085BF53D8CFC053A185C153FEC8C253C4
:10F64000CEB2C353A285C453A385C553A485C65364
:10F65000A585C753A685C853D6D3C953E6B2CA53A6
:10F66000B0BCCB53D1D3CC53ABCBCD53B4B7CE532B
:10F67000A785CF53A885D053A985D153A2B7D2531C
:10F68000AA85D353AB85D453E5CAD553AC85D6539D
:10F69000A1C8D753DCCAD853E4B1D953F0D0DA5358
:10F6A000AD85DB53D1C5DC53AE85DD53AF85DE536D
:10F6B000B085DF53C5DBE053FEB5E153B185E253BE
:10F6C000B285E353DABFE453C5B9E553E4BEE6536C
:10F6D000EDC1E753B385E853B6DFE953B5DFEA532D
:10F6E000BBD6EB53D0BDEC53D9D5ED53C8B0EE53D8
:10F6F000A3B6EF53C9BFF053A8CCF153B3DFF25315
:10F70000B7CAF353D2D3F453B485F553CFD8F653D5
:10F71000B6D2F753C5BAF853BECBF953BECCFA53A1
:10F72000B585FB53B7DFFC53F0B5FD53B4DFFE5393
:10F73000B685FF53B7850054B8850154F5D30254FC
:10F74000B9850354D4B30454F7B80554BA850654A4
:10F75000BADF0754BB850854CFBA0954AABC0A546F
:10F76000F5B50B54BC850C54ACCD0D54FBC30E54F5
:10F77000F3BA0F54F4C01054C2CD1154F2CF125446
:10F78000B8DF1354C5CF1454BD851554C0C21654E8
:10F79000B9DF1754F0C21854BE851954BF851A54E6
:10F7A000C0851B54FDBE1C54C1851D54DFC11E54B1
:10F7B000CCCD1F54F7D22054CDB72154C1DF2254F1
:10F7C000C2852354C4DF2454C3852554C4852654DC
:10F7D000F1B72754C9B02854D6B62954D4B72A54FF
:10F7E000C5852B54ACBA2C54FDCC2D54D4BF2E540B
:10F7F000B1CB2F54F4C63054C6853154A8D63254F8
:10F80000C5DF3354C7853454E2CE3554B3B33654D0
:10F81000C8853754C9853854FCCE3954B5B43A54E8
:10F82000CA853B54C7CE3C54F0BA3D54CB853E54B8
:10F83000E1CE3F54CC854054BDD14154CD85425496
:10F84000CE854354C0DF4454CF854554D0854654BB
:10F85000F4B44754D1854854CAB34954D2854A5464
:10F86000E6B84B54BBDF4C54D3854D54D4854E542D
:10F87000D5854F54D6855054C5C45154D78552545C
:10F88000BCDF5354BDDF5454BEDF5554BBC5565482
:10F89000BFDF5754C2DF5854B1D45954C3DF5A5450
:10F8A000D8855B54BAC75C54D8CE5D54D9855E54B4
:10F8B000DA855F54DB856054DC856154DD856254F4
:10F8C000D8C46354DE856454CADF6554DF8566544A
:10F8D000CFDF6754E0856854DCD66954E1856A540B
:10F8E000E2856B54E3856C54E4856D54E5856E5474
:10F8F000E6856F54E7857054E8857154C9DF72540A
:10F90000DADF7354B6CE7454E9857554C7BA7654A9
:10F91000CEDF7754C8DF7854DEC57954EA857A544F
:10F92000EB857B54EBC97C54F4BA7D54FCC37E5404
:10F93000EC857F54ED858054D7BE8154EE8582548A
:10F94000C6DF8354EF858454CDDF8554F08586541B
:10F95000D8C58754F1858854F2858954F3858A5433
:10F96000F4858B54A6D58C54CDBA8D54F5858E5420
:10F97000CCBE8F54BDD39054C0B89154F6859254E8
:10F98000E4D69354F7859454C7DF9554BEB9965482
:10F99000A7BF9754F8859854F9859954FCC19A5497
:10F9A000CBDF9B54CCDF9C54FA859D54D0DF9E5412
:10F9B000FB859F54FC85A054FD85A154FE85A2546F
:10F9C0004086A354DBDFA454E5DFA5544186A6544A
:10F9D000D7DFA754D6DFA854C9D7A954E3DFAA5468
:10F9E000E4DFAB54EBE5AC54A7D2AD54D2DFAE5458
:10F9F0004286AF54A9BFB0544386B154DBD4B2544D
:10FA00004486B354C8BFB454D4DFB5544586B65405
:10FA10004686B7544786B854CCCFB9544886BA54B2
:10FA20004986BB54DDDFBC544A86BD54CAD1BE549E
:10FA30004B86BF54DEDFC054A7B0C154B7C6C25412
:10FA4000D3DFC3544C86C454E5BAC5544D86C6545E
:10FA5000DFB6C754DBCDC854FEB9C954D5D4CA5497
:10FA60004E86CB544F86CC54DFDFCD54ECCFCE54F2
:10FA7000A5B0CF54E7DFD054D1DFD154C6D1D25492
:10FA8000D5DFD354D8DFD454D9DFD554DCDFD654F6
:10FA90005086D754A9BBD8545186D954E0DFDA54E4
:10FAA000E1DFDB545286DC54E2DFDD54E6DFDE5476
:10FAB000E8DFDF54B4D3E0545386E1545486E25473
:10FAC0005586E3545686E4545786E554E7B8E65421
:10FAD000B6C5E754EADFE854DAC9E954A8C1EA54E4
:10FAE000C4C4EB545886EC545986ED54DEBFEE5432
:10FAF000F8CFEF545A86F0545B86F1545C86F2548A
:10FB0000DCD5F354EEDFF4545D86F5545E86F6548E
:10FB10005F86F7546086F8546186F9546286FA5419
:10FB2000B8B2FB546386FC54DFBAFD54ECDFFE54DC
:10FB30006486FF54C1DB005565860155E4D102554A
:10FB40006686035567860455688605556986065599
:10FB5000F4CB0755BDB408556A860955A6B00A55B9
:10FB60006B860B556C860C556D860D556E860E5545
:10FB70006F860F55F1DF1055C6CC1155F2DF1255C7
:10FB80007086135571861455EDDF1555728616551E
:10FB900073861755748618557586195576861A55C5
:10FBA00077861B55E9DF1C5578861D5579861E55CD
:10FBB0007A861F557B862055EBDF21557C862255A2
:10FBC000EFDF2355F0DF2455BDBB25557D86265537
:10FBD0007E862755F3DF28558086295581862A554C
:10FBE000F4DF2B5582862C55A3BB2D5583862E55CD
:10FBF000DBCA2F55A8CE3055A7E03155AAB33255F0
:10FC000084863355A6E03455858635558686365527
:10FC100087863755A1E038558886395589863A5503
:10FC20008A863B558B863C55FEDF3D558C863E557E
:10FC3000D9CD3F55FCDF40558D864155FADF425501
:10FC40008E864355D0BF4455C4D745558F864655FB
:10FC5000CCC947559086485591864955F8DF4A5595
:10FC6000A1B04B5592864C5593864D5594864E5572
:10FC700095864F5596865055FDDF515597865255BE
:10FC800098865355998654559A865555FBDF565597
:10FC9000A2E057559B8658559C8659559D865A55C6
:10FCA0009E865B559F865C55A8E05D55A0865E5597
:10FCB000A1865F55A2866055A3866155C8B7625577
:10FCC000A4866355A5866455A1C66555B6C9665513
:10FCD000B2C06755F5DF6855A6866955A7866A558F
:10FCE000BEC56B55A8866C55C4D86D55F9DF6E55E9
:10FCF000F6C46F55A9867055AA867155AB867255A4
:10FD0000AC867355AD867455AE867555A3E07655B1
:10FD1000A4E07755A5E07855A5D07955AF867A55FA
:10FD2000B0867B55B4E07C55E4CC7D55B1867E55DC
:10FD3000B1E07F55B2868055A6BF8155AFE08255B0
:10FD4000B9CE8355ABE08455C6C98555B386865573
:10FD5000B4868755AEC08855AEE08955EDBA8A5550
:10FD6000B0BA8B55A9E08C55B5868D55B6868E55A3
:10FD7000B7868F55F6DF9055B8869155B3E092550A
:10FD8000B9869355BA869455B8E09555BB86965575
:10FD9000BC869755BD869855ADB49955B9E09A552E
:10FDA000BE869B55BF869C55B2CF9D55C8BA9E5501
:10FDB000C0869F55B0E0A055C186A155C286A25508
:10FDC000C386A355C486A455C586A555C686A65523
:10FDD000C786A755FAD0A855C886A955C986AA5579
:10FDE000CA86AB55CB86AC55CC86AD55CD86AE55C7
:10FDF000CE86AF55CF86B055D086B155ACE0B25562
:10FE0000D186B355FBD4B455D286B555F7DFB65578
:10FE1000D386B755E7C5B855D486B955ADE0BA55C0
:10FE2000D586BB55F7D3BC55D686BD55B6E0BE5575
:10FE3000B7E0BF55D786C055D886C155D986C255BB
:10FE4000DA86C355DB86C455C4E0C555E1D0C65536
:10FE5000DC86C755DD86C855DE86C955BCE0CA5567
:10FE6000DF86CB55E086CC55C9E0CD55CAE0CE55EE
:10FE7000E186CF55E286D055E386D155BEE0D25516
:10FE8000AAE0D355A4C9D455C1E0D555E486D655CA
:10FE9000B2E0D755E586D855E686D955E786DA55D6
:10FEA000E886DB55E986DC55C8CADD55C3E0DE557A
:10FEB000EA86DF55B5E0E055EB86E155CBCEE2555D
:10FEC000EC86E355C3CBE455CDE0E555C6E0E655F9
:10FED000C2E0E755ED86E855CBE0E955EE86EA55F8
:10FEE000BAE0EB55BFE0EC55C0E0ED55EF86EE55BE
:10FEF000F086EF55C5E0F055F186F155F286F255E2
:10FF0000C7E0F355C8E0F455F386F555CCE0F65557
:10FF1000F486F755BBE0F855F586F955F686FA559F
:10FF2000F786FB55F886FC55F986FD55D4CBFE5572
:10FF3000D5E0FF55FA860056D6E00156D2E00256CB
:10FF4000FB860356FC860456FD860556FE8606563D
:10FF50004087075641870856D0E00956CEBC0A565E
:10FF600042870B5643870C56D1E00D5644870E56F8
:10FF7000C2B80F56C5D81056458711564687125637
:10FF80004787135648871456498715564A87165689
:10FF90004B8717564C871856EAD019564D871A5674
:10FFA0004E871B56EFC21C564F871D5650871E5654
:10FFB000CFE01F56BDE0205651872156528722566A
:10FFC00053872356D4E02456D3E02556548726562B
:10FFD00055872756D7E028565687295657872A56D9
:10FFE00058872B5659872C56DCE02D56D8E02E56D4
:10FFF0005A872F565B8730565C873156F6D6325675
:020000040801F1
:10000000B0B333565D873456ECD735565E873656D7
:10001000BBCB37565F87385660873956DAE03A5699
:1000200061873B56FBCE3C5662873D5663873E5602
:1000300064873F56D9BA405665874156668742560F
:100040006787435668874456698745566A87465688
:100050006B8747566C8748566D8749566E874A5658
:100060006F874B5670874C56E1E04D56DDE04E569B
:10007000ADD24F567187505672875156738752567C
:100080007487535675875456E2E055567687565610
:1000900077875756DBE05856D9E05956DFE05A5675
:1000A00078875B5679875C56E0E05D567A875E56C6
:1000B0007B875F567C8760567D8761567E87625658
:1000C000DEE0635680876456E4E0655681876656B5
:1000D0008287675683876856F7C66956ACD86A56D2
:1000E000EBD46B56E6E06C56C9CA6D5684876E56E3
:1000F00085876F568687705687877156E5E07256FA
:1001000088877356898774568A8775568B87765683
:10011000C1B877568C8778568D8779568E877A56F0
:100120008F877B56E7E07C56E8E07D5690877E56C9
:1001300091877F56928780569387815694878256FF
:10014000958783569687845697878556E9E0865625
:10015000E3E0875698878856998789569A878A5602
:100160009B878B569C878C569D878D569E878E5677
:10017000BFBA8F56E7CC90569F879156A08792566C
:10018000A1879356EAE09456A2879556A387965680
:10019000A4879756A5879856A6879956A7879A56F3
:1001A000A8879B56A9879C56AA879D56AB879E56C3
:1001B000AC879F56AD87A056AE87A156AF87A25693
:1001C000B087A356F9CFA456B187A556B287A656D5
:1001D000B387A756B487A856B587A956B687AA5637
:1001E000B787AB56B887AC56B987AD56BA87AE5607
:1001F000BB87AF56EBE0B056BC87B156BD87B25651
:10020000BE87B356BF87B456C087B556C187B656AA
:10021000C287B756C2C8B856C387B956C487BA563C
:10022000C587BB56C687BC56C0BDBD56C787BE5620
:10023000C887BF56C987C056CA87C156CB87C25622
:10024000CC87C356CD87C456CE87C556CF87C656F2
:10025000D087C756D187C856D287C956D387CA56C2
:10026000D2C4CB56D487CC56D587CD56D687CE565A
:10027000D787CF56D887D056D987D156DA87D25666
:10028000DB87D356DC87D456ECE0D556DD87D656CF
:10029000DE87D756EDE0D856DF87D956E087DA56A5
:1002A000F4C7DB56C4CBDC56E187DD56EEE0DE5604
:1002B000D8BBDF56B6D8E056F2D2E156EFE0E256B0
:1002C000C5CDE356E287E456DAB6E556E387E6564F
:1002D000E487E756E587E856E687E956E787EA5672
:1002E000E887EB56F1E0EC56E987ED56B0D4EE56D0
:1002F000EA87EF56EB87F056A7C0F156D1B4F25615
:10030000EC87F356ED87F456A7CEF556F0E0F65697
:10031000EE87F756EF87F856F087F956F2E0FA566F
:10032000CCB9FB56F187FC56F287FD56FAB9FE565A
:10033000BCCDFF56F3E00057F3870157F48702570F
:10034000F5870357D4C60457F4E00557F6870657D8
:10035000B2D40757F7870857A6C80957F6E00A57D7
:10036000F5E00B57F8870C57F9870D57FA870E57AA
:10037000FB870F57FC871057FD871157FE871257D1
:100380004088135741881457428815574388165799
:1003900044881757458818574688195747881A5769
:1003A00048881B5749881C57F7E01D574A881E5735
:1003B0004B881F57C1CD20574C8821574D88225755
:1003C0004E882357A5CA24574F882557508826574B
:1003D0005188275752882857DAD42957D7DB2A570C
:1003E000D9DB2B5753882C57D8DB2D57E7B92E571D
:1003F000DCDB2F57DDDB3057D8B531575488325707
:1004000055883357DADB345756883557578836576F
:1004100058883757598838575A883957DBDB3A5745
:10042000A1B33B57DFDB3C575B883D575C883E57A9
:10043000F8BB3F575D884057B7D641575E88425753
:10044000E0DB43575F8844576088455761884657CB
:1004500062884757F9BE48576388495764884A57A6
:10046000BBB74B5765884C57D0DB4D57AECC4E577A
:10047000B2BF4F57B5BB5057F8D75157D3BF52579C
:100480006688535767885457688855576988565700
:100490006A885757E9BF58576B8859576C885A571D
:1004A000E1BC5B57B3CC5C57DEDB5D57D3B05E5726
:1004B000EBCE5F57D8B76057B9D76157C2C66257FE
:1004C0006D8863576E886457A4C065576F886657F8
:1004D000B9CC675770886857E7DB6957E1DB6A5723
:1004E000BAC66B57E3DB6C5771886D57E8DB6E5704
:1004F00072886F57F7C57057738871577488725731
:1005000075887357EADB74577688755777887657FE
:10051000E9DB7757C0BF78577888795779887A5759
:100520007A887B57E6DB7C57E5DB7D577B887E57F7
:100530007C887F577D8880577E8881578088825746
:10054000B9B48357ACC08457A2C28557E2DB865743
:10055000E4DB8757818888578288895783888A5740
:1005600084888B57CDD08C57EDDB8D5785888E577F
:1005700086888F578788905788889157898892579F
:10058000DDC09357F2DB94578A8895578B8896572E
:100590008C8897578D8898578E8899578F889A5747
:1005A00090889B57E2B69C5791889D5792889E579A
:1005B00093889F579488A057F3DBA157D2DBA257AB
:1005C000B8B9A357ABD4A457ECDBA5579588A65769
:1005D000D1BFA757F0DBA8579688A957D1DBAA57F8
:1005E0009788AB57E6B5AC579888AD57EBDBAE575D
:1005F000E5BFAF579988B0579A88B1579B88B257D3
:10060000EEDBB3579C88B457F1DBB5579D88B657DE
:100610009E88B7579F88B857F9DBB957A088BA5753
:10062000A188BB57A288BC57A388BD57A488BE57D2
:10063000A588BF57A688C057A788C157A888C257A2
:10064000A1B9C357A3B0C457A988C557AA88C6572C
:10065000AB88C757AC88C857AD88C957AE88CA574A
:10066000AF88CB57F1C2CC57B088CD57B188CE57A1
:10067000C7B3CF57EFDBD057B288D157B388D25723
:10068000F8DBD357B488D457D2C6D557F4DBD65746
:10069000B588D757B688D857F5DBD957F7DBDA577F
:1006A000F6DBDB57B788DC57B888DD57FEDBDE5753
:1006B000B988DF57F2D3E057BAB2E157BA88E257A8
:1006C000BB88E357BC88E457FDDBE557BD88E65798
:1006D000BE88E757BF88E857C088E957C188EA57FE
:1006E000C288EB57C388EC57C488ED57A4DCEE579B
:1006F000C588EF57FBDBF057C688F157C788F2571C
:10070000C888F357C988F457FADBF557CA88F657F3
:10071000CB88F757CC88F857FCDBF957E0C5FA5778
:10072000F9BBFB57CD88FC57CE88FD57A3DCFE579D
:10073000CF88FF57D0880058A5DC0158D1880258CF
:10074000C3CC0358D2880458D3880558D488065897
:10075000D1B60758C0DD0858D5880958D6880A5838
:10076000D7880B58A1DC0C58D8880D58A2DC0E583D
:10077000D9880F58DA881058DB881158B5C7125835
:10078000DC881358DD881458DE881558E9B61658E9
:10079000DF881758E0881858E1881958A7DC1A58DC
:1007A000E2881B58E3881C58E4881D58E5881E58C9
:1007B000A6DC1F58E6882058A9DC2158A4B122588D
:1007C000E7882358E8882458CCB52558E988265866
:1007D000EA882758EB882858EC882958ED882A5849
:1007E000B0BF2B58EE882C58EF882D58F0882E5823
:1007F000F1882F58F2883058DFD13158F3883258B9
:10080000F4883358F5883458F6883558C2B63658C7
:10081000F7883758F8883858F9883958FA883A5894
:10082000FB883B58FC883C58FD883D58FE883E5864
:1008300040893F584189405842894158438942582C
:100840004489435845894458A8DC45584689465848
:100850004789475848894858498949584A894A58D0
:100860004B894B584C894C58FACB4D58F3EB4E58AA
:100870004D894F584E8950584F895158DCCB5258AA
:100880005089535851895458FECB5558528956585F
:100890005389575854895858C1CC595855895A5872
:1008A00056895B5857895C5858895D5859895E58F4
:1008B000FBC85F585A8960585B8961585C896258E7
:1008C0005D8963585E8964585F896558AADC6658FB
:1008D00060896758618968586289695863896A586C
:1008E00064896B58EECC6C58ABDC6D5865896E58DA
:1008F00066896F5867897058688971586989725814
:100900006A8973586B8974586C8975586D897658E3
:100910006E8977586F8978587089795871897A58B3
:1009200072897B5873897C5874897D5875897E5883
:10093000D3DB7F5876898058AFDC8158ACDC825895
:1009400077898358B3BE845878898558FBCA8658FE
:10095000798987587A8988587B898958ADDC8A5883
:100960007C898B587D898C587E898D5880898E58DA
:1009700081898F58828990588389915884899258A7
:10098000CAC99358B9C49458858995588689965888
:10099000878997588889985889899958BDC79A58DE
:1009A000AEDC9B588A899C588B899D588C899E58AF
:1009B000F6D49F58E6D0A0588D89A1588E89A258A8
:1009C0008F89A3589089A4589189A5589289A658CF
:1009D0009389A7589489A858ABC4A958D5B6AA58E2
:1009E0009589AB589689AC589789AD589889AE5877
:1009F0009989AF589A89B0589B89B1589C89B25847
:100A00009D89B3589E89B4589F89B558A089B65816
:100A1000A189B758A289B858A389B958A489BA58E6
:100A2000A589BB58A689BC58D4DBBD58A789BE5838
:100A3000A889BF58A989C058AA89C158DAB1C25833
:100A4000AB89C358AC89C458AD89C558D5DBC658E5
:100A5000AE89C758AF89C858B089C958B189CA5832
:100A6000B289CB58B389CC58B489CD58B589CE5802
:100A7000B689CF58B789D058B889D158D6DBD25863
:100A8000B989D358BA89D458BB89D558BEBAD65873
:100A9000BC89D758BD89D858BE89D958BF89DA587A
:100AA000C089DB58C189DC58C289DD58C389DE584A
:100AB000C489DF58C589E058C689E158C789E2581A
:100AC000C889E358C989E458C0C8E558CA89E658B6
:100AD000CB89E758CC89E858CD89E958CE89EA58BE
:100AE000CF89EB58BFCAEC58C9C8ED58D089EE5829
:100AF000B3D7EF58D189F058F9C9F158D289F258D3
:100B0000D389F358C7BFF458D489F558D589F65816
:100B1000F8BAF758D689F858D789F958BCD2FA5894
:100B2000D889FB58D989FC58DA89FD58DB89FE58E9
:100B3000DC89FF58DD890059DE890159DF890259B6
:100B4000BAE20359E0890459A6B40559E189065966
:100B5000E2890759B8B10859E3890959E4890A5962
:100B6000E5890B59E6890C59E7890D59B4B80E5936
:100B7000E8890F59C4CF1059E9891159EA891259E6
:100B8000EB891359EC891459E7D91559A6CF165991
:100B9000E2CD1759ED891859EE891959EDD91A592D
:100BA000E0B61B59EF891C59B9D21D59F0891E595D
:100BB000F1891F59BBB92059F2892159F38922596A
:100BC000F4892359F5892459B9E22559B7E2265900
:100BD000F6892759F3B42859F7892959ECCC2A59B1
:100BE000ABCC2B59F2B72C59F8892D59B2D82E59C4
:100BF000EBD12F59BBBA3059F9893159A7CA3259AB
:100C0000FA893359FB893459B7CD3559FC8936599E
:100C1000FD893759C4D23859E4BF3959D0BC3A5943
:100C2000E1B63B59FE893C59C5DE3D59408A3E59E3
:100C3000418A3F59428A4059438A4159C6DE425946
:100C4000BCDB4359448A4459D9D14559458A465950
:100C5000468A4759E6C64859CEC44959EEB74A595B
:100C6000478A4B59DCB74C59488A4D59498A4E59E5
:100C7000FCBF4F59E0D750594A8A5159F5C65259CD
:100C80004B8A53594C8A5459BCB15559C8DE5659F0
:100C9000B1BD5759D7CC5859CADE59594D8A5A59FE
:100CA000C9DE5B594E8A5C594F8A5D59508A5E593C
:100CB000518A5F59528A6059ECB56159538A625919
:100CC000DDC96359548A6459558A6559C2B0665959
:100CD000568A6759578A6859588A6959598A6A5988
:100CE0005A8A6B595B8A6C595C8A6D595D8A6E5958
:100CF0005E8A6F595F8A7059608A7159618A725928
:100D0000628A7359AEC57459ABC57559638A7659F1
:100D1000CCC47759648A7859E9BC7959FDCB7A59A2
:100D2000658A7B59668A7C59678A7D59C3BA7E5920
:100D3000688A7F59698A80596A8A8159F9E5825996
:100D4000E7C88359FAE58459FDCD85596B8A8659E0
:100D5000B1D78759BEB88859E8C289596C8A8A596F
:100D6000D1C88B596D8A8C596E8A8D59FBE58E5985
:100D70006F8A8F59708A9059718A9159728A9259E3
:100D8000CAB69359CBBC9459738A9559748A9659AB
:100D9000FDD19759A1E69859758A9959EEC39A5988
:100DA000768A9B59778A9C59788A9D59798A9E5967
:100DB000A4E69F597A8AA0597B8AA1597C8AA259B4
:100DC0007D8AA359FEE5A459A5E6A559D7CDA65914
:100DD0007E8AA759808AA859C1B7A959FCE5AA59A2
:100DE000FDE5AB59A3E6AC59818AAD59828AAE596B
:100DF000DDC4AF59A8E6B059838AB159848AB25983
:100E0000A7E6B359858AB459868AB559878AB659EF
:100E1000888AB759898AB8598A8AB959C3C3BA59CD
:100E20008B8ABB59DEC6BC598C8ABD598D8ABE5986
:100E3000AAE6BF598E8AC0598F8AC159908AC25971
:100E4000918AC359928AC459938AC559948AC659BA
:100E5000B7C4C759958AC859968AC959978ACA5931
:100E6000A2E6CB59BCCACC59988ACD59998ACE5999
:100E70009A8ACF599B8AD059E3BDD159C3B9D25967
:100E8000A6E6D359D5D0D459AFCED5599C8AD659D8
:100E90009D8AD759A9E6D859B0E6D9599E8ADA5918
:100EA000A6D2DB599F8ADC59AABDDD59ADE6DE59D1
:100EB000A08ADF59A18AE059A28AE159A38AE2599E
:100EC000A48AE359AFE6E459A58AE559D1C0E659A9
:100ED000A68AE759A78AE859CCD2E959A88AEA59DB
:100EE000A98AEB59AA8AEC59A7BCED59AB8AEE59ED
:100EF000AC8AEF59AD8AF059AE8AF159AF8AF259EE
:100F0000B08AF359B18AF459B28AF559B38AF659BD
:100F1000B48AF759B58AF859B68AF959B1E6FA5937
:100F2000B78AFB59F6D2FC59B88AFD59B98AFE59DD
:100F3000BA8AFF59CBD7005ABB8A015AFECD025A52
:100F4000BC8A035ADECD045AA6C2055AABE6065A3D
:100F5000ACE6075ABFBD085AAEE6095AB3E60A5ACC
:100F6000BD8A0B5ABE8A0C5AB2E60D5ABF8A0E5A77
:100F7000C08A0F5AC18A105AC28A115AB6E6125A4A
:100F8000C38A135AB8E6145AC48A155AC58A165A1F
:100F9000C68A175AC78A185AEFC4195AC88A1A5AE1
:100FA000C98A1B5ACA8A1C5AC8C41D5ACB8A1E5ADF
:100FB000CC8A1F5AEABE205AEFC9215ACD8A225A3A
:100FC000CE8A235AB7E6245ACF8A255AF0B6265A33
:100FD000D08A275AD18A285AD28A295AE4C32A5A4F
:100FE000D38A2B5AD48A2C5AD58A2D5AD68A2E5A6D
:100FF000D78A2F5AD88A305AD98A315AE9D3325AE5
:10100000B4E6335ADA8A345AB5E6355ADB8A365AA8
:10101000A2C8375ADC8A385ADD8A395ADE8A3A5AE7
:10102000DF8A3B5AE08A3C5ABDE63D5AE18A3E5A85
:10103000E28A3F5AE38A405AB9E6415AE48A425A60
:10104000E58A435AE68A445AE78A455AE88A465A64
:10105000C5C6475AE98A485AEA8A495AF1CD4A5AD6
:10106000BBE64B5AEB8A4C5AEC8A4D5AED8A4E5AE3
:10107000EE8A4F5AEF8A505AF08A515AF18A525AE0
:10108000F28A535AF38A545AF48A555ABCE6565A8D
:10109000F58A575AF68A585AF78A595AF88A5A5A84
:1010A000E9BB5B5AF98A5C5AFA8A5D5AFB8A5E5A36
:1010B000FC8A5F5AFD8A605AFE8A615A408B625AE6
:1010C000BEE6635A418B645A428B655A438B665A1B
:1010D000448B675ABAE6685A458B695A468B6A5AF6
:1010E000B7C06B5A478B6C5A488B6D5A498B6E5AF6
:1010F0004A8B6F5A4B8B705A4C8B715A4D8B725A6C
:101100004E8B735A4F8B745AA4D3755ABFE6765AD6
:10111000F4C9775AC3E6785A508B795A518B7A5A68
:10112000C4E67B5A528B7C5A538B7D5A548B7E5A21
:10113000558B7F5AF6D0805A568B815A578B825ADC
:10114000588B835A598B845A5A8B855A5B8B865A93
:101150005C8B875A5D8B885A5E8B895A5F8B8A5A63
:10116000608B8B5A618B8C5A628B8D5A638B8E5A33
:10117000648B8F5A658B905A668B915A678B925A03
:10118000BDC3935A688B945A698B955A6A8B965A49
:101190006B8B975A6C8B985A6D8B995A6E8B9A5AA7
:1011A000C4C39B5AC2E69C5A6F8B9D5A708B9E5A41
:1011B000718B9F5A728BA05A738BA15A748BA25A4F
:1011C000758BA35A768BA45A778BA55A788BA65A1F
:1011D000798BA75A7A8BA85A7B8BA95A7C8BAA5AEF
:1011E000C1E6AB5A7D8BAC5A7E8BAD5A808BAE5A22
:1011F000818BAF5A828BB05A838BB15A848BB25A8F
:10120000C7E6B35AB1CFB45A858BB55AF4EBB65A88
:10121000868BB75A878BB85ACAE6B95A888BBA5A9E
:10122000898BBB5A8A8BBC5A8B8BBD5A8C8BBE5A0E
:10123000C5E6BF5A8D8BC05A8E8BC15ADEBCC25ACE
:10124000A9C9C35A8F8BC45A908BC55A918BC65A61
:10125000928BC75A938BC85A948BC95AB5BCCA5A39
:10126000958BCB5A968BCC5AD3CFCD5A978BCE5ADF
:10127000988BCF5A998BD05A9A8BD15A9B8BD25A32
:10128000C8E6D35A9C8BD45AC9E6D55A9D8BD65AF8
:10129000CEE6D75A9E8BD85AD0E6D95A9F8BDA5AC7
:1012A000A08BDB5AA18BDC5AD1E6DD5AA28BDE5A29
:1012B000A38BDF5AA48BE05ACBE6E15AD5B5E25AAC
:1012C000A58BE35ACCE6E45AA68BE55AA78BE65ADF
:1012D000CFE6E75AA88BE85AA98BE95ADBC4EA5A49
:1012E000AA8BEB5AC6E6EC5AAB8BED5AAC8BEE5A96
:1012F000AD8BEF5AAE8BF05AAF8BF15ACDE6F25A66
:10130000B08BF35AB18BF45AB28BF55AB38BF65AB1
:10131000B48BF75AB58BF85AB68BF95AB78BFA5A81
:10132000B88BFB5AB98BFC5ABA8BFD5ABB8BFE5A51
:10133000BC8BFF5ABD8B005BBE8B015BBF8B025B1E
:10134000C08B035BC18B045BC28B055BC38B065BED
:10135000C48B075BC58B085BC68B095BD2E60A5B57
:10136000C78B0B5BC88B0C5BC98B0D5BCA8B0E5B91
:10137000CB8B0F5BCC8B105BCD8B115BCE8B125B61
:10138000CF8B135BD08B145BD18B155BD28B165B31
:10139000D4E6175BD3E6185BD38B195BD48B1A5B4F
:1013A000D58B1B5BD68B1C5BD78B1D5BD88B1E5BD9
:1013B000D98B1F5BDA8B205BDB8B215BDC8B225BA9
:1013C000DD8B235BDE8B245BDF8B255BE08B265B79
:1013D000E18B275BE28B285BE38B295BE48B2A5B49
:1013E000E58B2B5BE68B2C5BE78B2D5BE88B2E5B19
:1013F000E98B2F5BEA8B305BEB8B315BEC8B325BE9
:10140000D5E6335BED8B345BF8D9355BEE8B365B21
:10141000EF8B375BD6E6385BF08B395BF18B3A5B51
:10142000F28B3B5BF38B3C5BF48B3D5BF58B3E5B64
:10143000F68B3F5BF78B405BD7E6415BF88B425BFB
:10144000F98B435BFA8B445BFB8B455BFC8B465B08
:10145000FD8B475BFE8B485B408C495B418C4A5B54
:10146000428C4B5B438C4C5B448C4D5B458C4E5BA0
:10147000468C4F5B478C505BD3D7515BDDE6525BAC
:10148000488C535BDEE6545BD7BF555BD0D4565BCC
:10149000498C575BD6D7585BE6B4595BEFCB5A5BA8
:1014A000DAE65B5BC3D85C5BCED75D5BA2D05E5BEC
:1014B0004A8C5F5BCFC3605B4B8C615B4C8C625B27
:1014C000DFE6635BBEBC645BC2B9655BDBE6665BA3
:1014D000A7D1675B4D8C685B4E8C695BA2BA6A5B77
:1014E000CFC26B5B4F8C6C5BABD86D5B508C6E5B13
:1014F000518C6F5B528C705BEBCA715BEEE5725B7B
:10150000538C735BDCE6745B548C755BF5B7765B70
:10151000558C775B568C785B578C795B588C7A5BF3
:10152000E6C87B5B598C7C5B5A8C7D5BF5C47E5B2B
:101530005B8C7F5B5C8C805BB2E5815BFEC4825B15
:101540005D8C835BFCCB845BB3E5855BACD5865B54
:101550005E8C875BEED3885BD8CA895BB2B08A5B4E
:101560005F8C8B5BCECB8C5BEACD8D5B608C8E5BB6
:10157000618C8F5BEABA905B628C915B638C925B4F
:10158000648C935BB5E5945B658C955BB4E5965B89
:10159000668C975BDAD7985BD9B9995BE6D69A5B8C
:1015A000A8B69B5BF0CD9C5BCBD29D5BA6B19E5B4E
:1015B000B5CA9F5B678CA05BE8B3A15BF3C9A25B74
:1015C000CDBFA35BFBD0A45BD2CAA55BB6E5A65B8F
:1015D000C2BBA75B688CA85B698CA95B6A8CAA5BA1
:1015E000DCCFAB5BACB9AC5B6B8CAD5B6C8CAE5BDE
:1015F0006D8CAF5B6E8CB05BD7D4B15B6F8CB25B24
:10160000708CB35BA6BAB45BE7D1B55BFCCFB65BBD
:10161000D2BCB75B718CB85BB7E5B95BDDC8BA5BB0
:10162000728CBB5B738CBC5B748CBD5BEDBFBE5BB3
:10163000F6B1BF5BDECBC05B758CC15B768CC25BE9
:10164000C5BCC35B778CC45BC4BCC55BFAD2C65B4C
:10165000DCC3C75BDCBFC85B788CC95B798CCA5BB9
:101660007A8CCB5B7B8CCC5BBBB8CD5B7C8CCE5B54
:101670007D8CCF5B7E8CD05BC2C3D15B808CD25B18
:10168000AEBAD35BA2D4D45B818CD55B828CD65BA3
:10169000838CD75B848CD85B858CD95B868CDA5B3A
:1016A000878CDB5B888CDC5B898CDD5BDEC7DE5B7B
:1016B000AFC4DF5BECB2E05B8A8CE15BD1B9E25B8B
:1016C0008B8CE35B8C8CE45BBBE5E55BC8C1E65BC4
:1016D0008D8CE75B8E8CE85BAFD5E95B8F8CEA5B2A
:1016E000908CEB5B918CEC5B928CED5B938CEE5B66
:1016F000BCE5EF5B948CF05BBEE5F15B958CF25B37
:10170000968CF35B978CF45B988CF55B998CF65B0D
:101710009A8CF75B9B8CF85BE7B4F95BD4B6FA5B09
:10172000C2CBFB5BB0D1FC5BBCB5FD5B9C8CFE5BB4
:101730009D8CFF5BD9CA005C9E8C015CE2B7025CA9
:101740009F8C035CA08C045CE4C9055CA18C065CE6
:10175000ABBD075CA28C085CA38C095CBECE0A5CA6
:10176000F0D70B5CA48C0C5CA58C0D5CA68C0E5C7D
:10177000A78C0F5CA1D0105CA88C115CD9C9125C3D
:10178000A98C135CAA8C145CFBB6155CD8E6165CBD
:10179000E2BC175CAB8C185CBEB3195CAC8C1A5CF9
:1017A000D0C91B5CAD8C1C5CD9E61D5CA2B31E5C71
:1017B000AE8C1F5CAF8C205CB08C215CB18C225C49
:1017C000CCDE235CB28C245CC8D3255CCDDE265CE9
:1017D000B38C275CA2D2285CB48C295CB58C2A5CC3
:1017E000B68C2B5CB78C2C5CCEDE2D5CB88C2E5C62
:1017F000B98C2F5CBA8C305CBB8C315CCDBE325C5A
:10180000BC8C335CBD8C345CCFDE355CBE8C365C0E
:10181000BF8C375CC08C385CACCA395CFCD23A5C9B
:10182000DFB33B5CEAE53C5CE1C43D5CA1BE3E5CF1
:10183000B2CE3F5CF2C4405CD6BE415CA8C6425CFE
:10184000E3B2435CC18C445CC28C455CD3BE465C55
:10185000C38C475CC48C485CFCC7495CEBCC4A5CDD
:10186000ECBD4B5CDDCE4C5CC58C4D5CC68C4E5CDF
:10187000BACA4F5CC1C6505CECE5515CBCD0525C4E
:10188000C78C535CC88C545CC98C555CB9D5565C0C
:10189000CA8C575CCB8C585CCC8C595CEDE55A5C9F
:1018A000CD8C5B5CCE8C5C5CCF8C5D5CD08C5E5CEC
:1018B000F4CA5F5CD18C605CC0CD615CC5C2625C07
:1018C000D28C635CEFE5645CD38C655CC4C2665CFF
:1018D000F0E5675CD48C685CD58C695CD68C6A5CFE
:1018E000D78C6B5CD88C6C5CD98C6D5CDA8C6E5C44
:1018F000F8E56F5CCDCD705CDB8C715CBDC9725C52
:10190000DC8C735CDD8C745CDE8C755CDF8C765CEF
:10191000E08C775CE18C785CE28C795CD9D27A5C83
:10192000A8E17B5CE38C7C5CE48C7D5CE58C7E5C7C
:10193000E68C7F5CECD3805CE78C815CEACB825CDC
:10194000F1C6835CE88C845CE98C855CEA8C865CFF
:10195000EB8C875CEC8C885CACE1895CED8C8A5C00
:10196000EE8C8B5CEF8C8C5CA7E18D5CA9E18E5CCE
:10197000F08C8F5CF18C905CAAE1915CAFE1925CA1
:10198000F28C935CF38C945CEDB2955CF48C965C79
:10199000ABE1975CDAB8985CADE1995CAEE19A5C3A
:1019A000B0E19B5CBAB59C5CB1E19D5CF58C9E5C42
:1019B000F68C9F5CF78CA05CF88CA15CF98CA25C27
:1019C000B3E1A35CB8E1A45CFA8CA55CFB8CA65CDB
:1019D000FC8CA75CFD8CA85CFE8CA95CD2D1AA5CB7
:1019E000408DAB5CB6E1AC5CB5E1AD5CEBC1AE5C2F
:1019F000418DAF5C428DB05C438DB15CB7E1B25CB0
:101A0000448DB35CC0D4B45C458DB55CB2E1B65CCA
:101A1000468DB75CBAE1B85CB6B0B95C478DBA5CCC
:101A2000488DBB5C498DBC5C4A8DBD5CB4E1BE5C3D
:101A30004B8DBF5CF9BFC05C4C8DC15CB9E1C25C31
:101A40004D8DC35C4E8DC45CBBE1C55C4F8DC65CE7
:101A5000508DC75C518DC85C528DC95C538DCA5C7A
:101A6000548DCB5CBEE1CC5C558DCD5C568DCE5C8F
:101A7000578DCF5C588DD05C598DD15C5A8DD25C1E
:101A8000BCE1D35C5B8DD45C5C8DD55C5D8DD65C3C
:101A90005E8DD75C5F8DD85C608DD95CC5D6DA5C15
:101AA000618DDB5C628DDC5C638DDD5C648DDE5C96
:101AB000658DDF5C668DE05C678DE15CBFCFE25CCD
:101AC000688DE35C698DE45CBDE1E55CBFE1E65CEB
:101AD000CDC2E75C6A8DE85CEBB6E95C6B8DEA5CD5
:101AE000F8D3EB5C6C8DEC5C6D8DED5CCDC7EE5C82
:101AF0006E8DEF5C6F8DF05CE5B7F15C708DF25C24
:101B0000718DF35C728DF45C738DF55C748DF65C95
:101B1000758DF75C768DF85C778DF95C788DFA5C65
:101B2000798DFB5CFEBEFC5C7A8DFD5C7B8DFE5C82
:101B30007C8DFF5C7D8D005D7E8D015D808D025D05
:101B4000C0E1035DC1E1045D818D055D828D065DAF
:101B5000C7E1075DE7B3085D838D095D848D0A5D8C
:101B6000858D0B5D868D0C5D878D0D5D888D0E5D81
:101B7000E9C60F5D898D105D8A8D115D8B8D125DBB
:101B80008C8D135D8D8D145DDEB4155D8E8D165DAF
:101B9000C2D1175D8F8D185D908D195D918D1A5D85
:101BA000928D1B5DC8E11C5D938D1D5D948D1E5D46
:101BB000C6E11F5D958D205D968D215D978D225D1F
:101BC000988D235D998D245DC5E1255D9A8D265DF7
:101BD000C3E1275DC2E1285D9B8D295DC0B12A5D0F
:101BE0009C8D2B5D9D8D2C5D9E8D2D5DB8D52E5DC4
:101BF000C4E12F5D9F8D305DA08D315DA18D325D83
